:100000000C94F24B0C94134C0C9448D50C94134C58
:100010000C94134C0C94134C0C94134C0C94134CE4
:100020000C94134C0C94134C0C94134C0C9473D7E9
:100030000C94134C0C94134C0C9469B80C94134C02
:100040000C94134C0C94134C0C94134C0C94134CB4
:100050000C94134C0C94134C0C94134C0C94134CA4
:100060000C94134C0C9462D50C94F1D40C94134C56
:100070000C94B8CE0C945ACE0C9496CE0C94134C8F
:100080000C9413D60C94134C0C94134C0C94134CEA
:100090000C94134C0C94134C0C94134C0C94134C64
:1000A0000C94134C0C94134C0C94134C0C9444BFB0
:1000B0000C94E8BF0C94134C0C94134C0C945ABA47
:1000C0000C94134C0C94134C0C94134C0C94134C34
:1000D0000C94134C0C94134C0C94134C0C94134C24
:1000E0000C94DFA90C94134C0C94134C0C94134CEB
:1000F0000C94134C0C94134C0C94134C0C94134C04
:100100000C941BBF0C94BFBF0C94F2BE0C9496BF12
:100110000C94134C0C94134C0C94134C0C94134CE3
:100120000C94134C0C94134C0C94134C0C94134CD3
:100130000C94134C0C94BEB90C94134C0C94134CAB
:100140000C94134C0C94134C0C94134C0C94134CB3
:100150000C94134C0C94134C0C94D5A90C94134C84
:100160000C94134C0C94134C0C94134C0C94134C93
:100170000C94134C0C94134C0C94134C0C94134C83
:100180000C94134C0C94134C0C94134C0C94134C73
:100190000C94134C0C94134C0C94134C0C94134C63
:1001A0000C946DBF0C9411C00C94134C0C94134C14
:1001B0000C940CBA0C94134C0C94134C0C94134CDC
:1001C0000C94134C0C94134C0C94134C0C94134C33
:1001D0000C94134C0C94134C0C94134C0C94134C23
:1001E0000C94134C0C94134C6C75767580758A7551
:1001F0009575997B997B997B997B997B9B75997B6D
:10020000997B997B997B997B997B9D75A775B17536
:10021000BB75C575997B997B997B997B997B997BFC
:10022000CF75997B2576997B997B997B997B997B77
:10023000997B997B6476997B8079997B997B997B73
:10024000997B997B997B997B997B8079997B997B29
:10025000997B91769676A076AA76AC76B676C176BC
:10026000997BCC76997B997B0977997B997B997B54
:10027000997B997B997B997B997B997B997B997BDE
:10028000997B997B997B997B1377997B997B997B58
:10029000997B997B997B997B997B997B1D775A7781
:1002A0009777E077EA77037803780D7817782178E5
:1002B0002B7835783A7844784E78977B977B977B84
:1002C000977B977B977B977B977B977B977B977B9E
:1002D000977B977B977B977B977B977B977B977B8E
:1002E000977B0D78977B977B977B977B977B977B0B
:1002F000977B977B977B977B977B977B977B977B6E
:10030000977B977B977B587862786C787678977B29
:10031000977B977B977B977B977B977B977B0378E4
:10032000247BE57AE97AF17ACD7AD17AD97ADD7AC5
:10033000FD7A107B187B1C7B207B7C7BF57AF17827
:1003400002791379997B997B8B785D75997B2479F8
:10035000357946798079F4776879997B9C78997BAF
:100360005779AD788078997B997B997BBE78CF78E7
:10037000E0788BBE93BE9BBEA3BEABBEB3BEBBBE7E
:10038000C3BEB6C113C11BC123C12BC133C13BC105
:1003900043C14BC153C15BC163C16BC173C17BC15D
:1003A0009BC19BC19BC19BC19BC19BC19BC19BC16D
:1003B0009BC19BC19BC19BC19BC19BC19BC19BC15D
:1003C0009BC19BC19BC19BC19BC19BC19BC19BC14D
:1003D0009BC19BC19BC19BC19BC19BC19BC19BC13D
:1003E0009BC19BC19BC183C18BC19BC19BC19BC155
:1003F0009BC19BC19BC19BC19BC19BC19BC19BC11D
:100400009BC19BC19BC19BC19BC19BC19BC19BC10C
:100410009BC19BC19BC19BC19BC19BC19BC19BC1FC
:100420009BC19BC19BC19BC19BC19BC19BC19BC1EC
:100430009BC19BC19BC19BC19BC19BC19BC19BC1DC
:100440009BC19BC19BC19BC193C1084AD73B3BCE7B
:10045000016E84BCBFFDC12F3D6C74319ABD5683C3
:100460003DDA3D00C77F11BED9E4BB4C3E916BAA7B
:10047000AABE000000803F05A84CCDB2D44EB938CA
:1004800036A9020C50B9918688083CA6AAAA2ABEB1
:10049000000000803F07634236B79BD8A71A39682F
:1004A0005618AEBAAB558C1D3CB7CC5763BD6DED3D
:1004B000FD753EF6177231BF000000803F08000056
:1004C00000BE922449123EABAAAA2ABECDCCCC4C87
:1004D0003E00000080BEABAAAAAA3E00000000BFFA
:1004E000000000803F0000000000084178D3BB43BB
:1004F00087D1133D190E3CC3BD4282AD2B3E68EC43
:100500008276BED98FE1A93E4C80EFFFBE01C4FFC9
:100510007F3F0000000000000C9495B10C941F5B1D
:100520000C948BC10C94315B0C94EB670C9474C5E8
:100530000C949ECB0C9434AB0C94E97A0C947678A2
:100540000C94CDD10C94C3BE0C94DF5E0C949176C8
:100550000C943EBE0C9493C10C94D95F0C94207BF8
:100560000C9424790C94B75E0C94375B0C94E2D213
:100570000C94BB5E0C94A7750C9462BE0C947BC16A
:100580000C9468790C94A55F0C947E6C0C94346286
:100590000C94A3BE0C94294C0C946C750C945BC108
:1005A0000C94C6C50C941F4C0C94485B0C94DB5DFA
:1005B0000C9453630C94EB5E0C94CF5B0C94E3C0EF
:1005C0000C94154C0C9488610C9440AB0C94B17550
:1005D0000C94BB750C94B6C10C9491B10C94AC61A5
:1005E0000C946AC60C94B7670C94035E0C94CF5EAF
:1005F0000C9416680C94DB5E0C94C55F0C94255B20
:100600000C9483C10C944E780C94675B0C9455B198
:100610000C94297E0C9456BE0C94C4720C943B9698
:100620000C94E0780C94A0760C94C15F0C941A5F43
:100630000C94BBBE0C94885B0C94864F0C948A750A
:100640000C94F5CD0C94D75E0C94685C0C94AC764D
:100650000C94F55D0C94125B0C94E75E0C94BD5FFA
:100660000C94E45C0C944BC10C9471B10C94535BEE
:100670000C9480750C94F3620C946B580C942B5B67
:100680000C945A710C9446790C94EF5E0C949C78FF
:100690000C94F1780C9464670C94B15F0C945EBE7A
:1006A0000C9496680C9442BE0C947E6F0C94497D19
:1006B0000C94A15B0C94395F0C9406880C94725BCB
:1006C0000C94FB5E0C9462830C94684C0C948DB17A
:1006D0000C94AF5E0C94D17C0C949BBE0C94357939
:1006E0000C943E5C0C942CAB0C9407CE0C9440B153
:1006F0000C942DD20C945A770C949D750C94ABBE2F
:100700000C9403780C94EDB20C9462780C94316CD8
:100710000C9463C10C94FCAF0C9495750C9499B136
:100720000C94247B0C94F8AF0C9406730C945C67C7
:100730000C94CF750C94D15C0C9402790C9447BE48
:100740000C9444AB0C94AB6C0C9491D40C94DDC021
:100750000C94AA760C94F6AF0C94305E0C94866FD1
:100760000C9468670C94B6760C9413770C94C35E63
:100770000C942BC10C94C06C0C94FDBC0C9428AB55
:100780000C940A5E0C94E57A0C9435780C943D72C6
:100790000C946BC10C940D780C94E3BD0C943CABA1
:1007A0000C94C95F0C94187B0C94D37D0C946067F7
:1007B0000C94A15F0C94115E0C947C7B0C9453C13F
:1007C0000C94E0770C94794C0C948FBD0C9464617C
:1007D0000C942B780C94AD780C940A610C94517D98
:1007E0000C94EA770C94CD7A0C9423C10C940C628F
:1007F0000C94D1830C94E15F0C94CA620C94AA5DB2
:100800000C94EB7B0C94947D0C941A630C94C5753A
:100810000C94977B0C94CDD00C94DD5F0C940E62FD
:100820000C94CB5E0C9413790C94CC760C94EB6BFB
:100830000C9459CB0C94E0640C9464760C9475C5BC
:100840000C94C4B20C94D17A0C945D750C94DD7A3E
:100850000C94AC850C9476750C94997B0C948B78E5
:100860000C94297D0C9475CD0C94316D0C944F5ED5
:100870000C9496760C94D3610C9497770C94217811
:100880000C94A3620C9417780C9457790C94F1BCD7
:100890000C9446D30C94BE780C947BBD0C949BC1F5
:1008A0000C9459620C94075C0C94AB5E0C946061E0
:1008B0000C94C1760C94BD660C940BBE0C946C78B1
:1008C0000C94B35E0C94BCAF0C94ED5F0C94BF5EC3
:1008D0000C94BEAF0C94F85F0C9433C10C949D67DC
:1008E0000C94D35E0C94A1660C94A9C50C94A9BD7C
:1008F0000C948BBE0C943ABE0C940B670C947E62E5
:100900000C941BC10C94F35E0C9480780C945C5B8B
:100910000C947D5B0C9493BE0C94FDC00C94CD5F45
:100920000C94525D0C946C670C9496CD0C94247DC1
:100930000C94557D0C943D5B0C94686B0C94FBCF30
:100940000C94FE7D0C9464D20C94E35E0C94B3BEC4
:100950000C9424AB0C9413C10C94F57A0C945ABEED
:100960000C94D5830C9443C10C943A780C9458722F
:100970000C9438AB0C94F4770C9473C10C94597D9F
:100980000C9408CD0C9480790C9456680C9461D129
:100990000C948DC50C94FF520C94D55F0C94AD5FF4
:1009A0000C945C5F0C94C75E0C94D65D0C94F75E5F
:1009B0000C943BC10C94B55F0C94D15F0C940977F7
:1009C0000C943D5F0C94CF780C94D97A0C94107BE6
:1009D0000C94D1670C94B85B0C94FD7A0C9430ABFA
:1009E0000C9401C10C941D770C94606C0C94F17AFA
:1009F0000C949B750C94B95F0C94A95F0C94D983EB
:100A00000C944D7D0C9444780C94C0AF0C94A15C74
:100A10000C9458780C94DB7B0C94FC5D0C9425763C
:100A20000C94E5BC0C9448AB0C941C7B0C942DAC42
:100A30005B257325735D20257320257320706F73EC
:100A40006974696F6E2531382E336625730A005B31
:100A5000257325735D202573202573206F666673CB
:100A600065742532302E336625730A005B257325A5
:100A7000735D202573207A65726F206261636B6FEE
:100A800066662531392E336625730A005B2573258A
:100A9000735D202573206C61746368206261636BF1
:100AA0006F66662531382E336625730A005B257321
:100AB00025735D202573206C617463682076656CF6
:100AC0006F636974792531332E306625732F6D6914
:100AD0006E0A005B257325735D20257320736561A5
:100AE0007263682076656C6F636974792531322E84
:100AF000306625732F6D696E0A005B257325735D63
:100B000020257320737769746368206D61782531BF
:100B10003764205B303D6F66662C313D686F6D69D0
:100B20006E672C323D6C696D69742C333D6C696D58
:100B300069742B686F6D696E675D0A005B257325AC
:100B4000735D20257320737769746368206D696E07
:100B500025313764205B303D6F66662C313D686F10
:100B60006D696E672C323D6C696D69742C333D6C18
:100B7000696D69742B686F6D696E675D0A005B252E
:100B80007325735D20257320726164697573207607
:100B9000616C75652532302E346625730A005B253D
:100BA0007325735D202573206A756E6374696F6E9B
:100BB00020646576696174696F6E2531342E346600
:100BC000257320286C6172676572206973206661E5
:100BD00073746572290A005B257325735D20257384
:100BE000206A65726B20686F6D696E672531362EDD
:100BF000306625732F6D696E5E33202A2031206D9B
:100C0000696C6C696F6E0A005B257325735D202526
:100C100073206A65726B206D6178696D756D253121
:100C2000352E306625732F6D696E5E33202A203194
:100C3000206D696C6C696F6E0A005B257325735DAE
:100C40002025732074726176656C206D696E696D04
:100C5000756D2531372E336625730A005B257325A4
:100C6000735D2025732074726176656C206D6178E8
:100C7000696D756D2531372E336625730A005B2546
:100C80007325735D2025732076656C6F63697479B5
:100C9000206D6178696D756D2531312E3066257353
:100CA0002F6D696E0A005B257325735D2025732007
:100CB0006665656472617465206D6178696D756DD6
:100CC0002531312E306625732F6D696E0A005B2544
:100CD0007325735D2025732061786973206D6F64BF
:100CE00065253138642025730A005B6D615D202025
:100CF0006D696E20617263207365676D656E742522
:100D000031382E336625730A005B736C5D202073C7
:100D10006F6674206C696D697420656E61626C65C4
:100D2000253132640A005B63745D202063686F7252
:100D300064616C20746F6C6572616E636525313718
:100D40002E346625730A005B6A615D20206A756E29
:100D50006374696F6E20616363656C657261746949
:100D60006F6E25382E306625730A005B6764695DF7
:100D70002064656661756C742067636F64652064C8
:100D8000697374616E6365206D6F646525326420DC
:100D90005B303D4739302C313D4739315D0A005BCE
:100DA0006770615D2064656661756C742067636F50
:100DB0006465207061746820636F6E74726F6C2557
:100DC0003364205B303D4736312C313D4736312E80
:100DD000312C323D4736345D0A005B67636F5D201E
:100DE00064656661756C742067636F646520636F0A
:100DF0006F72642073797374656D253364205B3181
:100E00002D3620284735342D473539295D0A005BBA
:100E100067756E5D2064656661756C742067636FCD
:100E2000646520756E697473206D6F646525356423
:100E3000205B303D4732302C313D4732315D0A0076
:100E40005B67706C5D2064656661756C74206763B8
:100E50006F646520706C616E6525313064205B3095
:100E60003D4731372C313D4731382C323D47313900
:100E70005D0A00256320776F726B206F666673656D
:100E8000743A2531322E336625730A002563206DAE
:100E9000616368696E6520706F736E3A2531312E1B
:100EA000336625730A00256320706F736974696F58
:100EB0006E3A2531352E336625730A00546F6F6CF8
:100EC000206E756D62657220202020202020202059
:100ED0002025640A00466565642072617465206D92
:100EE0006F64653A20202020202025730A00446981
:100EF0007374616E6365206D6F64653A20202020F5
:100F000020202025730A0050617468204D6F6465AD
:100F10003A202020202020202020202025730A0095
:100F2000506C616E653A2020202020202020202057
:100F3000202020202025730A004D6F74696F6E20D9
:100F40006D6F64653A20202020202020202025730A
:100F50000A00436F6F7264696E6174652073797300
:100F600074656D3A20202025730A00556E697473EC
:100F70003A20202020202020202020202020202057
:100F800025730A00486F6D696E672073746174651C
:100F90003A202020202020202025730A0046656565
:100FA00064686F6C642073746174653A202020203B
:100FB000202025730A004D6F74696F6E2073746171
:100FC00074653A202020202020202025730A004329
:100FD00079636C652073746174653A202020202049
:100FE0002020202025730A00526177206D616368FC
:100FF000696E652073746174653A20202025730A38
:10100000004D616368696E652073746174653A2090
:1010100020202020202025730A004C696E65206E58
:10102000756D6265723A2531302E30660A0046656C
:10103000656420726174653A2531362E33662573F6
:101040002F6D696E0A0056656C6F636974793A2575
:1010500031372E336625732F6D696E0A00B4108305
:10106000106310473935202D20756E6974732D700B
:1010700065722D7265766F6C7574696F6E206D6F19
:10108000646500473934202D20756E6974732D70A6
:1010900065722D6D696E757465206D6F64652028AD
:1010A000692E652E206665656472617465206D6FBA
:1010B00064652900473933202D20696E7665727387
:1010C000652074696D65206D6F646500F010D01047
:1010D000473931202D20696E6372656D656E7461CC
:1010E0006C2064697374616E6365206D6F64650064
:1010F000473930202D206162736F6C7574652064F0
:10110000697374616E6365206D6F646500411129B8
:10111000111311473634202D20636F6E74696E757C
:101120006F7573206D6F6465004736312E31202D49
:101130002065786163742073746F70206D6F6465CF
:1011400000473631202D206578616374207061740A
:1011500068206D6F6465007B116C115D114731393A
:10116000202D20595A20706C616E6500473138205F
:101170002D20585A20706C616E6500473137202D44
:1011800020585920706C616E65000712F511DC1152
:10119000BB119411473830202D2063616E63656C5C
:1011A000206D6F74696F6E206D6F646520286E6F9F
:1011B0006E65206163746976652900473320202DB0
:1011C00020636F756E74657220636C6F636B7769F3
:1011D0007365206172632066656564004732202074
:1011E0002D20636C6F636B77697365206172632078
:1011F0006665656400473120202D206C696E65614D
:1012000072206665656400473020202D206C696E71
:1012100065617220747261766572736520287365EA
:10122000656B2900CE12B4129A12801266124C120B
:101230003212473539202D20636F6F7264696E61F9
:1012400074652073797374656D20360047353820D6
:101250002D20636F6F7264696E617465207379739A
:1012600074656D203500473537202D20636F6F7210
:1012700064696E6174652073797374656D203400E0
:10128000473536202D20636F6F7264696E61746517
:101290002073797374656D203300473535202D2018
:1012A000636F6F7264696E617465207379737465BE
:1012B0006D203200473534202D20636F6F726469D2
:1012C0006E6174652073797374656D2031004735E4
:1012D00033202D206D616368696E6520636F6F72C6
:1012E00064696E6174652073797374656D000113B0
:1012F000FB12F412486F6D696E6700486F6D65648C
:10130000004E6F7420486F6D656400351330132BE9
:1013100013251320131713456E6420486F6C640067
:10132000486F6C6400446563656C00506C616E00CE
:1013300053796E63004F666600481344133F1348A9
:101340006F6C640052756E0053746F700072136896
:101350001362135B1357134A6F6700486F6D696E12
:10136000670050726F6265004D616368696E696EF7
:1013700067004F666600A813A2139C13971393137C
:101380008D13841353687574646F776E00437963AB
:101390006C6500456E640053746F7000416C61723F
:1013A0006D00526561647900496E697469616C69A8
:1013B0007A696E67000B140514FF13FA13F613F223
:1013C00013ED13E713E113DA13D613CD1353687536
:1013D00074646F776E004A6F6700486F6D696E675F
:1013E000004379636C650050726F626500486F6CF2
:1013F000640052756E00456E640053746F70004156
:101400006C61726D00526561647900496E6974693E
:10141000616C697A696E670032141C14473231209E
:101420002D206D696C6C696D65746572206D6F64DB
:101430006500473230202D20696E63686573206D2A
:101440006F6465006C14611455144C145B72616414
:101450006975735D005B696E686962697465645D76
:10146000005B7374616E646172645D005B646973D8
:1014700061626C65645D00861482147D142064656D
:101480006700206D6D0020696E002A2A2A204E4FC9
:1014900054494345202A2A2A205265736574746989
:1014A0006E672062617564207261746520746F20BC
:1014B0002573005B626175645D2055534220626153
:1014C0007564207261746525313564205B313D3966
:1014D0003630302C323D31393230302C333D3338D8
:1014E0003430302C343D35373630302C353D3131C9
:1014F000353230302C363D3233303430305D0A00F6
:101500005B72786D5D2073657269616C2052582042
:101510006D6F646525313564205B303D7374726591
:10152000616D696E675F6D6F64652C313D6C696ECE
:10153000655F6D6F64655D0A005B65785D202065A1
:101540006E61626C6520666C6F7720636F6E74727B
:101550006F6C25313064205B303D6F66662C313D09
:10156000584F4E2F584F46462C323D5254532F431E
:1015700054535D0A005B65655D2020656E61626C99
:1015800065206563686F25313864205B303D6F6688
:10159000662C313D6F6E5D0A005B65635D202065E2
:1015A0007870616E64204C4620746F2043524C4624
:1015B000206F6E205458253664205B303D6F666680
:1015C0002C313D6F6E5D0A00FB15F615F015EA151E
:1015D000E415DD15D6153233303430300031313575
:1015E0003230300035373630300033383430300068
:1015F0003139323030003936303000300073797391
:10160000006662000000000702497DD3610C620899
:101610003B291CDC437379730066760000000007E9
:10162000034D7DD3610C620C3BEC51783F737973B1
:10163000006870000000000700517DD3611A631438
:101640003B0000803F73797300687600000000075C
:1016500000557DD361297D183B00000041737973EB
:10166000006964000000000400597DD17C0C620414
:101670003B00000000000000006E000000000001C0
:1016800000AB5EA15BCA62F83200000000000000FF
:10169000006C696E6500000100AB5EB85BCA62F861
:1016A00032000000000000000076656C00000000C1
:1016B00002115ECF5B0C62043B00000000000000E2
:1016C000006665656400000002305E075C0C620421
:1016D0003B00000000000000007374617400000013
:1016E00000AF5E125B0C62043B00000000000000D3
:1016F000006D61637300000000B35E1F5B0C620449
:101700003B000000000000000063796373000000EC
:1017100000B75E255B0C62043B0000000000000087
:10172000006D6F747300000000BB5E2B5B0C6204E5
:101730003B0000000000000000686F6C64000000C7
:1017400000BF5E315B0C62043B0000000000000043
:1017500000756E697400000000C75E3D5B0C62049A
:101760003B0000000000000000636F6F720000008B
:1017700000CB5E485B0C62043B00000000000000F0
:10178000006D6F6D6F00000000CF5E535B0C620454
:101790003B0000000000000000706C616E00000063
:1017A00000D35E5C5B0C62043B00000000000000A4
:1017B000007061746800000000D75E675B0C620413
:1017C0003B0000000000000000646973740000002A
:1017D00000DB5E725B0C62043B0000000000000056
:1017E0000066726D6F00000000DF5E7D5B0C6204BE
:1017F0003B0000000000000000746F6F6C000000F0
:1018000000E35E885B0C62043B000000006D706FBB
:10181000006D706F7800000003ED5F685C0C62047F
:101820003B000000006D706F006D706F790000006C
:1018300003ED5F685C0C62043B000000006D706F9C
:10184000006D706F7A00000003ED5F685C0C62044D
:101850003B000000006D706F006D706F6100000054
:1018600003ED5F685C0C62043B000000006D706F6C
:10187000006D706F6200000003ED5F685C0C620435
:101880003B000000006D706F006D706F6300000022
:1018900003ED5F685C0C62043B00000000706F7336
:1018A00000706F737800000003E15F3E5C0C62041F
:1018B0003B00000000706F7300706F7379000000D0
:1018C00003E15F3E5C0C62043B00000000706F733C
:1018D00000706F737A00000003E15F3E5C0C6204ED
:1018E0003B00000000706F7300706F7361000000B8
:1018F00003E15F3E5C0C62043B00000000706F730C
:1019000000706F736200000003E15F3E5C0C6204D4
:101910003B00000000706F7300706F736300000085
:1019200003E15F3E5C0C62043B000000006F6673E5
:10193000006F66737800000003F85FA15C0C62041E
:101940003B000000006F6673006F66737900000053
:1019500003F85FA15C0C62043B000000006F66733B
:10196000006F66737A00000003F85FA15C0C6204EC
:101970003B000000006F6673006F6673610000003B
:1019800003F85FA15C0C62043B000000006F66730B
:10199000006F66736200000003F85FA15C0C6204D4
:1019A0003B000000006F6673006F66736300000009
:1019B00003F85FA15C0C62043B00000000686F6DDF
:1019C00000686F6D6500000000C35E375BDB5D047F
:1019D0003B00000000686F6D00686F6D78000000CC
:1019E00000E15F64610C62CD3200000000686F6D41
:1019F00000686F6D7900000000E15F64610C62CEE9
:101A00003200000000686F6D00686F6D7A000000A2
:101A100000E15F64610C62CF3200000000686F6D0E
:101A200000686F6D6100000000E15F64610C62D0CE
:101A30003200000000686F6D00686F6D620000008A
:101A400000E15F64610C62D13200000000686F6DDC
:101A500000686F6D6300000000E15F64610C62D29A
:101A60003200000000707262007072626500000057
:101A70000074C564610C62D33200000000707262B1
:101A800000707262780000000374C5D3610C62D4E8
:101A90003200000000707262007072627900000013
:101AA0000374C5D3610C62D832000000007072620A
:101AB000007072627A0000000374C5D3610C62DCAE
:101AC00032000000007072620070726261000000FB
:101AD0000374C5D3610C62E03200000000707262D2
:101AE00000707262620000000374C5D3610C62E48E
:101AF00032000000007072620070726263000000C9
:101B00000374C5D3610C62E832000000006A6F679D
:101B1000006A6F67780000000074C56061F55DF2CF
:101B200032000000006A6F67006A6F67790000008A
:101B30000074C56061FC5DF232000000006A6F67EE
:101B4000006A6F677A0000000074C56061035EF28E
:101B500032000000006A6F67006A6F676100000072
:101B60000074C560610A5EF2320000000070777296
:101B700000707772310000000062BE8FBD0C6204FD
:101B80003B00000000707772007077723200000036
:101B90000062BE8FBD0C62043B00000000707772D3
:101BA00000707772330000000062BE8FBD0C6204CB
:101BB0003B00000000707772007077723400000004
:101BC0000062BE8FBD0C62043B00000000310000CB
:101BD00000316D6100000003003EBE64610E62587A
:101BE0005900000000310000003173610000000363
:101BF0000342BED361E5BC63596666E63F3100002F
:101C0000003174720000000B0447BED361F1BC6761
:101C1000595C8FA24031000000316D690000000363
:101C20000056BE6461FDBC595900000041310000FE
:101C30000031706F00000003005ABE646134625DC1
:101C400059000000003100000031706D00000003F9
:101C5000005EBE64617BBD5E590000004032000042
:101C600000326D6100000003003EBE64610E6277C9
:101C7000590000803F320000003273610000000311
:101C80000342BED361E5BC82596666E63F3200007E
:101C9000003274720000000B0447BED361F1BC86B1
:101CA000595C8FA24032000000326D6900000003D1
:101CB0000056BE6461FDBC7859000000413200004E
:101CC0000032706F00000003005ABE646134627C11
:101CD000590000803F3200000032706D00000003A8
:101CE000005EBE64617BBD7D590000004033000092
:101CF00000336D6100000003003EBE64610E629619
:101D000059000000403300000033736100000003FD
:101D10000342BED361E5BCA1596666E63F330000CD
:101D2000003374720000000B0447BED361F1BCA500
:101D3000597777074033000000336D6900000003D6
:101D40000056BE6461FDBC9759000000413300009D
:101D50000033706F00000003005ABE646134629B60
:101D600059000000003300000033706D00000003D4
:101D7000005EBE64617BBD9C5900000040340000E1
:101D800000346D6100000003003EBE64610E62B568
:101D9000590000404034000000347361000000032B
:101DA0000342BED361E5BCC0596666E63F3400001D
:101DB000003474720000000B0447BED361F1BCC450
:101DC000590000B44334000000346D690000000382
:101DD0000056BE6461FDBCB65900000041340000ED
:101DE0000034706F00000003005ABE64613462BAB0
:101DF00059000000003400000034706D0000000342
:101E0000005EBE64617BBDBB5900000040780000ED
:101E10000078616D00000003005C5FD15CE45C89C8
:101E2000310000803F7800000078766D0000000BE4
:101E300000A55FD3610B678E310000C844780000B5
:101E4000007866720000000B00A15FD3610B678A07
:101E5000310000C8447800000078746E0000000B68
:101E600003AD5FD3610B679631000000007800007E
:101E70000078746D0000000B03A95FD3610B6792BB
:101E8000310000964378000000786A6D0000000B76
:101E900000B15FD361525D9A310000C84278000002
:101EA00000786A680000000B00B55FD361AA5D9EF0
:101EB000310000C84278000000786A640000000B1E
:101EC00004B95FD3610B67A631CDCC4C3D780000DF
:101ED0000078736E0000000300C15F6461E3C0AD71
:101EE000300000803F780000007873780000000325
:101EF00000C55F6461E3C0AE300000000078000000
:101F0000007873760000000B00C95FD3610B67AEE9
:101F10003100007A4478000000786C760000000BF5
:101F200000CD5FD3610B67B2310000C8427800007A
:101F300000786C620000000B03D15FD3610B67B6C1
:101F4000310000204178000000787A620000000B28
:101F500003D55FD3610B67BA310000004079000000
:101F60000079616D00000003005C5FD15CE45CBE41
:101F7000310000803F7900000079766D0000000B91
:101F800000A55FD3610B67C3310000C8447900002E
:101F9000007966720000000B00A15FD3610B67BF80
:101FA000310000C8447900000079746E0000000B15
:101FB00003AD5FD3610B67CB3100000000790000F7
:101FC0000079746D0000000B03A95FD3610B67C734
:101FD000310000E14379000000796A6D0000000BD8
:101FE00000B15FD361525DCF310000C8427900007B
:101FF00000796A680000000B00B55FD361AA5DD369
:10200000310000C84279000000796A640000000BCA
:1020100004B95FD3610B67DB31CDCC4C3D79000057
:102020000079736E0000000300C15F6461E3C0AF1C
:10203000300000803F7900000079737800000003D1
:1020400000C55F6461E3C0B030000000407900006B
:10205000007973760000000B00C95FD3610B67E362
:102060003100007A4479000000796C760000000BA2
:1020700000CD5FD3610B67E7310000C842790000F3
:1020800000796C620000000B03D15FD3610B67EB3A
:10209000310000204179000000797A620000000BD5
:1020A00003D55FD3610B67EF31000000407A000079
:1020B000007A616D00000003005C5FD15CE45CF3BA
:1020C000310000803F7A0000007A766D0000000B3E
:1020D00000A55FD3610B67F831000096447A0000D9
:1020E000007A66720000000B00A15FD3610B67F4F9
:1020F00031000096447A0000007A746E0000000BF4
:1021000003AD5FD3610B670032000000007A00006E
:10211000007A746D0000000B03A95FD3610B67FCAC
:1021200031000096427A0000007A6A6D0000000BD0
:1021300000B15FD361525D04320000C8427A0000F2
:10214000007A6A680000000B00B55FD361AA5D08E1
:10215000320000C8427A0000007A6A640000000B76
:1021600004B95FD3610B671032CDCC4C3D7A0000CF
:10217000007A736E0000000300C15F6461E3C0B1C8
:1021800030000000007A0000007A7378000000033D
:1021900000C55F6461E3C0B2300000803F7A000098
:1021A000007A73760000000B00C95FD3610B6718DB
:1021B00032000016447A0000007A6C760000000BB2
:1021C00000CD5FD3610B671C320000C8427A00006B
:1021D000007A6C620000000B03D15FD3610B6720B3
:1021E00032000020417A0000007A7A620000000B81
:1021F00003D55FD3610B672432000000406100000B
:102200000061616D00000003005C5FD15CE45C284C
:10221000320000803F6100000061766D0000000325
:1022200000A55FD3611A632D320000614561000093
:10223000006166720000000300A15FD3611A632988
:1022400032000061456100000061746E000000030F
:1022500003AD5FD3610B673532000080BF610000C2
:102260000061746D0000000303A95FD3611A63313C
:1022700032000080BF61000000616A6D0000000351
:1022800000B15FD361525D39320000C84261000085
:1022900000616A680000000300B55FD361AA5D3D7C
:1022A000320000C84261000000616A64000000035F
:1022B00004B95FD3611A634532CDCC4C3D61000057
:1022C000006172610000000B03BD5FD3611A6349B6
:1022D000320000803F6100000061736E0000000367
:1022E00000C15F6461E3C0B3300000803F61000063
:1022F000006173780000000300C55F6461E3C0B44F
:1023000030000000406100000061737600000003AF
:1023100000C95FD3611A634D3200001644610000AA
:1023200000616C760000000300CD5FD3611A635139
:10233000320000C84261000000616C6200000003CE
:1023400003D15FD3611A6355320000204161000060
:1023500000617A620000000303D55FD3611A6359FC
:1023600032000000406200000062616D0000000366
:10237000005C5FD15CE45C5D320000000062000044
:102380000062766D0000000300A55FD3611A6362EE
:1023900032000061456200000062667200000003C6
:1023A00000A15FD3611A635E3200006145620000E4
:1023B0000062746E0000000303AD5FD3610B676AB7
:1023C00032000080BF6200000062746D00000003F4
:1023D00003A95FD3611A636632000080BF62000008
:1023E00000626A6D0000000300B15FD361525D6E50
:1023F000320000C84262000000626A64000000030C
:1024000000B95FD3611A637A32CDCC4C3D620000D3
:10241000006272610000000B03BD5FD3611A637E2E
:10242000320000803F6300000063616D0000000324
:10243000005C5FD15CE45C9232000000006300004D
:102440000063766D0000000300A55FD3611A6397F7
:102450003200006145630000006366720000000303
:1024600000A15FD3611A63933200006145630000ED
:102470000063746E0000000303AD5FD3610B679FC0
:1024800032000080BF6300000063746D0000000331
:1024900003A95FD3611A639B32000080BF63000011
:1024A00000636A6D0000000300B15FD361525DA359
:1024B000320000C84263000000636A640000000349
:1024C00000B95FD3611A63AF32CDCC4C3D630000DD
:1024D000006372610000000B03BD5FD3611A63B338
:1024E000320000803F70310000703166727100036D
:1024F0000024ABD3611A6334580000C84270310025
:1025000000703163736C00030028ABD3611A633829
:102510005800007A44703100007031637368000322
:10252000002CABD3611A633C580000FA44703100B0
:1025300000703163706C00030330ABD3611A6340E9
:10254000580000003E703100007031637068000375
:102550000334ABD3611A634458CDCC4C3E70310088
:1025600000703177736C00030038ABD3611A634895
:102570005800007A447031000070317773680003AE
:10258000003CABD3611A634C580000FA4470310030
:1025900000703177706C00030340ABD3611A635055
:1025A000580000003E703100007031777068000301
:1025B0000344ABD3611A635458CDCC4C3E70310008
:1025C000007031706F6600030348ABD3611A635823
:1025D00058CDCCCC3D673534006735347800000BDE
:1025E00003D95FD3610B67F9300000000067353411
:1025F000006735347900000B03D95FD3610B67FDA9
:102600003000000000673534006735347A00000B75
:1026100003D95FD3610B67013100000000673534D7
:10262000006735346100000B03D95FD3610B670588
:102630003100000000673534006735346200000B5C
:1026400003D95FD3610B670931000000006735349F
:10265000006735346300000B03D95FD3610B670D4E
:102660003100000000673535006735357800000B14
:1026700003D95FD3610B671131000016436735350D
:10268000006735357900000B03D95FD3610B6715FF
:102690003100006143673535006735357A00000B3E
:1026A00003D95FD3610B671931000000006735352E
:1026B000006735356100000B03D95FD3610B671DDF
:1026C0003100000000673535006735356200000BCA
:1026D00003D95FD3610B67213100000000673535F6
:1026E000006735356300000B03D95FD3610B6725A5
:1026F0003100000000673536006735367800000B82
:1027000003D95FD3610B67293100000000673536BC
:10271000006735367900000B03D95FD3610B672D55
:102720003100000000673536006735367A00000B4F
:1027300003D95FD3610B6731310000000067353684
:10274000006735366100000B03D95FD3610B673535
:102750003100000000673536006735366200000B37
:1027600003D95FD3610B673931000000006735364C
:10277000006735366300000B03D95FD3610B673DFB
:102780003100000000673537006735377800000BEF
:1027900003D95FD3610B6741310000000067353713
:1027A000006735377900000B03D95FD3610B6745AC
:1027B0003100000000673537006735377A00000BBD
:1027C00003D95FD3610B67493100000000673537DB
:1027D000006735376100000B03D95FD3610B674D8C
:1027E0003100000000673537006735376200000BA5
:1027F00003D95FD3610B67513100000000673537A3
:10280000006735376300000B03D95FD3610B675551
:102810003100000000673538006735387800000B5C
:1028200003D95FD3610B6759310000000067353869
:10283000006735387900000B03D95FD3610B675D02
:102840003100000000673538006735387A00000B2A
:1028500003D95FD3610B6761310000000067353831
:10286000006735386100000B03D95FD3610B6765E2
:102870003100000000673538006735386200000B12
:1028800003D95FD3610B67693100000000673538F9
:10289000006735386300000B03D95FD3610B676DA8
:1028A0003100000000673539006735397800000BCA
:1028B00003D95FD3610B67713100000000673539C0
:1028C000006735397900000B03D95FD3610B677559
:1028D0003100000000673539006735397A00000B98
:1028E00003D95FD3610B6779310000000067353988
:1028F000006735396100000B03D95FD3610B677D39
:102900003100000000673539006735396200000B7F
:1029100003D95FD3610B678131000000006735394F
:10292000006735396300000B03D95FD3610B6785FE
:102930003100000000673932006739327800000149
:1029400003D95FD3610C626A33000000006739323B
:10295000006739327900000103D95FD3610C626EE0
:102960003300000000673932006739327A00000115
:1029700003D95FD3610C6272330000000067393203
:10298000006739326100000103D95FD3610C6276C0
:1029900033000000006739320067393262000001FD
:1029A00003D95FD3610C627A3300000000673932CB
:1029B000006739326300000103D95FD3610C627E86
:1029C00033000000006732380067323878000001B9
:1029D00003DD5FD3610C6282330000000067323890
:1029E000006732387900000103DD5FD3610C628635
:1029F0003300000000673238006732387A00000187
:102A000003DD5FD3610C628A330000000067323857
:102A1000006732386100000103DD5FD3610C628E14
:102A2000330000000067323800673238620000016E
:102A300003DD5FD3610C629233000000006732381F
:102A4000006732386300000103DD5FD3610C6296DA
:102A50003300000000673330006733307800000136
:102A600003DD5FD3610C629A3300000000673330EE
:102A7000006733307900000103DD5FD3610C629E93
:102A80003300000000673330006733307A00000104
:102A900003DD5FD3610C62A23300000000673330B6
:102AA000006733306100000103DD5FD3610C62A673
:102AB00033000000006733300067333062000001EC
:102AC00003DD5FD3610C62AA33000000006733307E
:102AD000006733306300000103DD5FD3610C62AE39
:102AE00033000000006A6964006A696461000000E4
:102AF0000074C5AC61F3622E3B000000006A69649B
:102B0000006A6964620000000074C5AC61F362325F
:102B10003B000000006A6964006A696463000000A9
:102B20000074C5AC61F362363B000000006A696462
:102B3000006A6964640000000074C5AC61F3623A25
:102B40003B00000000737973006A61000000000F11
:102B500000FB5ED3610B67C7300050434873797345
:102B6000006374000000000F041A5FD3610B67CB91
:102B7000300AD7233C73797300736C0000000007A0
:102B800000395F64610E62CF30000000007379731A
:102B9000007374000000000700FDC06461DDC0A286
:102BA0003000000000737973006D740000000007AE
:102BB000023ABED361A9BD54590000004000000094
:102BC000006D6500000000000075C50BBE0BBE0463
:102BD0003B00000000000000006D640000000000E9
:102BE0000075C5E3BDE3BD043B00000000737973CD
:102BF00000656A000000000700D183646134622030
:102C00003B0000803F737973006A76000000000784
:102C100000D58364616283C63D0000004073797310
:102C2000006A73000000000700D98364613462C841
:102C30003D0000803F737973007476000000000748
:102C4000006AC664613462C75A0000803F737973BA
:102C500000717600000000070099B164617E628D0A
:102C600058000000007379730073760000000007BD
:102C700000FCAF646159629A580000803F73797319
:102C8000007369000000000700F8AF8861C0AF9BC7
:102C90005800007A437379730065630000000007F1
:102CA000005C6764611668BC2900000000737973DA
:102CB000006565000000000700606764619668BDFC
:102CC0002900000000737973006578000000000798
:102CD00000646764615668BE290000803F737973A1
:102CE0000072786D0000000700686764613462BF9D
:102CF000290000803F7379730062617564000004ED
:102D0000006C676461BD66BA290000A04000000045
:102D1000007372000000000000F6AFBCAFBEAF044D
:102D20003B00000000000000007172000000000085
:102D3000008DB140B10C62043B00000000000000B7
:102D400000716900000000000091B155B10C6204EF
:102D50003B0000000000000000716F000000000058
:102D60000095B171B10C62043B000000000000004E
:102D700000657200000000000074C52DAC0C6204F8
:102D80003B00000000000000007166000000000031
:102D90000074C56061D65D043B00000000000000C7
:102DA000007278000000000000A9C5A1660C620452
:102DB0003B00000000000000006D73670000000091
:102DC0000075C560610C62043B000000000000005B
:102DD00000636C65617200000074C5FF52FF52040D
:102DE0003B000000000000000074657374000000E8
:102DF0000074C5D37D01C1043B0000000000000049
:102E000000646566610000000074C5FE7D0A61040F
:102E10003B0000000000000000626F6F74000000C3
:102E20000074C5297E247D043B00000000000000E2
:102E30000068656C700000000074C5947D0C62042D
:102E40003B000000000000000068000000000000DF
:102E50000074C5947D0C62043B000000007379731C
:102E60000067706C0000000700E75E64615962DD76
:102E700030000000007379730067756E0000000772
:102E800000EB5E64613462DE300000803F73797372
:102E90000067636F0000000700EF5E64610E62DC94
:102EA000300000803F737973006770610000000795
:102EB00000F35E64615962DF300000004073797393
:102EC000006764690000000700F75E64613462E037
:102ED00030000000000000000067630000000000F8
:102EE0000074C5DB7BEB7B043B00000000000000AE
:102EF000006D61000000000B043D5FD3610B67D4DF
:102F000030CDCCCC3D000000006664000000000322
:102F1000008DC564613462C73D00000000756461C6
:102F2000007564613000000300A9C5AC61F362C0A4
:102F30003A000000007564610075646131000003AF
:102F400000A9C5AC61F362C43A0000000075646179
:102F5000007564613200000300A9C5AC61F362C86A
:102F60003A0000000075646100756461330000037D
:102F700000A9C5AC61F362CC3A0000000075646240
:102F8000007564623000000300A9C5AC61F362D033
:102F90003A0000000075646200756462310000034D
:102FA00000A9C5AC61F362D43A0000000075646208
:102FB000007564623200000300A9C5AC61F362D8F9
:102FC0003A0000000075646200756462330000031B
:102FD00000A9C5AC61F362DC3A00000000756463CF
:102FE000007564633000000300A9C5AC61F362E0C2
:102FF0003A000000007564630075646331000003EB
:1030000000A9C5AC61F362E43A0000000075646396
:10301000007564633200000300A9C5AC61F362E887
:103020003A000000007564630075646333000003B8
:1030300000A9C5AC61F362EC3A000000007564645D
:10304000007564643000000300A9C5AC61F362F050
:103050003A00000000756464007564643100000388
:1030600000A9C5AC61F362F43A0000000075646425
:10307000007564643200000300A9C5AC61F362F816
:103080003A00000000756464007564643300000356
:1030900000A9C5AC61F362FC3A000000005F7465F2
:1030A000005F74657800000002C6C5D3610C62FD44
:1030B00055000000005F7465005F746579000000D2
:1030C00002C6C5D3610C620156000000005F746542
:1030D000005F74657A00000002C6C5D3610C62050A
:1030E00056000000005F7465005F746561000000B9
:1030F00002C6C5D3610C620956000000005F74650A
:10310000005F74656200000002C6C5D3610C620DE9
:1031100056000000005F7465005F74656300000086
:1031200002C6C5D3610C621156000000005F7472C4
:10313000005F74727800000002C6C5D3610C622281
:1031400057000000005F7472005F74727900000025
:1031500002C6C5D3610C622657000000005F74727E
:10316000005F74727A00000002C6C5D3610C622A47
:1031700057000000005F7472005F7472610000000D
:1031800002C6C5D3610C622E57000000005F747246
:10319000005F74726200000002C6C5D3610C623227
:1031A00057000000005F7472005F747263000000DB
:1031B00002C6C5D3610C623657000000005F74730D
:1031C000005F74733100000002C6C5D3610C628DCC
:1031D00056000000005F7073005F707331000000E4
:1031E00002C6C5D3610C629D56000000005F637388
:1031F000005F63733100000002C6C5D3610C62AD8D
:1032000056000000005F6573005F657331000000C9
:1032100002C6C5D3610C62BD56000000005F787322
:10322000005F78733100000002C6C5D3610C62EF05
:1032300059000000005F6665005F666531000000B0
:1032400002C6C5D3610C62CD56000000005F7473E6
:10325000005F74733200000002C6C5D3610C629136
:1032600056000000005F7073005F70733200000052
:1032700002C6C5D3610C62A156000000005F6373F3
:10328000005F63733200000002C6C5D3610C62B1F7
:1032900056000000005F6573005F65733200000038
:1032A00002C6C5D3610C62C156000000005F78738E
:1032B000005F78733200000002C6C5D3610C62075C
:1032C0005A000000005F6665005F6665320000001E
:1032D00002C6C5D3610C62D156000000005F747352
:1032E000005F74733300000002C6C5D3610C6295A1
:1032F00056000000005F7073005F707333000000C1
:1033000002C6C5D3610C62A556000000005F63735E
:10331000005F63733300000002C6C5D3610C62B561
:1033200056000000005F6573005F657333000000A6
:1033300002C6C5D3610C62C556000000005F7873F9
:10334000005F78733300000002C6C5D3610C621FB2
:103350005A000000005F6665005F6665330000008C
:1033600002C6C5D3610C62D556000000005F7473BD
:10337000005F74733400000002C6C5D3610C62990B
:1033800056000000005F7073005F7073340000002F
:1033900002C6C5D3610C62A956000000005F6373CA
:1033A000005F63733400000002C6C5D3610C62B9CC
:1033B00056000000005F6573005F65733400000015
:1033C00002C6C5D3610C62C956000000005F787365
:1033D000005F78733400000002C6C5D3610C623709
:1033E0005A000000005F6665005F666534000000FB
:1033F00002C6C5D3610C62D956000000000000006F
:10340000005F64616D0000000074C54F5E4F5E0494
:103410003B00000000000000007365303000000237
:103420000074C58861A362A6580000000000000077
:1034300000736530310000020074C58861A362A882
:1034400058000000000000000073653032000002E8
:103450000074C58861A362AA580000000000000043
:1034600000736530330000020074C58861A362AC4C
:1034700058000000000000000073653034000002B6
:103480000074C58861A362AE58000000000000000F
:1034900000736530350000020074C58861A362B016
:1034A0005800000000000000007365303600000284
:1034B0000074C58861A362B25800000000000000DB
:1034C00000736530370000020074C58861A362B4E0
:1034D0005800000000000000007365303800000252
:1034E0000074C58861A362B65800000000000000A7
:1034F00000736530390000020074C58861A362B8AA
:103500005800000000000000007365313000000228
:103510000074C58861A362BA580000000000000072
:1035200000736531310000020074C58861A362BC7C
:1035300058000000000000000073653132000002F6
:103540000074C58861A362BE58000000000000003E
:1035500000736531330000020074C58861A362C046
:1035600058000000000000000073653134000002C4
:103570000074C58861A362C258000000000000000A
:1035800000736531350000020074C58861A362C410
:103590005800000000000000007365313600000292
:1035A0000074C58861A362C65800000000000000D6
:1035B00000736531370000020074C58861A362C8DA
:1035C0005800000000000000007365313800000260
:1035D0000074C58861A362CA5800000000000000A2
:1035E00000736531390000020074C58861A362CCA4
:1035F0005800000000000000007365323000000237
:103600000074C58861A362CE58000000000000006D
:1036100000736532310000020074C58861A362D076
:103620005800000000000000007365323200000204
:103630000074C58861A362D2580000000000000039
:1036400000736532330000020074C58861A362D440
:1036500058000000000000000073653234000002D2
:103660000074C58861A362D6580000000000000005
:1036700000736532350000020074C58861A362D80A
:1036800058000000000000000073653236000002A0
:103690000074C58861A362DA5800000000000000D1
:1036A00000736532370000020074C58861A362DCD4
:1036B000580000000000000000736532380000026E
:1036C0000074C58861A362DE58000000000000009D
:1036D00000736532390000020074C58861A362E09E
:1036E0005800000000000000007379730000000023
:1036F0000074C5E0645363043B0000000000000058
:1037000000703100000000000074C5E064536304E1
:103710003B0000000000000000310000000000003D
:103720000074C5E0645363043B0000000000000027
:1037300000320000000000000074C5E06453630420
:103740003B0000000000000000330000000000000B
:103750000074C5E0645363043B00000000000000F7
:1037600000340000000000000074C5E064536304EE
:103770003B00000000000000007800000000000096
:103780000074C5E0645363043B00000000000000C7
:1037900000790000000000000074C5E06453630479
:1037A0003B00000000000000007A00000000000064
:1037B0000074C5E0645363043B0000000000000097
:1037C00000610000000000000074C5E06453630461
:1037D0003B0000000000000000620000000000004C
:1037E0000074C5E0645363043B0000000000000067
:1037F00000630000000000000074C5E0645363042F
:103800003B000000000000000067353400000000AD
:103810000074C5E0645363043B0000000000000036
:1038200000673535000000000074C5E06453630490
:103830003B0000000000000000673536000000007B
:103840000074C5E0645363043B0000000000000006
:1038500000673537000000000074C5E0645363045E
:103860003B00000000000000006735380000000049
:103870000074C5E0645363043B00000000000000D6
:1038800000673539000000000074C5E0645363042C
:103890003B0000000000000000673932000000001B
:1038A0000074C5E0645363043B00000000000000A6
:1038B00000673238000000000074C5E06453630400
:1038C0003B000000000000000067333000000000F3
:1038D0000074C5E0645363043B0000000000000076
:1038E000006D706F000000000074C5E06453630455
:1038F0003B0000000000000000706F73000000003B
:103900000074C5E0645363043B0000000000000045
:10391000006F6673000000000074C5E06453630428
:103920003B0000000000000000686F6D0000000018
:103930000074C5E0645363043B0000000000000015
:1039400000707262000000000074C5E064536304FC
:103950003B000000000000000070777200000000D3
:103960000074C5E0645363043B00000000000000E5
:10397000006A6F67000000000074C5E064536304D0
:103980003B00000000000000006A696400000000C5
:103990000074C5E0645363043B00000000000000B5
:1039A00000756461000000000074C5E064536304A6
:1039B0003B00000000000000007564620000000091
:1039C0000074C5E0645363043B0000000000000085
:1039D00000756463000000000074C5E06453630474
:1039E0003B0000000000000000756464000000005F
:1039F0000074C5E0645363043B0000000000000055
:103A0000005F7465000000000074C5E06453630447
:103A10003B00000000000000005F74720000000026
:103A20000074C5E0645363043B0000000000000024
:103A3000005F7473000000000074C5E06453630409
:103A40003B00000000000000005F707300000000F9
:103A50000074C5E0645363043B00000000000000F4
:103A6000005F6373000000000074C5E064536304EA
:103A70003B00000000000000005F657300000000D4
:103A80000074C5E0645363043B00000000000000C4
:103A9000005F7873000000000074C5E064536304A5
:103AA0003B00000000000000005F666500000000B1
:103AB0000074C5E0645363043B0000000000000094
:103AC000006D0000000000000074C5D1670C6204A6
:103AD0003B0000000000000000710000000000003A
:103AE0000074C5B7670C62043B00000000000000D2
:103AF000006F0000000000000074C59D670C6204A8
:103B00003B00000000000000002400000000000056
:103B10000074C5EB670C62043B00000000486F6D49
:103B2000696E67206572726F72202D202563206197
:103B30007869732073657474696E6773206D697337
:103B4000636F6E666967757265640050726F626953
:103B50006E67206572726F72202D20256320617858
:103B600069732063616E6E6F74206D6F766520647B
:103B70007572696E672070726F62696E67005B694B
:103B8000645D202054696E794720494425333073A1
:103B90000A005B68765D20206861726477617265F7
:103BA0002076657273696F6E2531362E32660A0093
:103BB0005B68705D20206861726477617265207057
:103BC0006C6174666F726D2531352E32660A005B4A
:103BD00066765D20206669726D7761726520766514
:103BE0007273696F6E2531362E32660A005B66622B
:103BF0005D20206669726D77617265206275696CFF
:103C0000642531382E32660A00456E7465722024B0
:103C1000626F6F743D3120746F20656E7465722021
:103C200074686520626F6F74206C6F616465722EBA
:103C30000A000A0A0A2323232054696E7947204286
:103C40004F4F54204C4F414445522048656C7020E2
:103C50002323230A00456E7465722024646566611F
:103C60003D3120746F20726573657420746865201F
:103C700073797374656D20746F2074686520666154
:103C800063746F72792064656661756C7420766107
:103C90006C7565732E0A546869732077696C6C20A3
:103CA0006F766572777269746520616E79206368DA
:103CB000616E67657320796F752068617665206D28
:103CC0006164652E0A000A0A0A2323232054696EC0
:103CD000794720524553544F52452044454641555B
:103CE0004C54532048656C70202323230A00496EEE
:103CF000766F6B652073656C6620746573742062E3
:103D00007920656E746572696E67202474657374BA
:103D10003D4E207768657265204E206973206F6E76
:103D200065206F663A0A202024746573743D312043
:103D300020736D6F6B6520746573740A2020247482
:103D40006573743D322020686F6D696E67207465FD
:103D5000737420202028796F75206D75737420741A
:103D600072697020686F6D696E672073776974631C
:103D7000686573290A202024746573743D332020FC
:103D800073717561726520746573742020202861D9
:103D900020736572696573206F6620737175617237
:103DA0006573290A202024746573743D34202061D2
:103DB0007263207465737420202020202028736F84
:103DC0006D65206C6172676520636972636C6573F1
:103DD000290A202024746573743D3520206477659A
:103DE0006C6C207465737420202020286D6F7665BC
:103DF000732073706163656420627920312073657C
:103E0000636F6E64206477656C6C73290A202024CC
:103E1000746573743D36202066656564686F6C64F4
:103E200020746573742028656E746572202120618A
:103E30006E64207E20746F20686F6C6420616E64F5
:103E400020726573746172742C207265737065637F
:103E5000746976656C79290A202024746573743D31
:103E60003720204D20636F64657320746573742060
:103E700020284D20636F64657320696E7465726DD0
:103E8000696E676C65642077697468206D6F76650C
:103E900073290A202024746573743D3820204A5306
:103EA0004F4E20746573742020202020286D6F747D
:103EB000696F6E20746573742072756E20757369F6
:103EC0006E67204A534F4E20636F6D6D616E647351
:103ED000290A202024746573743D392020696E7688
:103EE000657273652074696D6520746573740A204A
:103EF0002024746573743D313020726F746172795F
:103F0000206D6F74696F6E20746573740A202024AD
:103F1000746573743D313120736D616C6C206D6F0D
:103F200076657320746573740A2020247465737435
:103F30003D313220736C6F77206D6F76657320741E
:103F40006573740A202024746573743D31332063D3
:103F50006F6F7264696E6174652073797374656DD7
:103F6000206F666673657420746573742028473902
:103F7000322C204735342D473539290A0A546573C8
:103F8000747320617373756D6520612063656E7451
:103F900065726564205859206F726967696E206187
:103FA0006E64206174206C656173742038306D6DAF
:103FB00020636C656172616E636520696E20616C5F
:103FC0006C20646972656374696F6E730A546573FB
:103FD000747320617373756D65205A206861732056
:103FE0006174206C656173742034306D6D20706F66
:103FF0007369697469766520636C656172616E636B
:10400000650A5465737473207374617274207769E0
:1040100074682061204730205830205930205A30B1
:10402000206D6F76650A486F6D696E672069732031
:1040300074686520657863657074696F6E2E204EB4
:104040006F20696E697469616C20706F736974693F
:104050006F6E206F7220636C656172616E636520A4
:10406000697320617373756D65640A000A0A0A2317
:1040700023232054696E79472053454C46205445EC
:1040800053542048656C70202323230A0045616344
:1040900068202420636F6D6D616E642061626F76AD
:1040A0006520616C736F20646973706C6179732033
:1040B00074686520746F6B656E20666F7220656131
:1040C00063682073657474696E6720696E205B2075
:1040D0005D20627261636B6574730A546F20766948
:1040E00065772073657474696E677320656E746597
:1040F00072206120746F6B656E3A0A0A2020243C9E
:10410000746F6B656E3E0A0A466F72206578616D4A
:10411000706C65202479667220746F2064697370F6
:104120006C6179207468652059206D61782066651E
:10413000656420726174650A0A546F207570646149
:1041400074652073657474696E677320656E746539
:104150007220746F6B656E20657175616C7320766B
:10416000616C75653A0A0A2020243C746F6B656E99
:104170003E3D3C76616C75653E0A0A466F7220656D
:1041800078616D706C6520247966723D383030201E
:10419000746F20736574207468652059206D617890
:1041A0002066656564207261746520746F20383004
:1041B00030206D6D2F6D696E7574650A466F7220C3
:1041C000636F6E66696775726174696F6E2064658E
:1041D0007461696C73207365653A206874747073D8
:1041E0003A2F2F6769746875622E636F6D2F73792C
:1041F0006E746865746F732F54696E79472F776991
:104200006B692F54696E79472D436F6E66696775C8
:10421000726174696F6E0A00546865736520636F1C
:104220006D6D616E6473206172652061637469767F
:104230006520666F7220636F6E6669677572617460
:10424000696F6E3A0A2020247379732053686F7760
:104250002073797374656D202867656E6572616C73
:10426000292073657474696E67730A2020243120D5
:10427000202053686F77206D6F746F722031207328
:10428000657474696E677320286F72207768617433
:1042900065766572206D6F746F7220796F75207707
:1042A000616E7420312C322C332C34290A202024C6
:1042B0007820202053686F77205820617869732018
:1042C00073657474696E677320286F7220776861F4
:1042D0007465766572206178697320796F752077CF
:1042E000616E7420782C792C7A2C612C622C6329D5
:1042F0000A2020246D20202053686F7720616C6C89
:10430000206D6F746F722073657474696E67730AC1
:104310002020247120202053686F7720616C6C204E
:10432000617869732073657474696E67730A2020FD
:10433000246F20202053686F7720616C6C206F669B
:10434000667365742073657474696E67730A2020E0
:10435000242420202053686F7720616C6C207365C3
:104360007474696E67730A202024682020205368C3
:104370006F7720746869732068656C70207363724E
:1043800065656E0A0A000A0A0A2323232054696E0F
:10439000794720434F4E46494755524154494F4E65
:1043A0002048656C70202323230A000A466F722080
:1043B00064657461696C65642054696E794720692D
:1043C0006E666F207365653A2068747470733A2F57
:1043D0002F6769746875622E636F6D2F73796E74C1
:1043E0006865746F732F54696E79472F77696B69AD
:1043F0002F0A466F7220746865206C61746573744F
:10440000206669726D77617265207365653A206810
:10441000747470733A2F2F6769746875622E636FB6
:104420006D2F73796E746865746F732F54696E792C
:10443000470A506C65617365206C6F6720616E7907
:104440002069737375657320617420687474703AA1
:104450002F2F7777772E73796E746865746F732E4C
:10446000636F6D2F666F72756D730A486176652094
:1044700066756E0A000A4E6F74653A2054696E794B
:10448000472067656E657261746573206175746F2E
:104490006D617469632073746174757320726570E3
:1044A0006F7274732062792064656661756C740A3A
:1044B000546869732063616E20626520646973616A
:1044C000626C656420627920656E746572696E67DE
:1044D000202473763D300A53656520746865207723
:1044E000696B692062656C6F7720666F72206D6FF3
:1044F00072652064657461696C732E0A0054686586
:10450000736520636F6D6D616E64732061726520E9
:104510006163746976652066726F6D2074686520CA
:10452000636F6D6D616E64206C696E653A0A205E22
:1045300078202020202020202020202020205265AC
:104540007365742028636F6E74726F6C20782920F5
:104550002D20736F66747761726520726573657460
:104560000A20203F20202020202020202020202042
:10457000204D616368696E6520706F736974696F3F
:104580006E20616E642067636F6465206D6F646583
:104590006C2073746174650A202024202020202060
:1045A000202020202020202053686F7720616E6417
:1045B0002073657420636F6E6669677572617469D4
:1045C0006F6E2073657474696E67730A20202120F2
:1045D00020202020202020202020202046656564E7
:1045E000686F6C64202D2073746F70206D6F746918
:1045F0006F6E20776974686F7574206C6F73696E65
:104600006720706F736974696F6E0A20207E2020A6
:1046100020202020202020202020204379636C654A
:10462000205374617274202D2072657374617274EA
:104630002066726F6D2066656564686F6C640A2021
:1046400020682020202020202020202020202053EF
:10465000686F7720746869732068656C7020736375
:104660007265656E0A2020246820202020202020EA
:10467000202020202053686F7720636F6E66696763
:1046800075726174696F6E2068656C7020736372F7
:1046900065656E0A20202474657374202020202014
:1046A000202020204C6973742073656C662D74651E
:1046B0007374730A202024746573743D4E20202087
:1046C0002020202052756E2073656C662D746573F2
:1046D00074204E0A202024686F6D653D3120202013
:1046E0002020202052756E206120686F6D696E67F2
:1046F000206379636C650A202024646566613D311E
:1047000020202020202020526573746F7265206164
:104710006C6C2073657474696E677320746F2022EB
:10472000666163746F7279222064656661756C746A
:10473000730A000A0A0A2323232054696E7947204A
:1047400048656C70202323230A005B6A735D202078
:104750006A736F6E2073657269616C697A65207324
:1047600074796C65253964205B303D72656C6178C5
:1047700065642C313D7374726963745D0A005B6A11
:10478000765D20206A736F6E20766572626F736942
:10479000747925313564205B303D73696C656E74C6
:1047A0002C313D666F6F7465722C323D6D6573738D
:1047B000616765732C333D636F6E666967732C3474
:1047C0003D6C696E656E756D2C353D766572626FF8
:1047D00073655D0A005B656A5D2020656E61626CD1
:1047E00065206A736F6E206D6F64652531336420B8
:1047F0005B303D746578742C313D4A534F4E5D0AF1
:10480000000E5908590159FC58F358E858DD58D1A1
:1048100058C558B758A05891588458785864585774
:104820005842582E582B58285819580458EF57E01A
:1048300057D057BE57A7578A576D5754573E572DD5
:10484000571B570E57FC56E256DF56DC56D956D644
:1048500056D356D056CD56CA56C756C456C156BE64
:1048600056BB56B856B556B256AF56AC56A956A614
:1048700056A356A0569D569A569756945691568EC4
:10488000568B568856855682567F567C5679567674
:1048900056735670566D566A566756645661565E24
:1048A000565B565856555652564F564C56495646D4
:1048B00056435640561C56FC55E255C855AE558ACF
:1048C000556D5555553F5525550155E454D254B2B3
:1048D000549B5482546054475429540D54F553E367
:1048E00053C553B053AC53A853A453A0539C5398EF
:1048F00053945390538C538853845380537C5378F0
:10490000537453705356533C5329530D53FB52E485
:1049100052C352B2529252725258523E522752F4DD
:1049200051C751A75185515F5138511C51FD50E37A
:1049300050C950A4507B50635038500C50D64FA1F2
:104940004F8F4F7D4F6E4F5B4F424F204F0E4FFCAE
:104950004EEA4ED84EC64EB44EA24E904E7E4E6C8F
:104960004E5A4E484E364E244E204E1C4E184E1473
:104970004E104E0C4E084E044E004EFC4DF84DF4B9
:104980004DF04DEC4DE84DE44DE04DDC4DD84DD4AF
:104990004DC04DA24D864D5B4D364D114D0D4D090F
:1049A0004D054D014DFD4CF94CF54CF14CED4CE9EC
:1049B0004CE54CE14CDD4CD94CC54CA94C8D4C71AF
:1049C0004C554C394C1D4C014CE54BC94BAD4B91F2
:1049D0004B754B714B6D4B694B654B614B5D4B5947
:1049E0004B454B1D4BF64AD04AA34A7D4A504A4C90
:1049F0004A484A444A314A104AFB494A6F67676944
:104A00006E67206379636C65206661696C6564001C
:104A100050726F626520656E64706F696E74206994
:104A200073207374617274696E6720706F696E743D
:104A30000050726F6265206379636C6520666169FE
:104A40006C65640032343900323438003234370057
:104A5000486F6D696E67204572726F72202D204815
:104A60006F6D696E67207377697463686573206D15
:104A70006973636F6E6669677572656400486F6D10
:104A8000696E67204572726F72202D204E656761D6
:104A900074697665206C61746368206261636B6F12
:104AA000666600486F6D696E67204572726F72208E
:104AB0002D2054726176656C206D696E2026206D04
:104AC000617820617265207468652073616D65008E
:104AD000486F6D696E67204572726F72202D204C91
:104AE000617463682076656C6F636974792069739B
:104AF000207A65726F00486F6D696E67204572722B
:104B00006F72202D205365617263682076656C6F2B
:104B100063697479206973207A65726F00486F6DDC
:104B2000696E67204572726F72202D204261642089
:104B30006F72206E6F20617869732073706563698E
:104B40006669656400486F6D696E67206379636CA0
:104B500065206661696C6564003233390032333830
:104B600000323337003233360032333500323334DB
:104B70000032333300536F6674206C696D697420A2
:104B80006578636565646564202D2043206D6178D8
:104B900000536F6674206C696D6974206578636575
:104BA00065646564202D2043206D696E00536F6637
:104BB00074206C696D6974206578636565646564EB
:104BC000202D2042206D617800536F6674206C693F
:104BD0006D6974206578636565646564202D204285
:104BE000206D696E00536F6674206C696D69742066
:104BF0006578636565646564202D2041206D61786A
:104C000000536F6674206C696D6974206578636504
:104C100065646564202D2041206D696E00536F66C8
:104C200074206C696D69742065786365656465647A
:104C3000202D205A206D617800536F6674206C69B6
:104C40006D6974206578636565646564202D205AFC
:104C5000206D696E00536F6674206C696D697420F5
:104C60006578636565646564202D2059206D6178E1
:104C700000536F6674206C696D6974206578636594
:104C800065646564202D2059206D696E00536F6640
:104C900074206C696D69742065786365656465640A
:104CA000202D2058206D617800536F6674206C6948
:104CB0006D6974206578636565646564202D20588E
:104CC000206D696E00536F6674206C696D69742085
:104CD0006578636565646564003231390032313866
:104CE0000032313700323136003231350032313462
:104CF0000032313300323132003231310032313062
:104D0000003230390032303800323037003230363D
:104D10000054726170657A6F696420706C616E6EA8
:104D20006572206661696C656420746F20636F6EC4
:104D30007665726765004C696D6974207377697474
:104D4000636820686974202D2053687574646F77D8
:104D50006E206F63637572726564004D616368698C
:104D60006E6520697320616C61726D6564202D2011
:104D7000436F6D6D616E64206E6F742070726F632F
:104D80006573736564004D6F7665206C6573732081
:104D90007468616E206D696E696D756D2074696DE2
:104DA00065004D6F7665206C657373207468616E65
:104DB000206D696E696D756D206C656E6774680035
:104DC00047656E657269632054696E794720657224
:104DD000726F72003139390031393800313937009A
:104DE0003139360031393500313934003139330049
:104DF0003139320031393100313930003138390040
:104E00003138380031383700313836003138350024
:104E10003138340031383300313832003138310024
:104E2000313830005420776F726420697320696EC6
:104E300076616C6964005420776F72642069732016
:104E40006D697373696E67005220776F72642069B1
:104E50007320696E76616C6964005220776F7264AA
:104E6000206973206D697373696E67005120776FD5
:104E7000726420697320696E76616C6964005120E8
:104E8000776F7264206973206D697373696E670050
:104E90004C20776F726420697320696E76616C694B
:104EA00064004C20776F7264206973206D6973739E
:104EB000696E67004820776F726420697320696E9D
:104EC00076616C6964004820776F72642069732092
:104ED0006D697373696E67004520776F726420692E
:104EE0007320696E76616C6964004520776F726427
:104EF000206973206D697373696E67004420776F52
:104F0000726420697320696E76616C696400442064
:104F1000776F7264206973206D697373696E6700BF
:104F20005020776F7264206973206E6F7420612047
:104F300076616C696420746F6F6C206E756D62654C
:104F400072005020776F7264206973206E6F742036
:104F5000616E20696E7465676572005020776F72AC
:104F600064206973206E65676174697665005020FE
:104F7000776F7264206973207A65726F00502077B2
:104F80006F726420697320696E76616C6964005089
:104F900020776F7264206973206D697373696E671F
:104FA0000041726320737065636966696361746947
:104FB0006F6E206572726F72202D20656E64706F47
:104FC000696E74206973207374617274696E6720EE
:104FD000706F696E740041726320737065636966F7
:104FE00069636174696F6E206572726F72202D2023
:104FF00072616469757320617263206F7574206FCC
:105000006620746F6C6572616E6365004172632027
:1050100073706563696669636174696F6E20657238
:10502000726F72202D206D697373696E67206F66D1
:105030006673657428732900417263207370656319
:10504000696669636174696F6E206572726F722040
:105050002D206D697373696E6720617869732865A7
:1050600073290041726320737065636966696361C7
:1050700074696F6E206572726F72005370696E642E
:105080006C65206D757374206265207475726E692D
:105090006E6720666F72207468697320636F6D6D30
:1050A000616E64005370696E646C65206D75737415
:1050B000206265206F666620666F7220746869736F
:1050C00020636F6D6D616E64005370696E646C6512
:1050D000205320776F726420697320696E76616C4B
:1050E0006964005370696E646C65205320776F7239
:1050F00064206973206D697373696E67005370690A
:105100006E646C65207370656564206578636565A1
:10511000646564206D6178696D756D005370696EAA
:10512000646C652073706565642062656C6F7720C0
:105130006D696E696D756D0050726F6772616D6D2E
:10514000656420706F696E742073616D6520617392
:105150002063757272656E7420706F696E7400439F
:10516000757474657220636F6D70656E73617469B8
:105170006F6E2063616E6E6F7420626520656E6174
:10518000626C656400526571756573746564207640
:10519000656C6F63697479206578636565647320F5
:1051A0006C696D697473004730206F72204731203D
:1051B0006D7573742062652061637469766520661D
:1051C0006F722047353300526F74617279206178B5
:1051D00065732063616E6E6F742062652075736500
:1051E000642077697468207468697320636F6D6DDB
:1051F000616E6400496E76657273652074696D65D1
:10520000206D6F64652063616E6E6F74206265202F
:1052100075736564207769746820746869732063A6
:105220006F6D6D616E6400466565647261746520C2
:105230006E6F742073706563696669656400536599
:105240006C656374656420706C616E6520697320A1
:10525000696E76616C69640053656C65637465643E
:1052600020706C616E65206973206D697373696E5F
:105270006700417869732074617267657420706F8C
:10528000736974696F6E20697320696E76616C69E9
:105290006400417869732074617267657420706F6F
:1052A000736974696F6E206973206D697373696EB9
:1052B0006700417869732069732064697361626C67
:1052C0006564004178697320697320696E76616C4A
:1052D000696420666F72207468697320636F6D6DF6
:1052E000616E6400417869732063616E6E6F742033
:1052F00062652070726573656E7400417869732011
:10530000776F7264206D697373696E670047636FAE
:105310006465206D6F64616C2067726F75702076B4
:10532000696F6C6174696F6E004D20636F646520F6
:10533000756E737570706F727465640047636F6427
:105340006520636F6D6D616E6420756E737570702E
:105350006F727465640047656E65726963204763A8
:105360006F646520696E707574206572726F72006B
:1053700031323900313238003132370031323600C3
:1053800031323500313234003132330031323200C3
:1053900031323100313230003131390031313800B1
:1053A000313137003131360031313500313134009F
:1053B0004A534F4E20737472696E6720746F6F206A
:1053C0006C6F6E67004A534F4E20696E7075742083
:1053D00068617320746F6F206D616E7920706169F0
:1053E0007273004A534F4E2073796E746178206552
:1053F00072726F7200496E7075742076616C75659B
:105400002072616E6765206572726F7200496E70FE
:1054100075742065786365656473206D6178696D66
:10542000756D2076616C756500496E707574206CC1
:10543000657373207468616E206D696E696D756D3A
:105440002076616C756500496E70757420657863AF
:1054500065656473206D6178206C656E67746800A3
:10546000436F6D6D616E64206E6F74206163636560
:105470007074656420617420746869732074696D48
:105480006500506172616D657465722063616E6E56
:105490006F74206265207265616400506172616D95
:1054A0006574657220697320726561642D6F6E6C1E
:1054B0007900556E737570706F72746564206E75C7
:1054C0006D626572206F72204A534F4E207479705E
:1054D0006500426164206E756D62657220666F7250
:1054E0006D617400496E76616C6964206F72206D25
:1054F000616C666F726D656420636F6D6D616E6463
:1055000000556E7265636F676E697A656420636FBC
:105510006D6D616E64206F7220636F6E66696720C7
:105520006E616D650047656E6572696320617373B6
:10553000657274696F6E206661696C757265004D85
:10554000656D6F7279206661756C74206465746531
:105550006374656400537461636B206F7665726673
:105560006C6F7720646574656374656400436F6E67
:1055700074726F6C6C657220617373657274696F9D
:105580006E206661696C7572650043616E6F6E694D
:1055900063616C206D616368696E6520617373651A
:1055A0007274696F6E206661696C75726500506C0B
:1055B000616E6E657220617373657274696F6E20BF
:1055C0006661696C757265005374657070657220F0
:1055D000617373657274696F6E206661696C757250
:1055E0006500456E636F64657220617373657274E4
:1055F000696F6E206661696C75726500494F207332
:1056000075622D73797374656D206173736572743F
:10561000696F6E206661696C75726500436F6E66B6
:105620006967207375622D73797374656D2061737A
:1056300073657274696F6E206661696C757265005E
:1056400038390038380038370038360038350038F7
:105650003400383300383200383100383000373900
:105660000037380037370037360037350037340019
:1056700037330037320037310037300036390036E3
:1056800038003637003636003635003634003633CB
:1056900000363200363100363000353900353800FA
:1056A00035370035360035350035340035330035B3
:1056B00032003531003530003439003438003437A9
:1056C00000343600343500343400343300343200D2
:1056D000343100343000333900333800333700338D
:1056E0003600426164207374617475732072657052
:1056F0006F72742073657474696E6700506572739D
:10570000697374656E6365206572726F7200466CB2
:105710006F6174206973204E414E00466C6F617456
:1057200020697320696E66696E697465004D6F76D5
:10573000652074696D65206973204E414E004D6F80
:1057400076652074696D6520697320696E66696E7F
:105750006974650047656E65726963206578636585
:105760007074696F6E207265706F72740046616943
:105770006C656420746F2067657420706C616E6E58
:105780006572206275666665720053797374656D23
:1057900020616C61726D202D207368757474696E60
:1057A0006720646F776E00496E697469616C697A0D
:1057B0006174696F6E206661696C7572650052650F
:1057C00061642D6F6E6C792061646472657373001F
:1057D000496E76616C69642041646472657373001C
:1057E000446976696465206279207A65726F004643
:1057F0006C6F6174696E6720706F696E742065727A
:10580000726F7200496E7465726E616C2072616EA7
:105810006765206572726F7200496E7465726E61A1
:105820006C206572726F7200313900313800467534
:105830006E6374696F6E206973207374756262653C
:105840006400456E746572696E6720626F6F7420C4
:105850006C6F6164657200496E697469616C697A24
:10586000696E67004275666665722066756C6C20AD
:105870002D20666174616C004275666665722066F3
:10588000756C6C0042756666657220656D70747922
:10589000004E6F20737563682064657669636500E8
:1058A0004D61782066696C652073697A652065783A
:1058B0006365656465640046696C65206E6F74207D
:1058C0006F70656E00456E64206F662066696C655A
:1058D00000456E64206F66206C696E6500486172D9
:1058E00064207265736574005465726D696E6174CD
:1058F000656400436F6D706C657465004E6F6F700A
:105900000045616761696E004572726F72004F4BAE
:10591000005B7031706F665D2070776D207068611C
:105920007365206F66662020202531352E33662072
:105930005B302E2E315D0A005B70317770685D2020
:1059400070776D2063637720706861736520686984
:105950002531352E3366205B302E2E315D0A005BFB
:10596000703177706C5D2070776D20636377207085
:1059700068617365206C6F2531352E3366205B308E
:105980002E2E315D0A005B70317773685D20707771
:105990006D206363772073706565642068692531C5
:1059A000352E30662052504D0A005B703177736C93
:1059B0005D2070776D206363772073706565642068
:1059C0006C6F2531352E30662052504D0A005B70C9
:1059D000316370685D2070776D2063772070686137
:1059E0007365206869202531352E3366205B302EA3
:1059F0002E315D0A005B703163706C5D2070776DD5
:105A0000206377207068617365206C6F20253135C5
:105A10002E3366205B302E2E315D0A005B703163C1
:105A200073685D2070776D2063772073706565649F
:105A3000206869202531352E30662052504D0A00ED
:105A40005B703163736C5D2070776D2063772073BA
:105A500070656564206C6F202531352E30662052CC
:105A6000504D0A005B70316672715D2070776D2059
:105A70006672657175656E63792020202531352E3B
:105A8000306620487A0A0053595354454D205245F8
:105A9000414459004C6F6164696E6720636F6E66A4
:105AA0006967732066726F6D20454550524F4D00F7
:105AB000496E697469616C697A696E6720636F6E9B
:105AC0006669677320746F2050726F626F746978B3
:105AD000204669726562616C6C20563930207072A4
:105AE0006F66696C65007B226572223A7B22666272
:105AF000223A25302E32662C227374223A25642CE9
:105B0000226D7367223A222573227D7D0A007B6510
:105B1000723A7B66623A25302E32662C73743A25CF
:105B2000642C6D73673A222573227D7D0A005B71B8
:105B3000765D20207175657565207265706F727471
:105B400020766572626F73697479253764205B30E3
:105B50003D6F66662C313D73696E676C652C323D16
:105B6000747269706C655D0A00716F3A25640A0091
:105B700071693A25640A0071723A25640A005B7300
:105B8000765D2020737461747573207265706F7216
:105B90007420766572626F73697479253664205B50
:105BA000303D6F66662C313D66696C746572656464
:105BB0002C323D766572626F73655D0A005B7369B6
:105BC0005D202073746174757320696E74657276DC
:105BD000616C2531342E3066206D730A004D6F7470
:105BE0006F7220256320706F77657220656E616229
:105BF0006C65642073746174653A25322E30660AD0
:105C0000005B257325735D206D257320706F7765AC
:105C100072206D616E6167656D656E7425313064EB
:105C2000205B303D64697361626C65642C313D6159
:105C30006C77617973206F6E2C323D696E206379C9
:105C4000636C652C333D7768656E206D6F76696E89
:105C5000675D0A005B257325735D206D25732070D9
:105C60006F6C617269747925313864205B303D6EE8
:105C70006F726D616C2C313D726576657273655D16
:105C80000A005B257325735D206D2573206D6963A4
:105C9000726F737465707325313664205B312C32FA
:105CA0002C342C385D0A005B257325735D206D252F
:105CB000732074726176656C2070657220726576EF
:105CC0006F6C7574696F6E2531302E346625730ADA
:105CD000005B257325735D206D25732073746570DB
:105CE00020616E676C652532302E336625730A009D
:105CF0005B257325735D206D2573206D61702074A5
:105D00006F206178697325313564205B303D582CF4
:105D1000313D592C323D5A2E2E2E5D0A005B6D749A
:105D20005D20206D6F746F722069646C65207469EA
:105D30006D656F75742531342E3266205365630AA4
:105D400000505D4C5D475D2064656700206D6D000F
:105D500020696E005B73745D2020737769746368DB
:105D6000207479706525313864205B303D4E4F2CAE
:105D7000313D4E435D0A0054657374202325642031
:105D80006E6F7420666F756E640A004E3620473958
:105D90003220583735205930205A300A4E372046A5
:105DA0003530302E300A4E3820473159302E3239B6
:105DB000315A2D322E3139380A4E39205837342E87
:105DC00037363759302E3035385A2D322E33353557
:105DD0000A4E3130205837342E373039592D302E75
:105DE0003030305A2D322E3337310A4E313120586F
:105DF00037342E3532395A2D322E3236340A4E315E
:105E000032205837342E36333459302E3130355A0B
:105E10002D322E3331390A4E3133205837342E3853
:105E2000343359302E3331345A2D322E3138330A2F
:105E30004E3134205837352E30303059302E3437EB
:105E4000315A2D322E3132360A4E31352059302E0C
:105E50003635305A2D322E3130300A4E31362058F8
:105E600037342E37383359302E3433345A2D322EBE
:105E70003133310A4E3137205837342E35363659C2
:105E8000302E3231375A2D322E3234340A4E3138D8
:105E9000205837342E333530592D302E3030305A8B
:105EA0002D322E3138320A4E3139205837342E31C6
:105EB00037305A2D322E3134340A4E323020583792
:105EC000342E34323959302E3235395A2D322E3162
:105ED00036350A4E3231205837342E353333593067
:105EE0002E3336335A2D322E3139310A4E3232208A
:105EF0005837342E36383959302E3531395A2D32FB
:105F00002E3131340A4E3233205837342E3834345F
:105F100059302E3637345A2D322E3039360A4E3219
:105F200034205837352E30303059302E3833305AEF
:105F30002D322E3131340A4E32352059312E303146
:105F4000305A2D322E3134340A4E323620583734FE
:105F50002E37383759302E3739375A2D322E3039BF
:105F6000380A4E3237205837342E36323859302ED0
:105F70003633385A2D322E3130380A4E32382058C6
:105F800037342E34363959302E3437385A2D322E94
:105F90003135370A4E3239205837342E333039599B
:105FA000302E3331395A2D322E3131300A4E3330C2
:105FB000205837342E30343459302E3035335A2D62
:105FC000322E3130380A4E3331205837332E39399A
:105FD0003059302E3030305A2D322E3037370A4E6D
:105FE0003332205837332E3831315A2D312E39344F
:105FF000370A4E3333205837332E39373359302E42
:106000003136325A2D322E3037390A4E3334205839
:1060100037342E32343359302E3433325A2D322E17
:106020003038340A4E3335205837342E3435395908
:10603000302E3634395A2D322E3135370A4E33361A
:10604000205837342E36373659302E3836355A2DBB
:10605000322E3130390A4E3337205837342E383308
:106060003859312E3032375A2D322E3131310A4ED5
:106070003338205837352E30303059312E313839B9
:106080005A2D322E3136300A4E33392059312E33C3
:1060900036395A2D322E3139340A4E3430205837A1
:1060A000342E38343259312E3231315A2D322E318C
:1060B00033340A4E3431205837342E36383459317F
:1060C0002E3035335A2D322E3132300A4E343220B2
:1060D0005837342E34323159302E3739305A2D3228
:1060E0002E3137360A4E3433205837342E3331367A
:1060F00059302E3638345A2D322E3133370A4E3439
:1061000034205837342E31353859302E3532365AFE
:106110002D322E3037370A4E3435205837332E394A
:10612000343759302E3331365A2D322E3036370A25
:106130004E3436205837332E38393459302E3236D3
:10614000335A2D322E3034360A4E343720583733F6
:106150002E37333759302E3130355A2D312E3931D3
:10616000380A4E3438205837332E36333159302ED2
:106170003030305A2D312E3837320A4E34392058CB
:1061800037332E3435325A2D312E3831350A4E35CB
:1061900030205837332E36363559302E3231345A76
:1061A0002D312E3931340A4E3531205837332E38BF
:1061B000323559302E3337345A2D322E3032380A98
:1061C0004E3532205837332E38373959302E343245
:1061D000375A2D322E3037360A4E35332058373461
:1061E0002E30393259302E3634315A2D322E303944
:1061F000340A4E3534205837342E33303659302E49
:106200003835345A2D322E3139320A4E3535205830
:1062100037342E35313959312E3036385A2D322E09
:106220003134310A4E3536205837342E373333590E
:10623000312E3238315A2D322E3134330A4E353721
:10624000205837342E38343059312E3338385A2DBF
:10625000322E3137340A4E3538205837342E3839FB
:106260003359312E3434325A2D322E3136390A4ECA
:106270003539205837352E30303059312E353438B5
:106280005A2D322E3132310A4E36302059312E37C6
:1062900032385A2D322E3037360A4E3631205837A2
:1062A000342E38343359312E3537315A2D322E3180
:1062B00033300A4E3632205837342E37333859317E
:1062C0002E3436365A2D322E3139350A4E36332099
:1062D0005837342E34373659312E3230345A2D3225
:1062E0002E3134370A4E3634205837342E32313579
:1062F00059302E3934335A2D322E3230320A4E363E
:1063000035205837332E39303059302E3632385AFE
:106310002D322E3130310A4E3636205837332E3852
:10632000343859302E3537365A2D322E3039360A18
:106330004E3637205837332E35383659302E3331D4
:10634000345A2D312E3931330A4E363820583733EE
:106350002E33373759302E3130355A2D312E3830D3
:10636000380A4E3639205837332E32373259302ECC
:106370003030305A2D312E3738370A4E37302058CA
:1063800037332E3138325A2D312E3738370A4E37BF
:1063900031205837332E3039325A2D312E3735309F
:1063A0000A4E3732205837332E34313059302E339D
:1063B00031385A2D312E3836380A4E373320583777
:1063C000332E37383159302E3638395A2D322E3057
:1063D00038360A4E3734205837342E30393959314F
:1063E0002E3030375A2D322E3232340A4E37352085
:1063F0005837342E32303559312E3131335A2D320F
:106400002E3231310A4E3736205837342E33363457
:1064100059312E3237325A2D322E3137360A4E3715
:1064200037205837342E36323959312E3533375AD2
:106430002D322E3139310A4E3738205837342E3626
:10644000383259312E3539305A2D322E3137370AFC
:106450004E3739205837342E38393459312E3830A8
:10646000325A2D322E3036360A4E383020583735D3
:106470002E30303059312E3930385A2D322E3034BA
:10648000360A4E38312059322E3038375A2D322EB6
:106490003035310A4E3832205837342E3833395996
:1064A000312E3932375A2D322E3036320A4E3833A9
:1064B000205837342E36373959312E3736365A2D43
:1064C000322E3133360A4E3834205837342E363295
:1064D0003559312E3731335A2D322E3137300A4E5D
:1064E0003835205837342E35373259312E36353934
:1064F0005A2D322E3138300A4E3836205837342E45
:1065000033353859312E3434355A2D322E31353712
:106510000A4E3837205837342E31393759312E3218
:1065200038345A2D322E3139350A4E383820583702
:10653000342E30393059312E3137375A2D322E32F0
:1065400034350A4E3839205837332E3938335931DB
:106550002E3037305A2D322E3232350A4E39302015
:106560005837332E38323359302E3931305A2D3294
:106570002E3133380A4E3931205837332E333934DF
:1065800059302E3438325A2D312E3931370A4E399E
:1065900032205837332E31383059302E3236385A6F
:1065A0002D312E3832350A4E3933205837322E39B4
:1065B000363659302E3035345A2D312E3731310A96
:1065C0004E3934205837322E393133592D302E3050
:1065D00030305A2D312E3639330A4E39352058375E
:1065E000322E3733335A2D312E3634360A4E393661
:1065F000205837322E39393759302E3236345A2D09
:10660000312E3735330A4E3937205837332E32364C
:106610003059302E3532375A2D312E3930320A4E1C
:106620003938205837332E36323959302E383936EA
:106630005A2D322E3037370A4E3939205837332EFB
:1066400038343059312E3130375A2D322E323234DF
:106650000A4E313030205837332E38393359312EE5
:106660003136305A2D322E3234350A4E3130312007
:1066700058373559305A300A004E312054314D3692
:106680000A4E32204731370A4E33204732310A4E04
:10669000382046313830300A4E392047310A4E31E1
:1066A00030302047393220582D32352E3137375986
:1066B0002D33342E303732205A2D312E30303020C9
:1066C0002854454D502C2052454D4F5645204C41A5
:1066D000544552290A4E33343320582D32352E3545
:1066E0003935592D33342E3334390A4E333434206E
:1066F000582D32352E373031592D33342E34333630
:106700000A4E33343520582D32352E373931592D34
:1067100033342E3532300A4E33343620582D32354C
:106720002E383634592D33342E3630310A4E333428
:106730003720582D32352E393230592D33342E36FC
:1067400037390A4E33343820582D32352E39363009
:10675000592D33342E3735340A4E33343920582DE1
:1067600032352E393832592D33342E3832360A4EDE
:1067700033353020582D32352E393837592D3334B2
:106780002E3839350A4E33353120582D32352E39D1
:106790003736592D33342E3936310A4E33353220BF
:1067A000582D32352E393438592D33352E30323379
:1067B0000A4E33353320582D32352E393033592D8A
:1067C00033352E3038320A4E33353420582D323599
:1067D0002E383431592D33352E3133380A4E333576
:1067E0003520582D32352E373633592D33352E314D
:1067F00039300A4E33353620582D32352E3636395B
:10680000592D33352E3233390A4E33353720582D32
:1068100032352E353539592D33352E3238340A4E2E
:1068200033353820582D32352E343333592D333506
:106830002E3332350A4E33353920582D32352E322B
:106840003931592D33352E3336330A4E3336302015
:10685000582D32352E313334592D33352E333937C7
:106860000A4E33363120582D32342E393633592DD5
:1068700033352E3432380A4E33363220582D3234E6
:106880002E373737592D33352E3435350A4E3336BA
:106890003320582D32342E353737592D33352E3499
:1068A00037370A4E33363420582D32342E333637AC
:1068B000592D33352E3439360A4E33363520582D7E
:1068C00032342E313434592D33352E3531310A4E90
:1068D00033363620582D32332E393039592D333551
:1068E0002E3532320A4E33363720582D32332E367B
:1068F0003631592D33352E3532390A4E333638205C
:10690000582D32332E343033592D33352E35333222
:106910000A4E33363920582D32332E313333592D28
:1069200033352E3533320A4E33373020582D32323C
:106930002E383533592D33352E3532370A2F4E3216
:1069400035313820473058302E333237592D3333D4
:106950002E3532315A2D312E3030300A4E3235310B
:1069600039204D3330004E31204732300A4E352029
:10697000473430204731370A4E3130205431204DD2
:1069800030360A284E3135204739302047302058DC
:1069900030205930205A30290A4E323020533530B9
:1069A0003030204D3033200A4E32352058302E30D2
:1069B00036342059302E333236205A300A4E343095
:1069C00020473031204631362E300A4E353020589F
:1069D000302E3036342059302E3332360A4E35358B
:1069E0002058302E3036302059302E3239330A4E6E
:1069F00036302058302E3037372059302E32363747
:106A00000A4E36352058302E3131312059302E3251
:106A100035370A4E37302058302E3134392059302E
:106A20002E3235320A4E37352058302E3138382044
:106A300059302E3235350A4E38302058302E323209
:106A4000372059302E3236380A4E38352058302EFD
:106A50003235372059302E3237310A4E39302058EE
:106A6000302E3333352059302E3236350A4E3935F3
:106A70002058302E3431322059302E3237310A4EE0
:106A80003130302058302E3437342059302E3238BF
:106A9000370A4E3130352058302E343931205930B4
:106AA0002E3238390A4E3131302058302E353137B8
:106AB0002059302E3237330A4E3131352058302E9E
:106AC0003534342059302E3236330A4E31323020AC
:106AD00058302E3538302059302E3236310A4E316A
:106AE00032352058302E3539352059302E32363354
:106AF0000A4E3133302058302E3632312059302E64
:106B00003237340A4E3133352058302E363539205D
:106B100059302E3330360A4E3134302058302E362C
:106B200037332059302E3333350A4E31343520581F
:106B3000302E3637392059302E3336310A4E313522
:106B4000302058302E3637382059302E3338390A15
:106B50004E3135352058302E3637302059302E34CE
:106B600032300A4E3136302058302E3637302059E8
:106B7000302E3434360A4E3136352058302E3638E1
:106B8000302059302E3437340A4E313730205830C7
:106B90002E3730342059302E3439370A4E313735BC
:106BA0002058302E3733322059302E3531350A4EA9
:106BB0003138302058302E3739342059302E353383
:106BC000350A4E3138352058302E3837322059307A
:106BD0002E3536370A4E3139302058302E3935307F
:106BE0002059302E3630340A4E3139352058312E66
:106BF0003033312059302E3634370A4E323030207F
:106C000058312E3134392059302E3732320A4E3233
:106C100030352058312E3330382059302E38353425
:106C20000A4E3231302058312E3433302059302E34
:106C30003938340A4E3231352058312E3434372029
:106C400059302E3938360A4E3232302058312E36ED
:106C500032382059302E3832320A4E3232352058EE
:106C6000312E3733322059302E3731340A4E3233F9
:106C7000302058322E3030392059302E3338310AF6
:106C80004E3233352058322E3131362059302E32A3
:106C900036360A4E3234302058322E3232382059AD
:106CA000302E3135370A4E3234352058322E3238B4
:106CB000302059302E3132330A4E3235302058329E
:106CC0002E3333322059302E3039340A4E32353596
:106CD0002058322E3432332059302E3037300A4E7D
:106CE0003236302058322E3438392059302E303652
:106CF000350A4E3236352058322E35353720593048
:106D00002E3036360A4E3237302058322E36323751
:106D10002059302E3038340A4E3237352058322E32
:106D20003639332059302E3130390A4E323830203E
:106D300058322E3733302059302E3133330A4E3209
:106D400038352058322E3830352059302E313930F0
:106D50000A4E3239302058322E3832392059302EEE
:106D60003231360A4E3239352058322E38383020FA
:106D700059302E3239310A4E3330302058322E38C5
:106D800038342059302E3330300A4E3330352058C5
:106D9000322E3839382059302E3333320A4E3331BF
:106DA000302058322E3930352059302E3336370ABC
:106DB0004E3331352058322E3931302059302E346F
:106DC00030370A4E3332302058322E39303820597D
:106DD000302E3434360A4E3332352058322E393084
:106DE000312059302E3439350A4E33333020583261
:106DF0002E3839372059302E3439350A4E33333551
:106E00002058322E3839302059302E3532340A4E3F
:106E10003334302058322E3834322059302E363028
:106E2000340A4E3334352058322E3831342059301C
:106E30002E3636350A4E3335302058322E37393417
:106E40002059302E3735300A4E3335352058322E02
:106E50003739312059302E3833380A4E3336302006
:106E600058322E3831392059302E3937360A4E33C0
:106E700036352058322E3833372059312E303434BD
:106E80000A4E3337302058322E3836322059312EC0
:106E90003131320A4E3337352058322E38373720C9
:106EA00059312E3134350A4E3338302058322E398C
:106EB00031322059312E3231370A4E33383520588D
:106EC000322E3931372059312E3232360A4E33398B
:106ED000302058322E3935312059312E3238310A8E
:106EE0004E3339352058322E3937302059312E3231
:106EF00039350A4E3430302058322E39393620593F
:106F0000312E3239350A4E3430352058332E303157
:106F1000332059312E3237350A4E34313020583330
:106F20002E3032342059312E3235340A4E34313538
:106F30002058332E3037302059312E3135310A4E1A
:106F40003432302058332E3037372059312E3133F8
:106F5000340A4E3432352058332E313235205931EF
:106F60002E3033390A4E3433302058332E313338F3
:106F70002059312E3031390A4E3433352058332ED2
:106F80003230352059302E3930380A4E34343020E2
:106F900058332E3238322059302E3739370A4E3492
:106FA00034352058332E3336312059302E3639318E
:106FB0000A4E3435302058332E3432362059302E94
:106FC0003539320A4E3435352058332E3435362093
:106FD00059302E3534330A4E3436302058332E345F
:106FE00037392059302E3439330A4E34363520584B
:106FF000332E3439342059302E3437320A4E343758
:10700000302058332E3530352059302E3434360A5E
:107010004E3437352058332E3531382059302E3400
:1070200031370A4E3438302058332E35333020591A
:10703000302E3339310A4E3438352058332E353618
:10704000342059302E3330300A4E34393020583302
:107050002E3537372059302E3235330A4E343935F4
:107060002058332E3536382059302E3231320A4EE0
:107070003530302058332E3534342059302E3137C6
:10708000360A4E3530352058332E353431205930BC
:107090002E3134360A4E3531302058332E353533C3
:1070A0002059302E3131390A4E3531352058332EA2
:1070B0003537362059302E3130360A4E35323020B1
:1070C00058332E3539372059302E3130320A4E356B
:1070D00032352058332E3631382059302E31303960
:1070E0000A4E3533302058332E3633392059302E5E
:1070F0003132390A4E3533352058332E363530206B
:1071000059302E3135390A4E3534302058332E3629
:1071100036332059302E3137380A4E353435205821
:10712000332E3637382059302E3139320A4E353524
:10713000302058332E3639392059302E3139370A1C
:107140004E3535352058332E3732332059302E31D5
:1071500039360A4E3536302058332E3736342059DA
:10716000302E3137390A4E3536352058332E3830E7
:10717000352059302E3136350A4E353730205833C8
:107180002E3838342059302E3135390A4E353735BE
:107190002058332E3934392059302E3136350A4EA5
:1071A0003538302058332E3936362059302E313785
:1071B000350A4E3538352058332E39373820593076
:1071C0002E3139340A4E3539302058332E3937387C
:1071D0002059302E3232330A4E3539352058332E6D
:1071E0003936302059302E3234350A4E3630302080
:1071F00058332E3833342059302E3331310A4E363D
:1072000030352058332E3736322059302E3334352E
:107210000A4E3631302058332E3732362059302E30
:107220003338390A4E3631352058332E3730332033
:1072300059302E3435380A4E3632302058332E36F7
:1072400038322059302E3533300A4E3632352058F8
:10725000332E3637392059302E3533340A4E3633F3
:10726000302058332E3632362059302E3638310AF7
:107270004E3633352058332E3536382059302E3897
:1072800032380A4E3634302058332E3434342059B4
:10729000312E3038300A4E3634352058332E3430C3
:1072A000352059312E3136370A4E36353020583395
:1072B0002E3430342059312E3136370A4E3635359A
:1072C0002058332E3338372059312E3230380A4E79
:1072D0003636302058332E3338342059312E323060
:1072E000380A4E3636352058332E3336352059314C
:1072F0002E3236350A4E3637302058332E33353558
:107300002059312E3238350A4E3637352058332E33
:107310003334382059312E3330380A4E3638302045
:1073200058332E3333332059312E3335300A4E360D
:1073300038352058332E3332312059312E333931FC
:107340000A4E3639302058332E3331312059312E00
:107350003432380A4E3639352058332E33333920FB
:1073600059312E3432330A4E3730302058332E34D0
:1073700034302059312E3430360A4E3730352058CB
:10738000332E3531302059312E3430380A4E3731D2
:10739000302058332E3538352059312E3432310AC9
:1073A0004E3731352058332E3631312059312E3475
:1073B00033390A4E3732302058332E363131205986
:1073C000312E3434310A4E3732352058332E36318F
:1073D000352059312E3434310A4E3733302058336A
:1073E0002E3633362059312E3438380A4E3733355D
:1073F0002058332E3633342059312E3531370A4E4A
:107400003734302058332E3632322059312E35342D
:10741000330A4E3734352058332E36303520593123
:107420002E3536330A4E3735302058332E35373621
:107430002059312E3537350A4E3735352058332E01
:107440003534342059312E3538310A4E3736302014
:1074500058332E3437392059312E3539320A4E37C8
:1074600036352058332E3435312059312E353938C0
:107470000A4E3737302058332E3338372059312EC3
:107480003632360A4E3737352058332E33393020CE
:1074900059312E3633360A4E3738302058332E3590
:1074A00033322059312E3630320A4E373835205893
:1074B000332E3630312059312E3539370A4E37398F
:1074C000302058332E3636382059312E3539380A87
:1074D0004E3739352058332E3738322059312E3631
:1074E00031320A4E3830302058332E373934205953
:1074F000312E3631380A4E3830352058332E383652
:10750000382059312E3633360A4E38313020583330
:107510002E3931382059312E3635350A4E3831352D
:107520002058332E3934352059312E3636370A4E0D
:107530003832302058332E3936342059312E3638EF
:10754000350A4E3832352058332E393637205931E6
:107550002E3638350A4E3833302058332E393734EA
:107560002059312E3639390A4E3833352058332ECA
:107570003938342059312E3732350A4E38343020DC
:1075800058332E3938342059312E3735380A4E3891
:1075900034352058332E3937302059312E37393091
:1075A0000A4E3835302058332E3934352059312E93
:1075B0003831370A4E3835352058332E3931382096
:1075C00059312E3832360A4E3836302058332E385C
:1075D00039312059312E3832370A4E383635205855
:1075E000332E3834322059312E3830390A4E38375C
:1075F000302058332E3739382059312E3738340A55
:107600004E3837352058332E3734362059312E37FF
:1076100037320A4E3838302058332E363938205910
:10762000312E3736340A4E3838352058332E36331B
:10763000352059312E3736360A4E383930205833F6
:107640002E3535332059312E3738350A4E383935F5
:107650002058332E3437382059312E3832300A4EE4
:107660003930302058332E3430392059312E3836C5
:10767000340A4E3930352058332E333435205931C1
:107680002E3931380A4E3931302058332E323634C3
:107690002059322E3032330A4E3931352058332EAC
:1076A0003234382059322E3035310A4E39323020BA
:1076B00058332E3234302059322E3038310A4E3978
:1076C00032352058332E3331362059322E30383669
:1076D0000A4E3933302058332E3339302059322E68
:1076E0003130340A4E3933352058332E343134207A
:1076F00059322E3132310A4E3934302058332E343B
:1077000033312059322E3135330A4E393435205831
:10771000332E3433332059322E3138300A4E393536
:10772000302058332E3432372059322E3230350A39
:107730004E3935352058332E3431332059322E32DC
:1077400032340A4E3936302058332E3339322059EC
:10775000322E3234320A4E3936352058332E3333F6
:10776000352059322E3234340A4E393730205833CE
:107770002E3237382059322E3233360A4E393735C9
:107780002058332E3235362059322E3234320A4EBA
:107790003938302058332E3233392059322E323591
:1077A000310A4E3938352058332E32313120593292
:1077B0002E3238300A4E3939302058332E31373492
:1077C0002059322E3335360A4E3939352058332E6A
:1077D0003135392059322E3339370A4E3130303075
:1077E0002058332E3135302059322E3433380A4E5A
:1077F000313030352058332E3134302059322E3448
:1078000038310A4E313031302058332E3133322066
:1078100059322E3531300A4E313031352058332E21
:107820003131382059322E3534330A4E313032302E
:107830002058332E3039392059322E3537360A4EFA
:10784000313032352058332E3035312059322E36F2
:1078500033310A4E313033302058332E303033201C
:1078600059322E3636360A4E313033352058322EC4
:107870003935372059322E3638350A4E31303430CA
:107880002058322E3930372059322E3639390A4EA7
:10789000313034352058322E3836302059322E3798
:1078A00031310A4E313035302058322E38313920BE
:1078B00059322E3732370A4E313035352058322E74
:1078C0003736382059322E3734350A4E313036307B
:1078D0002058322E3731362059322E3735370A4E5E
:1078E000313036352058322E3637352059322E3742
:1078F00035370A4E313037302058322E353739205F
:1079000059322E3733310A4E313037352058322E26
:107910003537302059322E3732330A4E3130383035
:107920002058322E3535392059322E3732300A4E12
:10793000313038352058322E3533302059322E37F9
:1079400030310A4E313039302058322E3530312026
:1079500059322E3639330A4E313039352058322ECD
:107960003437312059322E3638330A4E31313030E7
:107970002058322E3434332059322E3636380A4EBF
:10798000313130352058322E3339362059322E36A7
:1079900033340A4E313131302058322E33353420D1
:1079A00059322E3539310A4E313131352058322E87
:1079B0003335322059322E3539310A4E3131323099
:1079C0002058322E3332352059322E3534330A4E78
:1079D000313132352058322E3331352059322E355F
:1079E00032310A4E313133302058322E3330372085
:1079F00059322E3439380A4E313133352058322E2F
:107A00003239362059322E3436340A4E3131343040
:107A10002058322E3239332059322E3432370A4E22
:107A2000313134352058322E3239352059322E3307
:107A300036360A4E313135302058322E333231202D
:107A400059322E3330330A4E313135352058322EEB
:107A50003335382059322E3234370A4E31313630F0
:107A60002058322E3431392059322E3230330A4EDA
:107A7000313136352058322E3431392059322E31B9
:107A800037390A4E313137302058322E34303520D4
:107A900059322E3135380A4E313137352058322E91
:107AA0003336322059322E3132330A4E31313830AA
:107AB0002058322E3335342059322E3130340A4E8C
:107AC000313138352058322E3335342059322E306A
:107AD00039310A4E313139302058322E3338302086
:107AE00059322E3036350A4E313139352058322E42
:107AF0003431302059322E3035310A4E3132303067
:107B00002058322E3431302059322E3034370A4E3C
:107B1000313230352058322E3430352059322E3023
:107B200032380A4E313231302058322E343038203B
:107B300059322E3031300A4E313231352058322E02
:107B40003431362059312E3939350A4E31323230FE
:107B50002058322E3433332059312E3938320A4EE0
:107B6000313232352058322E3433382059312E39C3
:107B700036330A4E313233302058322E34343720E7
:107B800059312E3934380A4E313233352058322E9D
:107B90003436312059312E3933380A4E31323430AF
:107BA0002058322E3438302059312E3933310A4E94
:107BB000313234352058322E3437382059312E386E
:107BC00039390A4E313235302058322E3438372088
:107BD00059312E3837350A4E313235352058322E4C
:107BE0003530342059312E3835340A4E3132363062
:107BF0002058322E3532372059312E3834380A4E3B
:107C0000313236352058322E3534392059312E381C
:107C100034390A4E313237302058322E353737203A
:107C200059312E3836310A4E313237352058322EFE
:107C30003630342059312E3836360A4E313238300B
:107C40002058322E3633312059312E3835340A4EF1
:107C5000313238352058322E3634302059312E38D2
:107C600032370A4E313239302058322E36343020F5
:107C700059312E3739320A4E313239352058322EA9
:107C80003632392059312E3735390A4E31333030BA
:107C90002058322E3631322059312E3732370A4EA3
:107CA000313330352058322E3537362059312E3683
:107CB00039340A4E313331302058322E35333620A4
:107CC00059312E3636320A4E313331352058322E64
:107CD0003437302059312E3631360A4E3133323076
:107CE0002058322E3334352059312E3535310A4E55
:107CF000313332352058322E3330372059312E353A
:107D000032310A4E313333302058322E3236302061
:107D100059312E3438320A4E313333352058322E11
:107D20003234332059312E3437370A4E3133343020
:107D30002058322E3232382059312E3436390A4EFC
:107D4000313334352058322E3232322059312E34EC
:107D500034380A4E313335302058322E3232382002
:107D600059312E3432350A4E313335352058322EC2
:107D70003235342059312E3430350A4E31333630D5
:107D80002058322E3236382059312E3337330A4EAE
:107D9000313336352058322E3237392059312E338F
:107DA00034320A4E313337302058322E33303820B7
:107DB00059312E3238370A4E313337352058322E6A
:107DC0003334302059312E3235340A4E3133383085
:107DD0002058322E3430372059312E3230310A4E6D
:107DE000313338352058322E3434312059312E3148
:107DF00035360A4E313339302058322E343534205E
:107E000059312E3133310A4E313339352058322E23
:107E10003436302059312E3130360A4E313430303C
:107E20002058322E3436342059312E3130320A4E19
:107E3000313430352058322E3437312059312E30FC
:107E400033360A4E313431302058322E3436362013
:107E500059302E3937310A4E313431352058322ECF
:107E60003435312059302E3839370A4E31343230DA
:107E70002058322E3431352059302E3739310A4EC0
:107E8000313432352058322E3430332059302E37A9
:107E900036370A4E313433302058322E33383820BA
:107EA00059302E3736350A4E313433352058322E7C
:107EB0003330362059302E3834310A4E3134343094
:107EC0002058322E3232322059302E3931310A4E7A
:107ED000313434352058322E3131342059302E3956
:107EE00039350A4E313435302058322E3030322078
:107EF00059312E3037360A4E313435352058312E2F
:107F00003930352059312E3133390A4E313436303B
:107F10002058312E3735342059312E3232330A4E23
:107F2000313436352058312E3633372059312E3200
:107F300037380A4E313437302058312E3538322018
:107F400059312E3330310A4E313437352058312EE5
:107F50003535382059312E3331350A4E31343830E9
:107F60002058312E3436302059312E3335320A4ED6
:107F7000313438352058312E3339392059312E33A8
:107F800036300A4E313439302058312E33333820D0
:107F900059312E3335340A4E313439352058312E8B
:107FA0003238372059312E3332390A4E313530309C
:107FB0002058312E3234382059312E3239340A4E7D
:107FC000313530352058312E3231372059312E326B
:107FD00035340A4E313531302058312E323134208B
:107FE00059312E3235320A4E313531352058312E45
:107FF0003137322059312E3139350A4E3135323050
:108000002058312E3132382059312E3133390A4E31
:10801000313532352058312E3131302059312E3121
:1080200031370A4E313533302058302E393538202B
:1080300059302E3934310A4E313533352058302EEF
:108040003839312059302E3837330A4E31353430F3
:108050002058302E3832352059302E3830380A4EDC
:10806000313534352058302E3735352059302E37BC
:1080700034370A4E313535302058302E36313920DC
:1080800059302E3633330A4E313535352058302E9F
:108090003437372059302E3532360A4E31353630A6
:1080A0002058302E3437372059302E3532340A4E8E
:1080B000313536352058302E3431312059302E3478
:1080C00037360A4E313537302058302E3333312091
:1080D00059302E3435340A4E313537352058302E4C
:1080E0003237382059302E3432370A4E3135383055
:1080F0002058302E3233312059302E3339370A4E42
:10810000313538352058302E3138332059302E3320
:1081100037390A4E313539302058302E3133352039
:1081200059302E3336350A4E313539352058302EF8
:108130003037362059302E3334310A4E313630350F
:1081400020473030204633302E300A4E3136313021
:10815000204D3035200A4E31363135204739302018
:108160005830205930205A300A4E31363135204DA2
:1081700033300A28456E64206F6620434E432050FA
:10818000726F6772616D2900284D53472A2A2A2A87
:10819000204D6963726F7374657020546573742029
:1081A0005B76315D202A2A2A2A290A473030204767
:1081B0003137204732312047343020473439204787
:1081C0003830204739300A6730783079307A300AD1
:1081D0007B22316D69223A317D0A7B22326D692220
:1081E0003A317D0A7B22336D69223A317D0A7B2246
:1081F000346D69223A317D0A6730207831300A7B4C
:1082000022316D69223A327D0A78300A7B22316D43
:1082100069223A347D0A7831300A7B22316D692235
:108220003A387D0A78300A6730207931300A7B226B
:10823000326D69223A327D0A79300A7B22326D69C9
:10824000223A347D0A7931300A7B22326D69223A32
:10825000387D0A79300A6730207A31300A7B223340
:108260006D69223A327D0A7A300A7B22336D6922A7
:108270003A347D0A7A31300A7B22336D69223A38EA
:108280007D0A7A300A6730206131300A7B22346DF2
:1082900069223A327D0A61300A7B22346D69223AC2
:1082A000347D0A6131300A7B22346D69223A387D8F
:1082B0000A61300A6D3200284D53472A2A2A2A20A3
:1082C000436F6F7264696E617465206F6666736573
:1082D00074732074657374205B76315D202A2A2ABA
:1082E0002A290A673030673137673231673430679F
:1082F00034396738306739300A6735340A673932BC
:10830000783079307A300A663630300A284D534753
:108310002A2A2A2A207465737420473932206F660E
:1083200066736574732A2A2A2A290A286D7367538B
:1083300074657020313A204D6F76652066726F6DDE
:1083400020302C3020746F2033302C30206D6D2085
:10835000696E20706F73697469766520582064694E
:1083600072656374696F6E290A286D73675374654B
:108370007020323A205265736574206F72696769A4
:108380006E20746F20302E30207573696E67204721
:108390003932290A286D73675374657020333A2087
:1083A0004D6F766520746F2032302C302E2053684C
:1083B0006F756C64206D6F7665203230206D6D2096
:1083C000696E20706F7369746976652058206469DE
:1083D00072656374696F6E20616E6420737461747A
:1083E0007573207265706F72742073686F756C643A
:1083F0002073746172742066726F6D20302C302986
:108400000A286D73675374657020343A204D6F7677
:108410006520746F20302E3020202053686F756CDB
:1084200064206D6F7665203230206D6D20696E207E
:108430006E6567617469766520582064697265634A
:1084400074696F6E20616E6420737461747573203B
:108450007265706F72742073686F756C64207374CA
:108460006172742066726F6D2032302C30290A6779
:10847000317833300A67393278300A6731783230F0
:108480000A6731783079300A2473720A6739327892
:10849000300A673470302E350A284D53472A2A2A6D
:1084A0002A207465737420473535206F66667365BE
:1084B00074732A2A2A2A290A286D736753746570EF
:1084C00020313A2053657420436F6F7264696E6186
:1084D00074652073797374656D2032205B67353560
:1084E0005D20746F206F6666736574206F6620353B
:1084F000302C3530290A286D73675374657020322B
:108500003A2053656C6563742047353520636F6F7F
:108510007264696E6174652073797374656D290A7C
:10852000286D73675374657020333A204D6F7665FC
:1085300020746F20302C302E2048656164207368D1
:108540006F756C64206D6F766520646961676F6E0E
:10855000616C6C7920696E202B5820616E64202B31
:108560005920616E64207374617475732072657034
:108570006F72742073686F756C64207374617274A9
:108580002066726F6D20302C30290A6731304C32F2
:1085900070327835307935300A6735350A6730788A
:1085A0003079300A673470302E350A284D53472A07
:1085B0002A2A2A2074657374204735332061627338
:1085C0006F6C757465206F7665727269646573206F
:1085D0002A2A2A2A290A286D736753746570203164
:1085E0003A2052756E206120737175617265206941
:1085F0006E204735352073797374656D290A286DAF
:1086000073675374657020323A2052756E20612072
:1086100073717561726520772F473533206F7665EA
:108620007272696465290A6730783079300A673078
:1086300078323079300A67307832307932300A67F0
:108640003078307932300A6730783079300A6734E0
:1086500070302E350A6735336730783079300A67E5
:108660003533673078323079300A673533673078A0
:1086700032307932300A67353367307830793230CA
:108680000A6735336730783079300A673078307967
:10869000300A673470302E350A284D53472A2A2A6B
:1086A0002A20746573742052657475726E20746F1D
:1086B00020686F6D65202A2A2A2A290A286D736787
:1086C0005374657020313A2052657475726E20744F
:1086D0006F20686F6D65207573696E67204732384B
:1086E000290A286D73675374657020323A205265E9
:1086F00073657420746F2047353420636F6F726424
:108700002073797374656D290A6732380A673534C6
:108710000A6D333000284D53472A2A2A2A205465EF
:108720007374206163637572616379206F6620736F
:108730006C6F77206D6F766573205B76315D202AD4
:108740002A2A2A290A6735350A6730783079300AAB
:10875000673470302E350A673470302E350A673131
:108760007831306632320A6735340A6730783079CA
:10877000300A6D333000284D53472A2A2A2A2054C4
:1087800065737420766572792073686F7274206DDA
:108790006F766573205B76315D202A2A2A2A290AA2
:1087A0006730783079300A673470302E350A673197
:1087B00078302E3166313030300A78300A78302EF9
:1087C000310A78300A78302E310A78300A78302E23
:1087D000310A78300A78302E310A78300A78302E13
:1087E000310A78300A78302E310A78300A78302E03
:1087F000310A78300A78302E310A78300A78302EF3
:10880000310A78300A78302E310A78300A78302EE2
:10881000310A78300A78302E310A78300A78302ED2
:10882000310A78300A78302E310A673470302E35AC
:108830000A78300A78302E30310A78300A78302EB3
:1088400030310A78300A78302E30310A78300A78A0
:10885000302E30310A78300A78302E30310A7830B4
:108860000A78302E30310A78300A78302E30310ACA
:1088700078300A78302E30310A78300A78302E304D
:10888000310A78300A78302E30310A78300A783060
:108890002E30310A78300A78302E30310A78300A9A
:1088A00078302E30310A78300A78302E30310A672D
:1088B00030783079300A6D3200284D53472A2A2A01
:1088C0002A20526F746172792041786973204D6F4C
:1088D00074696F6E2054657374205B76315D202A55
:1088E0002A2A2A290A6730306731376732316734DC
:1088F000306734396738306739300A673078307913
:10890000307A306130623063300A6735350A67305B
:10891000783079300A6633363030300A6730613368
:1089200036300A623336300A633336300A61300A31
:1089300062300A63300A673161313434300A62319F
:108940003434300A63313434300A61300A62300A18
:1089500063300A6731613134343062373230633327
:1089600036300A783079307A306130623063300ADC
:1089700067317836306131343430623732306333C6
:1089800036300A783079307A306130623063300ABC
:10899000673178363079353061313434306237328E
:1089A00030633336300A783079307A306130623073
:1089B00063300A6731783630793530783235613155
:1089C00034343062373230633336300A78307930BD
:1089D0007A306130623063300A6735340A67307844
:1089E0003079300A6D333000284D53472A2A2A2A1D
:1089F00020496E76657273652054696D65204D6FF0
:108A000074696F6E2054657374205B76315D202A23
:108A10002A2A2A290A6730306731376732316734AA
:108A2000306734396738306739300A6735350A6757
:108A300030783079300A6739330A66302E30310A9F
:108A400067317831300A7931300A7A31300A613150
:108A5000300A78300A79300A7A300A61300A673190
:108A60007831307931307A2D31306131300A6730E8
:108A7000783079307A3061300A66302E310A6732C8
:108A8000783130792D31307A2D32306931300A67C2
:108A900030783079307A300A6733783130792D3157
:108AA000307A2D32306931300A6730783079307A57
:108AB000300A673278323079307A2D32306931308D
:108AC0000A6730783079307A300A67337832307913
:108AD000306931300A6730783079307A300A67325D
:108AE000783079307A2D33306931300A6733783015
:108AF00079307A306931300A6730783079307A30BD
:108B00000A67327830793069323020284357203371
:108B100036302064656772656573290A673378307B
:108B2000793069323020284343572033363020646F
:108B3000656772656573290A6739340A6735340ACF
:108B40006730783079300A6D3330007B22676322DA
:108B50003A226730306731376732316734306734F3
:108B600039673830673930227D0A7B226763223AC1
:108B700022673535227D0A7B226763223A226730DD
:108B800078307930227D0A7B226763223A2266356B
:108B90003030227D0A7B226763223A22284D5347D8
:108BA0007371756172657329227D0A7B2267632266
:108BB0003A226730783230227D0A7B226763223A7C
:108BC00022793230227D0A7B226763223A22783072
:108BD000227D0A7B226763223A227930227D0A7B3A
:108BE000226763223A226731783130227D0A7B2264
:108BF0006763223A22793130227D0A7B2267632221
:108C00003A227830227D0A7B226763223A22793029
:108C1000227D0A7B226763223A22284D53476369EB
:108C200072636C657329227D0A7B226763223A2274
:108C30006732783130792D3130693130227D0A7BCD
:108C4000226763223A22673078307930227D0A7BAE
:108C5000226763223A226733783130792D313069C7
:108C60003130227D0A7B226763223A2267307830D6
:108C70007930227D0A7B226763223A22673278327A
:108C8000307930693130227D0A7B226763223A22B3
:108C9000673078307930227D0A7B226763223A225E
:108CA00067337832307930693130227D0A7B226730
:108CB00063223A22673078307930227D0A7B22673E
:108CC00063223A22673278307930693130227D0A66
:108CD0007B226763223A22673378307930693130FA
:108CE000227D0A7B226763223A22673534227D0A7D
:108CF0007B226763223A22673078307930227D0AFE
:108D00007B226763223A226D3330227D00284D5347
:108D1000472A2A2A2A204D636F646573207465737D
:108D200074205B76315D202A2A2A2A290A67353584
:108D30000A6730783079300A6D330A673470310A47
:108D40006D350A673470310A6D340A673470310A40
:108D50006D350A673470310A6D370A673470310A2D
:108D60006D390A673470310A6D380A673470310A18
:108D70006D390A663530300A67307832300A793218
:108D8000300A6D330A78300A6D340A79300A6D354D
:108D90000A67317831300A6D370A7931300A6D3817
:108DA0000A78300A6D390A79300A673278313079B9
:108DB0002D31306931300A6D330A673078307930BF
:108DC0000A6D340A6733783130792D3130693130AA
:108DD0000A6D350A6730783079300A6D370A6732A4
:108DE00078323079306931300A6D380A673078303E
:108DF00079300A6D390A6733783230793069313029
:108E00000A6730783079300A6732783079306931E2
:108E1000300A6733783079306931300A6735340A7F
:108E20006730783079300A6D333000284D53472A47
:108E30002A2A2A2046656564686F6C64205465732D
:108E400074205B76315D202A2A2A2A290A284D536C
:108E5000472A2A2A2A204D616E75616C6C7920653B
:108E60006E746572202120616E64207E20647572AC
:108E7000696E67206D6F76656D656E7420746F2006
:108E800074657374202A2A2A2A290A6735350A67E5
:108E900030783079300A673470330A6730306731A0
:108EA0003767323167343067343967383067393083
:108EB0000A663630300A6730783130307637362EF1
:108EC0003736350A783079300A6735340A673078B2
:108ED0003079300A6D333000284D53472A2A2A2A28
:108EE000204477656C6C2054657374205B76315D2B
:108EF000202A2A2A2A290A67303067313767323117
:108F00006739300A6735350A6730783079300A6654
:108F10003530300A67307831300A673470310A678B
:108F2000307832300A673470310A67307831300A6D
:108F3000673470310A67307830300A673470310A2C
:108F400079350A6735340A6730783079300A6D33FD
:108F50000A673470310A67307831307931300A6D00
:108F6000350A673470310A67307832307932300A26
:108F70006D340A673470310A6730783330793330B2
:108F80000A6D380A673470310A67307834307934C2
:108F9000300A6D390A673470310A673078353079B4
:108FA00035300A6730783079300A6D3330004E3111
:108FB0002067303067313767323167343067343992
:108FC0006738306739300A4E313020673078307971
:108FD000300A4E323020663530300A4E333020674A
:108FE00032783130792D31306931302028435720A3
:108FF0003237302064656772656573290A4E3430F4
:10900000206730783079300A4E3530206733783138
:1090100030792D31306931302028434357203930A1
:109020002064656772656573290A4E3630206730A3
:10903000783079300A4E38302067327832307930E3
:1090400069313020284357203138302064656772F9
:10905000656573290A4E3730206730783079300AD9
:109060004E383020673378323079306931302028FB
:109070004343572031383020646567726565732932
:109080000A4E3930206730783079300A4E3939202D
:1090900046313230300A4E31303020673278307904
:1090A00030693230202843572033363020646567DA
:1090B00072656573290A4E31313020673278307914
:1090C00030693230202843572033363020616761C1
:1090D000696E290A4E3132302066373030202843FD
:1090E00068616E67652066656564207261746520DD
:1090F0007768696C6520696E204732206D6F7469EE
:109100006F6E206D6F6465290A4E313330206732EF
:109110007830793069323020284357203336302078
:109120003372642074696D65290A4E3134302067CA
:109130003278307930693230202843572033363046
:10914000203474682074696D65290A4E31353020E9
:10915000663530300A4E313630206733783079301A
:109160007A34306932302028434357203336302058
:10917000646567726565732077697468206C696ED1
:109180006561722074726176656C290A4E313730E0
:10919000206733783079307A306932302028434381
:1091A000572033363020616761696E290A4E3138A5
:1091B00030206637303020286D73672A2A2A2A43E8
:1091C00068616E67652066656564207261746520FC
:1091D0007768696C6520696E204733206D6F74690C
:1091E0006F6E206D6F64652A2A2A2A290A4E31394A
:1091F0003020673378307930693230202843435744
:1092000020333630203372642074696D65290A4E2C
:10921000323030206733783079306932302028435B
:10922000435720333630203474682074696D6529C3
:109230000A4E32313020286D73672A2A2A2A473194
:1092400038204576616C20746573742A2A2A2A298D
:109250000A4E323230204731205833302E373037E3
:10926000205A35302E37323720463530300A4E32CC
:1092700033302047313820473032205836372E37A8
:109280003338205A32332E36313720523235204689
:109290003235300A4E323430206738300A4E32359B
:1092A00030206730783079307A300A4E32363020CC
:1092B0006D333000284D53472A2A2A2A20537175CE
:1092C00061726573204D6F74696F6E20546573749D
:1092D000205B76315D202A2A2A2A290A67303067E6
:1092E000313767323167343067343967383067393E
:1092F000300A6730783079300A6730783230202889
:10930000747261766572736520612032306D6D20F4
:1093100073717561726520696E205820616E6420DA
:1093200059290A7932300A78300A79300A67317857
:109330003130663530302028647261772061203109
:10934000306D6D2073717561726520696E205820D3
:10935000616E6420592061742046353030290A79C5
:1093600031300A78300A79300A67307A3230202872
:10937000747261766572736520612032306D6D2084
:1093800073717561726520696E205820616E64206A
:109390005A290A7832300A7A300A78300A673178E6
:1093A00032307932307A3230663530302028666596
:1093B000656420612032306D6D20646961676F6E75
:1093C000616C20696E20582C205920616E64205AEF
:1093D000290A783079307A300A7834307934307A22
:1093E0003430202874726176657273652061203490
:1093F000306D6D206375626520696E20582C205990
:1094000020616E64205A290A78343079307A300A23
:1094100078307934307A34300A7834307934307AAC
:10942000300A783079307A34300A78307934307ACA
:10943000300A78343079307A34300A783079307ABA
:10944000300A6738300A6730783079300A67307808
:10945000310A673078300A6D333000284D53472A7F
:109460002A2A2A20486F6D696E672054657374201C
:109470005B76315D202A2A2A2A290A6732382E3261
:10948000783079307A300A6D333000284D53472ACE
:109490002A2A2A20536D6F6B652054657374205BF4
:1094A00076315D202A2A2A2A290A4730302047317E
:1094B000372047323120473430204734392047386D
:1094C00030204739300A6D33673470310A6D3567A3
:1094D0003470310A6D34673470310A6D336734701B
:1094E000310A6D35673470310A6D37673470310A6F
:1094F0006D39673470310A6D38673470310A6D39EF
:109500000A6730783079307A300A67303020783224
:10951000300A78300A7932300A79300A7A32300AE1
:109520007A300A6132300A61300A473030207832AE
:109530003020793230207A3230206132300A4730A0
:1095400030207830207930207A302061300A47305E
:109550003120663330207832207932207A3220610F
:10956000320A7830207930207A302061300A673032
:1095700078310A673078300A6D32002C000A0025F5
:109580007300256C750025312E3066002573002C84
:10959000000A0025733A25730025733A256C75007F
:1095A00025733A25312E30660025733A2573005B0A
:1095B00074765D20207465787420766572626F73AE
:1095C00069747925313564205B303D73696C656E53
:1095D000742C313D766572626F73655D0A00256695
:1095E0000A00256C750A0025640A0025730A0074B8
:1095F000696E7967205B25735D206572723A20255C
:10960000733A202573200074696E7967205B257397
:109610005D206F6B3E2000456E64206F6620636F97
:109620006D6D616E642066696C650A0008CD59CB6A
:1096300075CD96CDF5CD9ECBCDD059CB61D1CDD1C9
:10964000FBCF9ECB0000400640061040B800B8CDCE
:10965000D059CB61D1CDD1FBCF9ECB0000400620AD
:10966000060840B800B846D359CB64D2E2D291D4B0
:109670002DD2A0084006050609010846D359CB643F
:10968000D2E2D207CE9ECBB00840060540B0308073
:109690000000000000F0E0D0C0100100CF673322CE
:1096A000211F1B1301016E616E00696E66004E4141
:1096B0004E494E495459494E46CDCCCC3D0AD7234C
:1096C0003C17B7D13877CC2B329595E6241FB14F94
:1096D0000A000020410000C84200401C4620BCBED9
:1096E0004CCA1B0E5AAEC59D7400407A10F35A0046
:1096F000A0724E18090010A5D4E80000E8764817BB
:109700000000E40B54020000CA9A3B000000E1F59F
:1097100005000080969800000040420F000000A065
:109720008601000000102700000000E80300000090
:10973000006400000000000A0000000000010000BA
:109740000000002C76D888DC674F0823DFC1DFAE2D
:1097500059E1B1B796E5E3E453C63AE651997696F6
:10976000E8E6C28426EB898C9B62ED407C6FFCEFBF
:10977000BC9C9F40F2BAA56FA5F490055A2AF75CED
:10978000936B6CF9676DC11BFCE0E40D47FEF5209F
:10979000E6B500D0ED902E03009435770500808467
:1097A0001E080000204E0A000000C80C333333337B
:1097B0000F986E12831141EF8D2114893BE65516E7
:1097C000CFFEE6DB18D1844B381BF77C1D901DA41F
:1097D000BBE424203284725E228100C9F124ECA112
:1097E000E53D270011241FBECFEFCDBFDFE5DEBF73
:1097F00000E00CBF13E2A0E0B0E2E0E2F0ED01E037
:109800000BBF02C007900D92A439B107D9F72AE522
:10981000A4E9B3E201C01D92AA3DB207E1F70E949C
:109820007B840C940EE80C940000FC016081718133
:10983000828193810E94DFD960934A330895FC01AD
:1098400060817181828193810E94DFD96093493365
:109850000895AF92BF92CF92DF92EF92FF920F9353
:109860001F93CF93DF937B018C018DECC82E82E395
:10987000D82EE601AA24A394BC2EBC18F70161914E
:109880007191819191917F012CEA35EC47E257E388
:109890000E946EDB18164CF4F80140815181628100
:1098A00073818B2D0E94E985A8820C5F1F4F219642
:1098B000F2E3C33DDF0701F7DF91CF911F910F91D5
:1098C000FF90EF90DF90CF90BF90AF900C94F48515
:1098D000FC0160817181828193810E94DFD9609354
:1098E0004B33613019F481E00E94F07B81E00C94ED
:1098F000117CCF93DF93CDB7DEB76897CDBFDEBFC6
:10990000FC0160817181828193810E94DFD9609323
:109910004C3381E0613019F40E94F07B0CC00E944E
:10992000117CCE01019628E1FC0111922A95E9F7FC
:10993000BC010E94684C6896CDBFDEBFDF91CF911D
:1099400008950F931F93CF93DF93CDB7DEB72D9775
:10995000CDBFDEBF27E0E8EDF0E28E010F5F1F4FC5
:10996000D80101900D922A95E1F7BC01660F771F8F
:10997000680F791F660F771F660F771F660F771FB7
:109980006F5F794E45E050E0CE0108960E947EE57B
:10999000688570E0C8010E94ACE5009739F46B85DA
:1099A00070E0C8010E94ACE5009711F0801B01C077
:1099B0008FEF2D96CDBFDEBFDF91CF911F910F911D
:1099C0000895EF92FF920F931F93CF93DF938C0133
:1099D000F62EE72EEC012D96FC01618572858385BC
:1099E00094850E94DFD91F926F93DF93CF930F5E10
:1099F0001F4F1F930F93DF93CF93EF92FF92E6EDEC
:109A0000FAE581818F9380818F930E9445E6EDB7BF
:109A1000FEB73C96EDBFFEBFDF91CF911F910F9136
:109A2000FF90EF9008950F931F93CF93DF93EC0176
:109A3000162F072F8C819D810E94A14C83305CF5ED
:109A40008F3FA1F528C09E01235F3F4F9F938F93C7
:109A50008C858F938B858F938A858F9389858F9340
:109A60003F932F936196DF93CF933F932F930F9361
:109A70001F938091D75A8F938091D65A8F930E94CB
:109A800045E68DB79EB740968DBF9EBFDF91CF91C3
:109A90001F910F910895EBE7F4E1659174914FE404
:109AA00050E08EEC9DE30E947EE5CDCFE091433304
:109AB000F0E0EE0FFF1FE958FB4E659174914FE403
:109AC00050E08EEC9DE30E947EE5BDCF0F931F9387
:109AD000CF93DF93EC01162F072F8C819D810E947D
:109AE000A14C83307CF58F3FC1F52CC0AE014F5E99
:109AF0005F4F9E01235F3F4F9F938F938C858F9382
:109B00008B858F938A858F9389858F935F934F93EE
:109B10003F932F935F934F933F932F930F931F93F5
:109B20008091D75A8F938091D65A8F930E9445E6A1
:109B30008DB79EB742968DBF9EBFDF91CF911F918B
:109B40000F910895EBE7F4E1659174914FE450E0D3
:109B50008EEC9DE30E947EE5C9CFE0914333F0E0B7
:109B6000EE0FFF1FE958FB4E659174914FE450E0F2
:109B70008EEC9DE30E947EE5B9CFDF92EF92FF92DB
:109B80000F931F93CF93DF93CDB7DEB72897CDBF49
:109B9000DEBF8B01E42ED52E37E0EFEDF0E2DE01E3
:109BA000119601900D923A95E1F728870E94A14CF9
:109BB000F82E288582E08F1518F0E22FF0E002C021
:109BC000E2E0F0E0EE0FFF1FE958FB4E6591749163
:109BD0004FE450E08EEC9DE30E947EE59F938F93CF
:109BE000F80183818F9382818F9381818F9380810C
:109BF0008F93E1E0F0E0EC0FFD1FEF0DF11D808190
:109C00001F928F93DF92EF928091D75A8F9380911A
:109C1000D65A8F930E9445E6CDBFDEBF2896CDBFB2
:109C2000DEBFDF91CF911F910F91FF90EF90DF90FA
:109C300008954F925F926F927F92AF92BF92CF92B0
:109C4000DF92EF92FF920F931F93CF93DF93CDECB0
:109C5000D2E302E911E35C018991813009F042C04D
:109C6000F801C480D580E680F78040805180628012
:109C70007380A3019201C701B6010E94C2D79F77EA
:109C80002CEA35EC47E257E30E946BD987FD2AC0E6
:109C900020E034E244E759ECC701B6010E946EDBD4
:109CA00018165CF4F5012081318142815381C7018E
:109CB000B6010E946EDB181604F120E034E244E79E
:109CC00059ECC301B2010E946EDB18165CF4F50179
:109CD0002081318142815381C301B2010E946BD93D
:109CE00087FD0BC00B5C1F4FF4E0AF0EB11C82E38D
:109CF000C33DD80709F0B0CF02C08CED01C080E0B1
:109D0000DF91CF911F910F91FF90EF90DF90CF9057
:109D1000BF90AF907F906F905F904F90089580912B
:109D2000C932811105C08091C8328093C73229C0E1
:109D3000823031F487E08093C7328091C83221C0ED
:109D4000833031F489E08093C7328091C83219C0E2
:109D5000843031F48AE08093C7328091C83211C0D8
:109D60008091CA32813031F485E08093C73280918E
:109D7000C83207C0823019F486E08093C7328091E0
:109D8000C832863019F08091C73208958BE08093F5
:109D9000C73208958091C83208958093CA328130C5
:109DA00059F018F0823041F0089588EF92E38093E3
:109DB000F6329093F73208958DE197E58093F6326D
:109DC0009093F7320895FC0184810895845B9F4F3E
:109DD000FC0180810895855B9F4FFC01808108957F
:109DE000825B9F4FFC0180810895815B9F4FFC0146
:109DF00080810895875B9F4FFC01808108950C94BA
:109E0000EA9ACD96FC0160817181828193810895E7
:109E1000FC01648308958B5A9F4FFC016083089571
:109E20008F5B9F4FFC01408351836283738308954E
:109E30006093F8327093F9328093FA329093FB3248
:109E40008DEE91E20C942C66BF92CF92DF92EF924E
:109E5000FF920F931F93CF93DF93D09045337C01F4
:109E60000AE613E38091443390E0EC01CC0FDD1F50
:109E7000C80FD91FCC0FDD1FCC0FDD1FCC0FDD1F8E
:109E8000CF51DF4C81E0D816A9F0B881A981CA80F2
:109E9000BB804091BD33413091F4F8012081318184
:109EA000428153816B2F7A2F8C2D9B2D0E94C3D71B
:109EB0009B0109C020E030E080E090E004C02B2F3F
:109EC0003A2F8C2D9B2DA901BC01F701458F568F90
:109ED000678F70A3F4E0EF0EF11C0C5F1F4F249608
:109EE00083E30238180771F6DF91CF911F910F912C
:109EF000FF90EF90DF90CF90BF900895835B9F4FCE
:109F0000FC01608388EF92E30C94244F4F925F92A0
:109F10006F927F928F929F92AF92BF92CF92DF9279
:109F2000EF92FF920F931F93CF93DF93CDB7DEB7DE
:109F30006897CDBFDEBF8C016091BD3370E080E0DB
:109F400090E00E940DDA2B013C01F80160817181E3
:109F5000828193810E94DFD970E05B01AA0CBB1C57
:109F6000A60EB71EAA0CBB1CAA0CBB1CAA0CBB1CC1
:109F7000C5018F519F4C5C010AE613E3FE01319647
:109F80004F01F501C190D190E190F1905F01F8018E
:109F900061917191819191918F01A30192010E9430
:109FA00010DC9B01AC01C701B6010E94C3D7F401CC
:109FB00061937193819391934F01F3E302381F07EB
:109FC00001F7CE0101960E94CD9A88EF92E30E949C
:109FD000244F6896CDBFDEBFDF91CF911F910F91C7
:109FE000FF90EF90DF90CF90BF90AF909F908F90B9
:109FF0007F906F905F904F900895885F924369F4CF
:10A00000E62FF0E0EE0FFF1FEE0FFF1FEE5AFC4CA5
:10A0100060817181828193810895862F0C94C29A08
:10A02000CF92DF92EF92FF920F931F93CF93DF9324
:10A03000EC0182E3C83FD80709F04AC070E0FB0199
:10A04000EE0FFF1FEE0FFF1FEE5AFC4CC080D180B9
:10A05000E280F38080914533813059F1809144331F
:10A0600090E0FC01EE0FFF1FE80FF91FEE0FFF1F3E
:10A07000E60FF71FEE0FFF1FEE0FFF1FEF51FF4C14
:10A0800000811181B281A3812091BD332130B1F4CF
:10A09000FB01EE0FFF1FEE0FFF1FE659FC4C208166
:10A0A000318142815381B8018B2F9A2F0E94C3D7EF
:10A0B00008C060E070E080E090E003C0B8018B2F42
:10A0C0009A2F9B01AC01C701B6010E94C2D703C001
:10A0D000862F0E94D69AC55BDF4F2881211106C0CA
:10A0E00023E333E34BEC51E40E9472D9DF91CF912B
:10A0F0001F910F91FF90EF90DF90CF90089588E12E
:10A10000EDEFF2E3A2E5B3E301900D928A95E1F75A
:10A110008091413381110CC08091FC32813041F437
:10A120001092353310923633109237331092383301
:10A1300008954F925F926F927F928F929F92AF920B
:10A14000BF92CF92DF92EF92FF920F931F93CF9324
:10A15000DF93CDB7DEB76997CDBFDEBF8091C9323F
:10A16000811155C08091EE32813009F050C00E94BB
:10A17000F8CA81114CC01092EE3299EF692E90E32B
:10A18000792E26E3822E912C8E010E5E1F4F36EE25
:10A19000A32E30E2B32E33C0F70181917F011F92CD
:10A1A0008F935F924F92BF92AF921F930F930E9433
:10A1B00010E7B80181E593E20E9491638D839E834D
:10A1C000F60181919191A191B1916F018A879B874D
:10A1D000AC87BD87CE0101960E948060CDBFDEBFF7
:10A1E0009EEDE91690E2F906B9F6E8E16E0E711CF3
:10A1F000FFEF8F1A9F0A8CE38816910441F0240127
:10A2000089EDE82E80E2F82E630188E7C8CF80E070
:10A210006996CDBFDEBFDF91CF911F910F91FF9067
:10A22000EF90DF90CF90BF90AF909F908F907F90F6
:10A230006F905F904F9008952F923F924F925F9250
:10A240006F927F928F929F92AF92BF92CF92DF9246
:10A25000EF92FF920F931F93CF93DF93CDB7DEB7AB
:10A260002997CDBFDEBF4C015B0140904733509032
:10A270004533209044336090BD33709043336B017D
:10A280008DEF92E38887998759E8E52E51E3F52E03
:10A2900098E1299E100111248401D6016D917D91D0
:10A2A0008D919D916D012CEA35EC47E257E30E94B8
:10A2B0006BD987FD80C0F70180818150823008F022
:10A2C0007AC041104CC0F1E05F1609F1E885F985CC
:10A2D000E20DF31DEC51F2408081898391819D83D1
:10A2E000B281A381E1E06E1217C0E885F985E359D8
:10A2F000FF4F2081318142815381BC018B2F9A2FE6
:10A300000E94C3D769837D838E839F8307C0198290
:10A310001D821E821F8202C0BE83AF8371100CC0DB
:10A3200023E333E34BEC51E4D8016D917D918D91A2
:10A330009C910E9410DC05C0F801608171818281CE
:10A34000938129813D814E815F810E94C3D7A88579
:10A35000B9856D937D938D939C9313972CC0A8859D
:10A36000B9858D919D910D90BC91A02D89839A8383
:10A37000AB83BC8371100EC023E333E34BEC51E499
:10A38000F80160817181828193810E9410DC9B01C0
:10A39000AC0105C0D8012D913D914D915C91698131
:10A3A0007A818B819C810E94C3D7E885F98560837F
:10A3B000718382839383888599850496888799879A
:10A3C00095E3E90EF11C0C5F1F4FA885B985A950D4
:10A3D000B34309F062CF6090433370904733F091FC
:10A3E0004533F983C09044332091BD332D838CE0F5
:10A3F000A80EB11CA8E2B2E3A887B98749E0E42E11
:10A4000043E3F42EB8E1CB9E600111248401F501F1
:10A4100061917191819191915F012CEA35EC47E254
:10A4200057E30E946BD987FD8CC0A885B9858C91B4
:10A43000882309F486C08150823030F4F8012484E6
:10A440003584468457843BC0611016C023E333E350
:10A450004BEC51E4D8011C966D917D918D919C91AE
:10A460001F970E9410DC20E030E044EB53E40E9490
:10A4700010DC1B012C010DC020E030E044EB53E464
:10A48000F80164857585868597850E9410DC1B011F
:10A490002C012BED3FE049EC50E4A885B98591965D
:10A4A0006D917D918D919C9194970E9410DC9B0100
:10A4B000AC01C201B1010E9472D91B012C017110C3
:10A4C00031C0B981B130E1F0F701EC0DFD1DEC5167
:10A4D000F240A081B18192808380ED81E130A1F4CE
:10A4E000F701E359FF4F2081318142815381BD0142
:10A4F000892D982D0E94C3D7DB01982E892E04C088
:10A50000A0E0B0E0912C812CA2019101BD01892D28
:10A51000982D0E94C3D7D7016D937D938D939C9303
:10A5200013970FC0A2019101F701608171818281AF
:10A5300093810E94C3D7D7016D937D938D939C9394
:10A540001397E885F985F596E887F987F4E0EF0E2B
:10A55000F11C0C5F1F4F88859985875C924309F039
:10A5600056CF2996CDBFDEBFDF91CF911F910F91BE
:10A57000FF90EF90DF90CF90BF90AF909F908F9023
:10A580007F906F905F904F903F902F9008958091B3
:10A59000C5309091C6308F3E924111F08FE50895FD
:10A5A00080917C3490917D348F3E9241B9F78091B7
:10A5B0004E3390914F338F3E924181F78091C43357
:10A5C0009091C5338F3E924149F780917557909194
:10A5D00076578F3E924111F78091325890913358BF
:10A5E0008F3E9241D9F680E00895CF93C82F0E9404
:10A5F000EDAB82E08093C8328C2FCF91089580918B
:10A60000C932811104C083E08093C83203C085E061
:10A610008093C83280E00895CF93C82F0E945EB720
:10A6200080E00E94FFB28C2F0E94EDAB86E0809309
:10A63000C8328C2FCF9108958093423380E00895E3
:10A640008093433380E008958093473380E00895FA
:10A65000AF92BF92CF92DF92EF92FF920F931F9330
:10A66000CF93DF939FEF980F963008F041C0A090F2
:10A6700043337A018B0198E1899F60011124F6012F
:10A68000EB53FF4C6F01C0E0D0E0BB24B394F70163
:10A6900061917191819191917F012CEA35EC47E2B2
:10A6A00057E30E946EDB1816E4F4A1100CC023E3FC
:10A6B00033E34BEC51E4F801608171818281938135
:10A6C0000E9410DC05C0F801608171818281938154
:10A6D000F601EC0FFD1F648F758F868F978FB092F8
:10A6E000EE3224960C5F1F4FC831D10581F602C0AF
:10A6F0008EE601C080E0DF91CF911F910F91FF9016
:10A70000EF90DF90CF90BF90AF900895CF93DF93FD
:10A71000CDB7DEB76897CDBFDEBF80934433682FD7
:10A7200070E080E090E00E940BDA69837A838B838B
:10A730009C831D821E821F82188619861A861B869C
:10A740001C861D861E861F86188A198A1A8A1B8AED
:10A750001C8A1D8A1E8A1F8A188EAE014F5F5F4FAA
:10A76000BA0186E89FE40E942B8780E06896CDBFFF
:10A77000DEBFDF91CF910895CF93DF93E8EFF2E34F
:10A7800086E5DF011D928A95E9F78BE5A6ECB3E338
:10A79000ED01982F19929A95E9F7A1E2B4E3ED0142
:10A7A00019928A95E9F78FEE92E18093C5309093E4
:10A7B000C63080937C3490937D3480934E33909355
:10A7C0004F338093C4339093C533809375579093E0
:10A7D00076578093325890933358E093F632F09343
:10A7E000F7328091DE30809343338091DC300E94D9
:10A7F00086538091DD30809342338091DF308093A7
:10A8000046338091E0308093473381E08093413339
:10A810008093BE3394E09093FC321092EF3210920A
:10A82000F0321092F1328093C8328093C7320E9486
:10A830009DB1DF91CF910C946D88CF92DF92EF9212
:10A84000FF92CF93C82F6A017B01E82FF0E0DF0170
:10A85000AA0FBB1FAA0FBB1FAE5ABC4CCD92DD92F4
:10A86000ED92FC921397EE0FFF1FEE0FFF1FE350C8
:10A87000FD4CC082D182E282F382B701A6010E9420
:10A88000DE85B701A6018C2F0E94E985CF91FF904C
:10A89000EF90DF90CF900C94F4859F92AF92BF928F
:10A8A000CF92DF92EF92FF920F931F93CF93DF939C
:10A8B000CDB7DEB76897CDBFDEBF962EA72EC62ECA
:10A8C000D72E7C0100E010E0B12CF601619171916E
:10A8D000819191916F012CEA35EC47E257E30E9498
:10A8E0006EDB1816A4F58091433381110EC023E36B
:10A8F00033E34BEC51E4F7016081718182819381F4
:10A900000E9410DCAB01BC0105C0F7014081518100
:10A9100062817381E1E0F0E0EC0FFD1FE00FF11FB9
:10A920004083518362837383C8018B539F4CFC0126
:10A93000E357FD4F4083518362837383E555F109EB
:10A9400040835183628373838B2D0E94DE85B39491
:10A950000C5F1F4FF4E0EF0EF11C0831110509F0F8
:10A96000B4CF492D5A2DBE016F5F7F4F89E29CE421
:10A970000E942B8780E06896CDBFDEBFDF91CF912C
:10A980001F910F91FF90EF90DF90CF90BF90AF900D
:10A990009F9008954F925F926F927F928F929F92B5
:10A9A000AF92BF92CF92DF92EF92FF920F931F93DD
:10A9B000CF93DF93CDB7DEB76897CDBFDEBF21E081
:10A9C0002093BD3380904433909043335B016C01FE
:10A9D00002E513E3882D90E07C01EE0CFF1CE80EED
:10A9E000F91EEE0CFF1CEE0CFF1CEE0CFF1CC70149
:10A9F0008F519F4C7C01F5016191719181919191F1
:10AA00005F012CEA35EC47E257E30E946EDB181633
:10AA100064F5F7012081318142815381F801608121
:10AA20007181828193810E94C2D72B013C019110D8
:10AA30000EC023E333E34BEC51E4F60160817181F6
:10AA4000828193810E9410DC9B01AC0105C0F6015C
:10AA50002081318142815381C301B2010E94C2D75A
:10AA6000F801608F718F828F938FF4E0CF0ED11C2D
:10AA70000C5F1F4F84E0E80EF11C93E30A361907C0
:10AA800009F0B9CF682D70E080E090E00E940BDA09
:10AA900069837A838B839C831D821E821F82188622
:10AAA00019861A861B861C861D861E861F86188A96
:10AAB000198A1A8A1B8A1C8A1D8A1E8A1F8A188E66
:10AAC000AE014F5F5F4FBA0186E89FE40E942B877B
:10AAD00080E06896CDBFDEBFDF91CF911F910F91CF
:10AAE000FF90EF90DF90CF90BF90AF909F908F90AE
:10AAF0007F906F905F904F900895CF93DF93CDB785
:10AB0000DEB76897CDBFDEBF1092BD3310926A33B7
:10AB100010926B3310926C3310926D3310926E332F
:10AB200010926F331092703310927133109272330F
:10AB300010927333109274331092753310927633EF
:10AB400010927733109278331092793310927A33CF
:10AB500010927B3310927C3310927D3310927E33AF
:10AB600010927F331092803310928133609144337E
:10AB700070E080E090E00E940BDA69837A838B8337
:10AB80009C831D821E821F82188619861A861B8648
:10AB90001C861D861E861F86188A198A1A8A1B8A99
:10ABA0001C8A1D8A1E8A1F8A188EAE014F5F5F4F56
:10ABB000BA0186E89FE40E942B8780E06896CDBFAB
:10ABC000DEBFDF91CF910895CF93DF93CDB7DEB78E
:10ABD0006897CDBFDEBF1092BD336091443370E003
:10ABE00080E090E00E940BDA69837A838B839C83F8
:10ABF0001D821E821F82188619861A861B861C8655
:10AC00001D861E861F86188A198A1A8A1B8A1C8A24
:10AC10001D8A1E8A1F8A188EAE014F5F5F4FBA01D0
:10AC200086E89FE40E942B8780E06896CDBFDEBF58
:10AC3000DF91CF910895CF93DF93CDB7DEB76897BB
:10AC4000CDBFDEBF81E08093BD336091443370E0BF
:10AC500080E090E00E940BDA69837A838B839C8387
:10AC60001D821E821F82188619861A861B861C86E4
:10AC70001D861E861F86188A198A1A8A1B8A1C8AB4
:10AC80001D8A1E8A1F8A188EAE014F5F5F4FBA0160
:10AC900086E89FE40E942B8780E06896CDBFDEBFE8
:10ACA000DF91CF910895CF931092FC320E941C51F6
:10ACB0008091CF30813069F48DEF92E30E94194E7C
:10ACC000C82F882331F00E94EDAB82E08093C83218
:10ACD00017C088EF92E30E94244F85E08093C8322A
:10ACE0008091C932811105C081E08093C9320E94F0
:10ACF00000B088EF92E30E94F79A0E947F50C0E074
:10AD00008C2FCF91089588E1E2E5F3E3A2E8B3E365
:10AD100001900D928A95E1F780E008950F931F93BB
:10AD2000CF93DF93CDB7DEB76A97CDBFDEBF8C017F
:10AD300081E08093453388EF92E3698F7A8F0E9498
:10AD4000244F698D7A8DC8010E9453560E946586F2
:10AD50008823E1F388E1E0E0F0E2DE011196019062
:10AD60000D928A95E1F7BE016F5F7F4F82E893E312
:10AD70000E9453566A96CDBFDEBFDF91CF911F91DF
:10AD80000F91089588E1E2E5F3E3AAE9B3E30190C6
:10AD90000D928A95E1F780E008950F931F93CF936A
:10ADA000DF93CDB7DEB76A97CDBFDEBF8C0181E000
:10ADB0008093453388EF92E3698F7A8F0E94244F06
:10ADC000698D7A8DC8010E9453560E94658688233A
:10ADD000E1F388E1E0E0F0E2DE01119601900D92EE
:10ADE0008A95E1F7BE016F5F7F4F8AE993E30E9486
:10ADF00053566A96CDBFDEBFDF91CF911F910F9161
:10AE00000895FB01DC0180914133811111C09B0148
:10AE1000AD0160E070E080E89FE30E9472D960932A
:10AE2000353370933633809337339093383318C06B
:10AE300080914333811109C023E333E34BEC51E4A8
:10AE4000CD010E9410DCFB0101C0CD01AF01BC01AE
:10AE500040933533509336336093373370933833A0
:10AE600080E008958093413380E0089580934633D5
:10AE700080E0089560933D3370933E3380933F3379
:10AE8000909340330E94838780E008950F931F932F
:10AE9000CF93DF93EC018B0180914133882399F0AC
:10AEA0008091353390913633A0913733B091383358
:10AEB000BC01CD019F772CEA35EC47E257E30E94B5
:10AEC0006BD987FD30C081E08093FC32B801CE01A0
:10AED0000E941C518091CF30813069F48DEF92E354
:10AEE0000E94194EC82F882331F00E94EDAB82E0FA
:10AEF0008093C83219C088EF92E30E94244F85E006
:10AF00008093C8328091C932811105C081E080935D
:10AF1000C9320E9400B088EF92E30E94F79AC82FCE
:10AF20000E947F5001C0CEE88C2FDF91CF911F91FE
:10AF30000F910895CF93DF93CDB7DEB76897CDBF5C
:10AF4000DEBF682F70E080E090E00E940BDA69833A
:10AF50007A838B839C831D821E821F8218861986AA
:10AF60001A861B861C861D861E861F86188A198ACD
:10AF70001A8A1B8A1C8A1D8A1E8A1F8A188EAE0195
:10AF80004F5F5F4FBA0185E19CE40E942B8780E010
:10AF90006896CDBFDEBFDF91CF910895CF93DF9349
:10AFA000CDB7DEB76897CDBFDEBF60914A3370E0A2
:10AFB00080E090E00E940BDA69837A838B839C8324
:10AFC0001D821E821F82188619861A861B861C8681
:10AFD0001D861E861F86188A198A1A8A1B8A1C8A51
:10AFE0001D8A1E8A1F8A188EAE014F5F5F4FBA01FD
:10AFF0008FE19CE40E942B8780E06896CDBFDEBF86
:10B00000DF91CF910895CF93DF93CDB7DEB76897E7
:10B01000CDBFDEBF682F70E080E090E00E940BDAC9
:10B0200069837A838B839C831D821E821F8218868C
:10B0300019861A861B861C861D861E861F86188A00
:10B04000198A1A8A1B8A1C8A1D8A1E8A1F8A188ED0
:10B05000AE014F5F5F4FBA0188E69CE40E942B87E8
:10B0600080E06896CDBFDEBFDF91CF910895CF938A
:10B07000DF93CDB7DEB76897CDBFDEBF682F70E036
:10B0800080E090E00E940BDA69837A838B839C8353
:10B090001D821E821F82188619861A861B861C86B0
:10B0A0001D861E861F86188A198A1A8A1B8A1C8A80
:10B0B0001D8A1E8A1F8A188EAE014F5F5F4FBA012C
:10B0C00089E79CE40E942B8780E06896CDBFDEBFB5
:10B0D000DF91CF910895CF93FC01608171818281CE
:10B0E00093810E94DFD96093C8321092CA3288EFF0
:10B0F00092E38093F6329093F7328091C932813097
:10B1000011F41092C9321092CB321092F1320E9497
:10B11000B09AC091C832C430C9F40E947D55809164
:10B12000DC300E9486538091DD30809342338091E1
:10B13000E0308093473380E00E94FFB280E00E94BD
:10B14000375881E080934133C093FC3281E0CF9146
:10B150000C94C4AE8093BA338093BB338093C333D3
:10B1600080E008952CEA35EC47E257E360916834BB
:10B170007091693480916A3490916B340E946EDBD7
:10B180001816B4F480910D3490910E34A0910F34C0
:10B19000B0911034BC01CD019F772CEA35EC47E229
:10B1A00057E30E946BD987FF03C01092BA3303C0E4
:10B1B00081E08093BA3380E008958093BA33809120
:10B1C0000D3490910E34A0910F34B09110348093CF
:10B1D000B2339093B333A093B433B093B53380E0DC
:10B1E00008952CEA35EC47E257E36091683470919A
:10B1F000693480916A3490916B340E946EDB18162A
:10B20000B4F480910D3490910E34A0910F34B0912C
:10B210001034BC01CD019F772CEA35EC47E257E3AF
:10B220000E946BD987FF03C01092BB3303C081E03B
:10B230008093BB3380E008958093BB3380910D34BD
:10B2400090910E34A0910F34B09110348093B633A6
:10B250009093B733A093B833B093B93380E0089597
:10B260002CEA35EC47E257E3609168347091693419
:10B2700080916A3490916B340E946EDB1816B4F49E
:10B2800080910D3490910E34A0910F34B091103410
:10B29000BC01CD019F772CEA35EC47E257E30E94D1
:10B2A0006BD987FF03C01092C33303C081E0809342
:10B2B000C33380E008958093C33380910D3490911F
:10B2C0000E34A0910F34B09110348093BF3390931B
:10B2D000C033A093C133B093C23380E00895BC0162
:10B2E0008DEE90E20C944F6681E08093EF320895EA
:10B2F00081E08093F032089581E08093F1320895E7
:10B300001F93CF93DF93CDB7DEB76897CDBFDEBF76
:10B310000E94EA9A8130B9F10E9409D60E94E8861B
:10B3200080E00E9415B010E0812F0E94C29AAB010C
:10B33000BC01812F0E941D541F5F1630A9F780E0C9
:10B3400090E0A0E4B0E489839A83AB83BC831D8240
:10B350001E821F82188619861A861B861C861D86E9
:10B360001E861F86188A198A1A8A1B8A1C8A1D8AB9
:10B370001E8A1F8A188EBE016F5F7F4FCB010E940D
:10B380006B5880E001C08AE66896CDBFDEBFDF91D2
:10B39000CF911F9108958091EF328130A9F42091CF
:10B3A000CA32213079F48091CB3281110BC082E016
:10B3B0008093CA328DE197E58093F6329093F7320D
:10B3C0002093CB321092EF328091F032813091F4A1
:10B3D0008091CA32882331F0823061F49091CB326F
:10B3E000943051F40E94EA9A811104C01092F03214
:10B3F0000E9480599091CB328091F1328130C1F41A
:10B400002091F032211114C09150933088F01092A5
:10B41000F13295E09093CB329093C8329091C9323B
:10B42000911104C08093C9320E9400B00E945CA3B5
:10B4300080E0089585E08093C8328091C9328111FF
:10B4400005C081E08093C9320C9400B00895CF9379
:10B45000DF93CDB7DEB76897CDBFDEBF8091C9322D
:10B46000882311F180E090E0A0E4B0E489839A831E
:10B47000AB83BC831D821E821F82188619861A86A2
:10B480001B861C861D861E861F86188A198A1A8AA4
:10B490001B8A1C8A1D8A1E8A1F8A188EBE016F5F36
:10B4A0007F4FCB010E946B586896CDBFDEBFDF9106
:10B4B000CF910895CF93DF93CDB7DEB76897CDBF17
:10B4C000DEBF80E090E0A0E4B0E489839A83AB83A0
:10B4D000BC831D821E821F82188619861A861B86CF
:10B4E0001C861D861E861F86188A198A1A8A1B8A40
:10B4F0001C8A1D8A1E8A1F8A188EAE014F5F5F4FFD
:10B50000BA018BE698E50E942B876896CDBFDEBF17
:10B51000DF91CF910895CF93DF93CDB7DEB76897D2
:10B52000CDBFDEBF80E090E0A0E8B0E489839A83DD
:10B53000AB83BC831D821E821F82188619861A86E1
:10B540001B861C861D861E861F86188A198A1A8AE3
:10B550001B8A1C8A1D8A1E8A1F8A188EAE014F5FA5
:10B560005F4FBA018BE698E50E942B876896CDBFA6
:10B57000DEBFDF91CF910895CF93DF93CDB7DEB7D4
:10B580002797CDBFDEBF97E0EFEDF0E2DE01119629
:10B5900001900D929A95E1F7873050F4E1E0F0E0E8
:10B5A000EC0FFD1FE80FF11D87FDFA95808101C0AA
:10B5B00080E22796CDBFDEBFDF91CF910895EF9255
:10B5C000FF920F931F93CF93DF931F92CDB7DEB7F8
:10B5D0007C018B01642F70E080E090E049830E9441
:10B5E0000BDAF701618772878387948782E087830C
:10B5F0004981E42FF0E0EE0FFF1FE00FF11F65918E
:10B6000074914FE450E08EEC9DE30E947EE5BC0116
:10B61000C7010F90DF91CF911F910F91FF90EF9095
:10B620000C94F165CF93DF93EC010E948F4E482F6D
:10B6300065EB73E1CE01DF91CF910C94DF5A40911D
:10B64000C83266E773E10C94DF5A4091C9326DE469
:10B6500073E10C94DF5A4091CA3269E373E10C94B0
:10B66000DF5A4091CB326BE073E10C94DF5A40918A
:10B67000CC326EEE72E10C94DF5AE091F632F0912A
:10B68000F732E55BFF4F408168E174E10C94DF5ACB
:10B69000E091F632F091F732E45BFF4F408164E2D3
:10B6A00072E10C94DF5AE091F632F091F732448166
:10B6B0006AE871E10C94DF5AE091F632F091F732CA
:10B6C000E65BFF4F408167E571E10C94DF5AE09142
:10B6D000F632F091F732E25BFF4F40816DE071E1AD
:10B6E0000C94DF5AE091F632F091F732E15BFF4FB4
:10B6F00040816CEC70E10C94DF5AE091F632F091ED
:10B70000F732E75BFF4F40816DE570E10C94DF5A43
:10B71000CF93DF93EC01E091F632F091F732EF5ADC
:10B72000FF4F608170E080E090E00E940BDA698753
:10B730007A878B879C8782E08F8380E0DF91CF912F
:10B740000895CF93DF93EC016091F8327091F93254
:10B750008091FA329091FB320E940BDA69877A87E6
:10B760008B879C8782E08F8380E0DF91CF91089563
:10B77000CF93DF93EC01E091F632F091F7326081E4
:10B780007181828193810E940BDA69877A878B8726
:10B790009C8782E08F8380E0DF91CF910895CF93E3
:10B7A000DF93EC018091CA32811105C019861A8697
:10B7B0001B861C8614C00E94B99A69877A878B877A
:10B7C0009C872091685721110AC025E832E441E2A4
:10B7D0005DE30E9410DC69877A878B879C878C8168
:10B7E0009D81FC01EE0FFF1FE80FF91FEE0FFF1FF9
:10B7F000EE0FFF1FEE0FFF1FE85FF94E859194914A
:10B80000888784E08F8380E0DF91CF910895CF9384
:10B81000DF93EC012091F6323091F732F901FD9679
:10B82000608171818281938169877A878B879C8708
:10B830003E96208121110AC025E832E441E25DE311
:10B840000E9410DC69877A878B879C878C819D8119
:10B85000FC01EE0FFF1FE80FF91FEE0FFF1FEE0FA9
:10B86000FF1FEE0FFF1FE85FF94E859194918887C7
:10B8700084E08F8380E0DF91CF910895CF93DF93B1
:10B88000EC018C819D810E94A14C682F8091F63241
:10B890009091F7320E94105069877A878B879C8736
:10B8A0008C819D81FC01EE0FFF1FE80FF91FEE0F49
:10B8B000FF1FEE0FFF1FEE0FFF1FE85FF94E859190
:10B8C0009491888784E08F8380E0DF91CF91089501
:10B8D000CF93DF93EC018C819D810E94A14C20913C
:10B8E000F6323091F732285F324369F4E82FF0E006
:10B8F000EE0FFF1FEE0FFF1FEE5AFC4C60817181AF
:10B900008281938102C00E94C29A69877A878B875D
:10B910009C878C819D81FC01EE0FFF1FE80FF91FB2
:10B92000EE0FFF1FEE0FFF1FEE0FFF1FE85FF94E38
:10B9300085919491888784E08F8380E0DF91CF9117
:10B940000895CF93DF93EC018C819D810E94A14CDF
:10B95000E091F632F091F73294E0899FE00DF11D0D
:10B960001124458D568D678D70A149875A876B8745
:10B970007C878C819D81FC01EE0FFF1FE80FF91F72
:10B98000EE0FFF1FEE0FFF1FEE0FFF1FE85FF94ED8
:10B9900085919491888784E08F8380E0DF91CF91B7
:10B9A0000895CF93DF93EC010E94646169857A85E5
:10B9B0008B859C850E94DFD9462F64E474E1CE011B
:10B9C000DF91CF910C94DF5ACF93DF93EC018C8100
:10B9D0009D810E94A14C833054F48F3FA9F407C08D
:10B9E000CE010E940E6280E01CC08DE61AC020E0ED
:10B9F00030E040E450E469857A858B859C850E941F
:10BA00006EDB181694F3ECCF20E030E040E050E419
:10BA100069857A858B859C850E946EDB18162CF3D0
:10BA2000DFCFDF91CF91089595E3899FF001112435
:10BA3000E656FE4C60817181828193810895CF9298
:10BA4000DF92EF92FF92CF93DF936A017B0125E3B0
:10BA5000829FC00111248B539F4CFC01EB52FF4F7E
:10BA60004083518362837383EC01C352DF4F20E034
:10BA700034E244E759E4C701B6010E9410DC9B019F
:10BA8000AC0160E070E080E89FE30E9472D96883B7
:10BA900079838A839B83DF91CF91FF90EF90DF9032
:10BAA000CF900895CF92DF92EF92FF92CF93DF93E2
:10BAB000EC01C984DA84EB84FC8420E034E244E7BE
:10BAC00059E4C701B6010E946EDB181664F420E049
:10BAD00034E244E759E4C701B6010E9472D969878C
:10BAE0007A878B879C87CE010E940B67C984DA8492
:10BAF000EB84FC848C819D810E94A14C25E3829F74
:10BB0000C00111248B539F4CFC01EB52FF4FC082AC
:10BB1000D182E282F382EC01C352DF4F20E034E2B3
:10BB200044E759E4C701B6010E9410DC9B01AC0157
:10BB300060E070E080E89FE30E9472D968837983B7
:10BB40008A839B8380E0DF91CF91FF90EF90DF901D
:10BB5000CF900895CF92DF92EF92FF92CF93DF9331
:10BB6000EC01C984DA84EB84FC8420E034E244E70D
:10BB700059E4C701B6010E946EDB181664F420E098
:10BB800034E244E759E4C701B6010E9472D96987DB
:10BB90007A878B879C87CE010E940B6780E0DF91BC
:10BBA000CF91FF90EF90DF90CF90089581E0809348
:10BBB000F03280E008952CEA35EC47E257E3FC01CF
:10BBC00061857285838594850E946EDB181614F456
:10BBD0000E941C6F80E008956091F2327091F33200
:10BBE0008091F4329091F53208950E941A6380E0BA
:10BBF0000E949F7180E008950E941A6381E00E9474
:10BC00009F7180E008950E941A6382E00E949F71F4
:10BC100080E008950E941A6383E00E949F7180E093
:10BC20000895CF93DF93EC01E091F632F091F73273
:10BC3000E55BFF4FE081F0E0EE0FFF1FE958FB4EA0
:10BC4000659174914FE450E08EEC9DE30E947EE597
:10BC5000AC0166E470E1CE01DF91CF910C944FC648
:10BC6000CF93DF93EC01E091F632F091F732E55B90
:10BC7000FF4FE081F0E0EE0FFF1FE958FB4E6591AA
:10BC800074914FE450E08EEC9DE30E947EE5AC01A0
:10BC90006EE270E1CE01DF91CF910C944FC6CF934D
:10BCA000DF93EC0181EF90E20E94E3E6CE010E9477
:10BCB000115ECE010E94305E6AE170E1CE010E9409
:10BCC00016C661E070E1CE010E94E1C568EE7FE03A
:10BCD000CE010E94E1C56FEC7FE0CE010E94E1C57C
:10BCE00066EB7FE0CE010E94E1C56DE97FE0CE0109
:10BCF0000E94E1C564E87FE0CE010E94E1C56BE6E9
:10BD00007FE0CE010E94E1C562E57FE0CE010E94A6
:10BD1000E1C569E37FE0CE010E94E1C560E27FE01A
:10BD2000CE010E94E1C567E07FE0CE010E94E1C53F
:10BD30006EEE7EE0CE010E94E1C565ED7EE0CE01B3
:10BD40000E94E1C56CEB7EE0CE010E9416C680E049
:10BD5000DF91CF9108956AE170E10C9416C661E01D
:10BD600070E10C94E1C568EE7FE00C94E1C56FECE6
:10BD70007FE00C94E1C566EB7FE00C94E1C56DE9D2
:10BD80007FE00C94E1C564E87FE00C94E1C56BE6CC
:10BD90007FE00C94E1C562E57FE00C94E1C569E3C6
:10BDA0007FE00C94E1C560E27FE00C94E1C567E0C0
:10BDB0007FE00C94E1C56EEE7EE00C94E1C565ED8C
:10BDC0007EE00C94E1C56CEB7EE00C9416C660E45A
:10BDD0007EE00C9416C66FE07EE00C9416C66AED09
:10BDE0007DE00C9416C66FE97DE00C9416C66BE6F8
:10BDF0007DE00C9416C6CF93DF93EC01E091F63210
:10BE0000F091F732E55BFF4FE081F0E0EE0FFF1FAE
:10BE1000E958FB4E659174914FE450E08EEC9DE340
:10BE20000E947EE5AC0167E47DE0CE01DF91CF9119
:10BE30000C944FC6CF93DF93EC01E091F632F09172
:10BE4000F732E55BFF4FE081F0E0EE0FFF1FE958AE
:10BE5000FB4E659174914FE450E08EEC9DE30E949F
:10BE60007EE5AC0166E27DE0CE01DF91CF910C94DE
:10BE70004FC669E07DE00C94F7C5CF93DF93EC01EA
:10BE8000E091F632F091F732E55BFF4FE081F0E0B0
:10BE9000EE0FFF1FE958FB4E659174914FE450E09F
:10BEA0008EEC9DE30E947EE5AC016AEE7CE0CE0163
:10BEB000DF91CF910C944FC60F931F93CF93DF93D5
:10BEC0008C01FC0161857285838594850E94DFD990
:10BED000E62FF0E0EE0FFF1FEC5BFB4E65917491D7
:10BEE0004FE450E08EEC9DE30E947EE5E8012D9644
:10BEF0009F938F93F80161857285838594850E9455
:10BF0000DFD91F926F93DF93CF930F5E1F4F1F9365
:10BF10000F93DF93CF938EEC9CE09F938F93E6ED8E
:10BF2000FAE581818F9380818F930E9445E6EDB77A
:10BF3000FEB73E96EDBFFEBFDF91CF911F910F91EF
:10BF4000089566EA7CE00C94134D6EE77CE00C9457
:10BF5000134D6CE57CE00C94134D6AE37CE00C948B
:10BF6000134D68E07CE00C94134D67ED7BE00C947E
:10BF7000134D6EE97BE00C94134D6EE77BE00C945F
:10BF8000134D6CE37BE00C94E14C6AEF7AE00C9487
:10BF9000E14C63ED7AE00C94134D6DEA7AE00C9479
:10BFA000134D6CE87AE00C94134D6CE67AE00C9437
:10BFB000134D6FE47AE00C94664D60E37AE00C94E4
:10BFC000664DBC01675F7F4F2091433346EA5EE0D8
:10BFD000FC01848195810C94BD4DBC01675F7F4F4E
:10BFE00021E04CE85EE0FC01848195810C94BD4D1C
:10BFF000BC01675F7F4F21E043E75EE0FC01848185
:10C0000095810C94BD4D0F931F93CF93DF93EC015B
:10C010000C811D810E94D66808171907C4F48C8111
:10C020009D81FC01EE0FFF1FE80FF91FEE0FFF1FB0
:10C03000EE0FFF1FEE0FFF1FE35FF94E25913491C6
:10C04000CE01F901DF91CF911F910F91199485E1F4
:10C05000DF91CF911F910F9108950F931F93CF936D
:10C06000DF93EC010C811D810E94D6680817190727
:10C07000C4F48C819D81FC01EE0FFF1FE80FF91FB6
:10C08000EE0FFF1FEE0FFF1FEE0FFF1FE55FF94ED4
:10C0900025913491CE01F901DF91CF911F910F913C
:10C0A000199485E1DF91CF911F910F9108950F931E
:10C0B0001F93CF93DF93EC010C811D810E94D66802
:10C0C00008171907C4F48C819D81FC01EE0FFF1F36
:10C0D000E80FF91FEE0FFF1FEE0FFF1FEE0FFF1F00
:10C0E000E75FF94E25913491CE01F901DF91CF91AF
:10C0F0001F910F911994DF91CF911F910F91089586
:10C10000CF93DF93EC018C819D810E94E9688823A5
:10C11000C9F08C819D81FC01EE0FFF1FE80FF91F14
:10C12000EE0FFF1FEE0FFF1FEE0FFF1FE95FF94E2F
:10C13000E491E1FF05C0CE01DF91CF910C9404851D
:10C1400080E001C085E1DF91CF9108950F931F93A7
:10C15000CF93DF93EC0181E00E9420531C821D826B
:10C1600080E090E08E010F5E1F4F47C08C819D8163
:10C170009C01220F331FF901E80FF91FEE0FFF1F7B
:10C18000EE0FFF1FEE0FFF1FE95FF94EE491E0FF96
:10C190002EC0280F391F220F331F220F331F220FEB
:10C1A000331F2F5E394EF901459155916591749178
:10C1B00049875A876B877C87BC01660F771F680F9A
:10C1C000791F660F771F660F771F660F771F6F5FE8
:10C1D000794E45E050E0C8010E947EE5CE010E9404
:10C1E0000360CE010E9480602C813D8101C09C01D2
:10C1F0002F5F3F4F2C833D83C9010E94D968811175
:10C20000B5CF81E00E9473ACDF91CF911F910F9168
:10C210000C945BACCF93DF93EC012CEA35EC47E256
:10C2200057E369857A858B859C850E946BD987FF4A
:10C2300005C0CE01DF91CF910C94FE7DCE010E940E
:10C24000A66082E08F8340E050E060E87FE34987AA
:10C250005A876B877C8780E0DF91CF91089580912A
:10C26000BE3A9091BF3A8F3E924111F08AE508950F
:10C270008091003B9091013B8F3E9241B9F78091B4
:10C280009435909195358F3E924181F78091B638E3
:10C290009091B7388F3E924149F78091B83890918C
:10C2A000B9388F3E924111F78091BC3A9091BD3AD6
:10C2B0008F3E9241D9F680911D3E8111D7CF0895CE
:10C2C000FC01178289E60895CF93DF93EC018C81FE
:10C2D0009D81FC01EE0FFF1FE80FF91FEE0FFF1FFE
:10C2E000EE0FFF1FEE0FFF1FE15FF94EA591B49116
:10C2F0006C9170E080E090E00E940BDA69877A87A9
:10C300008B879C8782E08F8380E0DF91CF910895B7
:10C31000CF93DF93EC018C819D81FC01EE0FFF1F19
:10C32000E80FF91FEE0FFF1FEE0FFF1FEE0FFF1FAD
:10C33000E15FF94EA591B4916D917D918D919C91A4
:10C340000E940BDA69877A878B879C8782E08F83CC
:10C3500080E0DF91CF910895CF93DF93DC011496B5
:10C360008D919C911597FC01EE0FFF1FE80FF91FAF
:10C37000EE0FFF1FEE0FFF1FEE0FFF1FE15FF94EE5
:10C38000C591D491488159816A817B8119964D93D9
:10C390005D936D937C931C9783E017968C9380E05C
:10C3A000DF91CF910895CF93DF93DC0114968D91A7
:10C3B0009C911597FC01EE0FFF1FE80FF91FEE0F80
:10C3C000FF1FEE0FFF1FEE0FFF1FE15FF94EC5913C
:10C3D000D491488159816A817B8119964D935D93EF
:10C3E0006D937C931C97FC01EE0FFF1FE80FF91F64
:10C3F000EE0FFF1FEE0FFF1FEE0FFF1FE85FF94E5E
:10C400008591949118968C93189784E017968C9345
:10C4100080E0DF91CF91089588E608950F931F93F0
:10C42000CF93DF93EC018C819D81FC01EE0FFF1F08
:10C43000E80FF91FEE0FFF1FEE0FFF1FEE0FFF1F9C
:10C44000E15FF94E0591149169857A858B859C850C
:10C450000E94DFD9F801608382E08F8380E0DF9162
:10C46000CF911F910F910895CF93DF93EC016985D0
:10C470007A858B859C850E94DFD96230B0F48C81EF
:10C480009D81FC01EE0FFF1FE80FF91FEE0FFF1F4C
:10C49000EE0FFF1FEE0FFF1FE15FF94EA591B49164
:10C4A0006C9382E08F8380E001C08EE6DF91CF91B4
:10C4B0000895CF93DF93EC0169857A858B859C8500
:10C4C0000E94DFD96330B0F48C819D81FC01EE0FB6
:10C4D000FF1FE80FF91FEE0FFF1FEE0FFF1FEE0FFC
:10C4E000FF1FE15FF94EA591B4916C9382E08F83B9
:10C4F00080E001C08EE6DF91CF910895CF93DF9366
:10C50000EC0169857A858B859C850E94DFD9643032
:10C51000B0F48C819D81FC01EE0FFF1FE80FF91F25
:10C52000EE0FFF1FEE0FFF1FEE0FFF1FE15FF94E33
:10C53000A591B4916C9382E08F8380E001C08EE678
:10C54000DF91CF9108950F931F93CF93DF93EC0169
:10C550008C819D81FC01EE0FFF1FE80FF91FEE0F8C
:10C56000FF1FEE0FFF1FEE0FFF1FE15FF94E05915A
:10C57000149169857A858B859C850E94DFD9F801A5
:10C580006083718382E08F8380E0DF91CF911F9180
:10C590000F9108950F931F93CF93DF93EC018C813C
:10C5A0009D81FC01EE0FFF1FE80FF91FEE0FFF1F2B
:10C5B000EE0FFF1FEE0FFF1FE15FF94E0591149183
:10C5C00069857A858B859C850E94DFD9F801608317
:10C5D00071838283938382E08F8380E0DF91CF91A8
:10C5E0001F910F910895CF93DF93DC0114968D91E5
:10C5F0009C911597FC01EE0FFF1FE80FF91FEE0F3E
:10C60000FF1FEE0FFF1FEE0FFF1FE15FF94EC591F9
:10C61000D49119964D915D916D917C911C974883B1
:10C6200059836A837B8383E017968C9380E0DF9144
:10C63000CF910895CF93DF93DC0114968D919C9157
:10C640001597FC01EE0FFF1FE80FF91FEE0FFF1FFC
:10C65000EE0FFF1FEE0FFF1FE15FF94EC591D49162
:10C6600019964D915D916D917C911C9748835983EA
:10C670006A837B83FC01EE0FFF1FE80FF91FEE0FAB
:10C68000FF1FEE0FFF1FEE0FFF1FE85FF94E8591B2
:10C69000949118968C93189784E017968C9380E069
:10C6A000DF91CF9108951F93CF93DF93EC01809199
:10C6B000203B8823D1F01DE10A80DB81C02D20972B
:10C6C00011F480E013C08F818F3FD9F3811104C032
:10C6D000CE010E942D6006C0CE010E940360CE01F3
:10C6E0000E948060115041F7ECCF85E6DF91CF9139
:10C6F0001F910895CF93DF93EC01BC018FEF90E27F
:10C700000E94B7E5892B41F0BE0182E091E20E94D0
:10C71000B7E521E0892B09F420E0822FDF91CF914A
:10C7200008950F931F93CF93DF93CDB7DEB729976B
:10C73000CDBFDEBF8B0144E050E0BC01CE010196CD
:10C740000E94D7E546E050E0B801CE0101960E9474
:10C75000C7E50E94D668181619060CF03FC079810B
:10C76000AA81BB811C810D8121E036E140E050E0CF
:10C77000F9016491671327C03196E491E11103C078
:10C78000A11121C029C0EA131EC0F9013296E4911B
:10C79000E11103C0B11117C01FC0EB1314C0F901A0
:10C7A0003396E491E11103C011110DC015C0E113DE
:10C7B0000AC0F9013496E491E11103C0011103C0EC
:10C7C0000BC0E01749F04F5F5F4F285E3F4F48179F
:10C7D000590709F0CDCF02C0CA0102C08FEF9FEF09
:10C7E0002996CDBFDEBFDF91CF911F910F910895A4
:10C7F000CF93DF93FC012189222371F1EC01619633
:10C80000BE0186E091E20E94B7E5892B39F1BE01B5
:10C810008FEF90E20E94B7E5892B11F1BE0189E00C
:10C8200091E20E94B7E5892BD9F0BE018DEE90E22E
:10C830000E94B7E5892BB1F0BE018CE091E20E9425
:10C84000B7E5892B79F0BE018DEE91E20E94B7E544
:10C85000892B51F485E009C080E007C082E005C063
:10C8600083E003C084E001C081E0DF91CF910895AF
:10C87000FC018FEF8783148215821186128613863E
:10C8800014861086118A1586178A108EA081B181B0
:10C89000109711F416820DC017968C911797873058
:10C8A00029F416968C918F5F868303C016968C911F
:10C8B0008683CF010895EF92FF920F931F93CF933A
:10C8C000DF93EC010C811D810E94D66808171907BF
:10C8D0000CF06FC00C811D81CE010E9438640C8366
:10C8E0001D837E0181E1E80EF11CB801660F771F00
:10C8F000600F711F660F771F660F771F660F771F18
:10C900006F5F794EC7010E945FE58E01035F1F4F85
:10C910002C813D81B901660F771F620F731F660F6F
:10C92000771F660F771F660F771F63507A4EC80117
:10C930000E945FE58D85882311F18C819D81FC012A
:10C94000EE0FFF1FE80FF91FEE0FFF1FEE0FFF1F87
:10C95000EE0FFF1FE95FF94EE491E2FF02C01D8672
:10C9600010C0F80101900020E9F7BF01601B710BB6
:10C97000605F7F4F6C0F7D1FC7010E94C0E58C81F7
:10C980009D81FC01EE0FFF1FE80FF91FEE0FFF1F47
:10C99000EE0FFF1FEE0FFF1FE55FF94E259134915B
:10C9A000CE01F901DF91CF911F910F91FF90EF9090
:10C9B0001994DF91CF911F910F91FF90EF900895FF
:10C9C0008F929F92AF92BF92CF92DF92EF92FF929F
:10C9D0000F931F93CF93DF9300D01F92CDB7DEB795
:10C9E0006C015C0181E1A80EB11C87E0F601878330
:10C9F000ADEFEA2EA5E1FA2E00E010E01DC0B70170
:10CA0000CE0101960E945FE5BE016F5F7F4FC501B9
:10CA10000E94B7E5892B59F44601F9E18F0E911C6C
:10CA2000F601058F168FC4010E945B6464010F5FDD
:10CA30001F4FF8E1EF0EF11CC8010E94D968811167
:10CA4000DECF2496CDBFDEBFDF91CF911F910F9136
:10CA5000FF90EF90DF90CF90BF90AF909F908F901E
:10CA60000895CF93DF931092BA381092BB38ADE798
:10CA7000B5E3E6E9F5E391E08FEFA083B183799622
:10CA80005B96ED93FC935C975D961D921C925E976E
:10CA9000EF016397988322961882219788832A96BC
:10CAA0001882599628E3E63BF20739F710929F382F
:10CAB0001092A038109296351092973510929C35AE
:10CAC00087E080939D3582E790E08093A73590932F
:10CAD000A8358FEA95E3DF91CF9108950F931F93C7
:10CAE000CF93DF930E943165EC018FEE92E180934A
:10CAF000BE3A9093BF3A8093003B9093013B809362
:10CB00009435909395358093B6389093B738809349
:10CB1000B8389093B9388093BC3A9093BD3A81E08D
:10CB20000E9420531C821D82CE010E94DB84209132
:10CB3000083B3091093B40910A3B50910B3B698582
:10CB40007A858B859C850E946BD9882339F0CE012C
:10CB5000DF91CF911F910F910C94A6600E9460AC61
:10CB60001C821D8280E090E08E010F5E1F4F2FC05F
:10CB70006C817D819B01220F331FF901E60FF71FA6
:10CB8000EE0FFF1FEE0FFF1FEE0FFF1FE95FF94EC5
:10CB9000E491E0FF17C0620F731F660F771F660FE7
:10CBA000771F660F771F6F5F794E45E050E0C80131
:10CBB0000E947EE5CE010E94DB84CE010E940360CC
:10CBC0006C817D816F5F7F4F6C837D83CB010E9481
:10CBD000D9688111CDCFDF91CF911F910F910C9426
:10CBE00073ACEF92FF920F931F93CF93DF938C015F
:10CBF0002091BA383091BB38EB0109900020E9F759
:10CC00002197C61BD70BAE01420F531F4130524034
:10CC1000D8F4F901E454F74C7F01AE014F5F5F4F48
:10CC2000CF010E9498E54091BA385091BB384F5FD0
:10CC30005F4F4C0F5D1F4093BA385093BB38F801DB
:10CC4000E78AF08E80E001C08DE0DF91CF911F91E7
:10CC50000F91FF90EF900895CF93DF932EE1CFEAED
:10CC6000D5E33F813F3F59F00A80DB81C02D2097FB
:10CC700019F480E090E010C0215099F7FACFBC0180
:10CC800081E593E20E9491638C839D83019689F3F1
:10CC9000CE010E945B64CE01DF91CF910895EF92A7
:10CCA000FF920F931F93CF93DF938B012EE1CFEA77
:10CCB000D5E33F813F3F59F00A80DB81C02D2097AB
:10CCC00019F480E090E01DC0215099F7FACF7E0161
:10CCD00021E1E20EF11C45E050E0BC01C7010E94D9
:10CCE000D7E5B801CE010E94F1658111EACFB70105
:10CCF00081E593E20E9491638C839D8385E08F831D
:10CD0000CE01DF91CF911F910F91FF90EF90089589
:10CD10002091203B213021F42091CA3D213029F47B
:10CD2000BC018DEE90E20C944F6680E090E0089597
:10CD30009091203B913019F4642F0C9457830C94FC
:10CD400061C5CF93DF93EC018091BF29811103C0AE
:10CD50000E9401D602C00E94FACC682F70E080E0E9
:10CD600090E00E940BDA69877A878B879C8782E044
:10CD70008F8380E0DF91CF9108950F931F93CF931E
:10CD8000DF93CDB7DEB7C058D109CDBFDEBFFC0100
:10CD900061857285838594850E94DFD98FEF860F28
:10CDA000863030F080E491E20E9488668EE62AC0E8
:10CDB0006093BA2981E08093BB29E62FF0E0EE0F63
:10CDC000FF1FE853FA4E659174914FE450E08EECEA
:10CDD0009DE30E947EE59F938F938AE894E19F9361
:10CDE0008F938E010F5F1F4F1F930F930E9439E7A0
:10CDF000C8010E9488660F900F900F900F900F90BF
:10CE00000F9080E0C058DF4FCDBFDEBFDF91CF91E4
:10CE10001F910F9108950F931F93CF93DF93EC0110
:10CE200088EF92E30E94EB4E882329F009851A854A
:10CE30008B859C8511C023E333E34BEC51E469857A
:10CE40007A858B859C850E9410DC8B01AB01BC012F
:10CE500049875A876B877C872C813D81F901EE0FCA
:10CE6000FF1FE20FF31FEE0FFF1FEE0FFF1FEE0F6E
:10CE7000FF1FE15FF94EA591B491A801BC014D934C
:10CE80005D936D937C931397F901EE0FFF1FE20FF3
:10CE9000F31FEE0FFF1FEE0FFF1FEE0FFF1FE85FE8
:10CEA000F94E85919491888784E08F8380E0DF91AB
:10CEB000CF911F910F91089569E975E10C94F7C521
:10CEC00065E775E10C94F7C569E375E10C94F7C566
:10CED00060E075E10C94F7C563EB74E10C94F7C561
:10CEE0001F93CF93DF93EC0110E08881882301F139
:10CEF0000E94316545E050E0BE0180EC95E30E9460
:10CF0000D7E560EC75E381E593E20E94916380933D
:10CF1000B3359093B4358FEA95E30E945B6442E0A9
:10CF200063E080E00E9498661F5F26961D31E9F657
:10CF300084E0DF91CF911F910895CF93DF93CDB718
:10CF4000DEB7EC97CDBFDEBF8CE3E8E1F0E2DE01B7
:10CF5000119601900D928A95E1F7CE0101960E94FB
:10CF60007067EC96CDBFDEBFDF91CF910895CF9370
:10CF7000DF93CDB7DEB7AA97CDBFDEBF8AE2E4E587
:10CF8000F0E2DE01119601900D928A95E1F7CE0153
:10CF900001960E947067AA96CDBFDEBFDF91CF9148
:10CFA0000895CF93DF93CDB7DEB76E97CDBFDEBFC9
:10CFB0008EE1EEE7F0E2DE01119601900D928A9586
:10CFC000E1F7CE0101960E9470676E96CDBFDEBF7D
:10CFD000DF91CF910895CF93DF93EC0143E759E7B9
:10CFE00063E770E0498B5A8B6B8B7C8B0E94E0640B
:10CFF00042E063E080E00E949866CE010E94D16723
:10D00000CE010E94B76720E731E340E0298B3A8BDD
:10D010004B8BCE010E94E06442E063E080E00E941E
:10D020009866CE01DF91CF910C949D67CF92DF92ED
:10D03000EF92FF92CF93DF93EC01C984DA84EB8403
:10D04000FC8420E030E040E85FE3C701B6010E94C5
:10D050006EDB18161CF1C701B6010E94DFD9609380
:10D06000BC2989859A85AB85BC85BC01CD019F779C
:10D070002CEA35EC47E257E30E946EDB18163CF4CD
:10D0800060E470E080E00E9487CB80E008C060E848
:10D0900070E080E00E9487CB80E001C08EE6DF91E7
:10D0A000CF91FF90EF90DF90CF900895CF92DF92D5
:10D0B000EF92FF92CF93DF93EC01C984DA84EB8483
:10D0C000FC8420E030E040E050E4C701B6010E945B
:10D0D0006EDB18161CF1C701B6010E94DFD9609300
:10D0E000BE2989859A85AB85BC85BC01CD019F771A
:10D0F0002CEA35EC47E257E30E946EDB18163CF44D
:10D1000064E070E080E00E9487CB80E008C068E0C7
:10D1100070E080E00E9487CB80E001C08EE6DF9166
:10D12000CF91FF90EF90DF90CF900895CF92DF9254
:10D13000EF92FF92CF93DF93EC01C984DA84EB8402
:10D14000FC8420E030E040E85FE3C701B6010E94C4
:10D150006EDB18161CF1C701B6010E94DFD960937F
:10D16000BD2989859A85AB85BC85BC01CD019F779A
:10D170002CEA35EC47E257E30E946EDB18163CF4CC
:10D1800060E170E080E00E9487CB80E008C060E250
:10D1900070E080E00E9487CB80E001C08EE6DF91E6
:10D1A000CF91FF90EF90DF90CF9008958CE891E0C1
:10D1B000089521E08334914008F020E0822F089503
:10D1C0009C012F55314081E02932310508F080E083
:10D1D000089521E08036914008F020E0822F0895E4
:10D1E000CF92DF92EF92FF92CF93DF93EC01C9844D
:10D1F000DA84EB84FC84A7019601C701B6010E9482
:10D2000031DD81113CC0E894F7F82FEF3FEF4FE795
:10D210005FE7C701B6010E9431DD81110AC02FEF1F
:10D220003FEF4FE75FE7C701B6010E946BD91816C1
:10D2300034F18C819D81FC01EE0FFF1FE80FF91F77
:10D24000EE0FFF1FEE0FFF1FEE0FFF1FE95FF94EFE
:10D25000E491E3FF14C088EF92E30E94EB4E81114A
:10D260000EC025E832E441E25DE369857A858B856D
:10D270009C850E9410DC69877A878B879C87DF9169
:10D28000CF91FF90EF90DF90CF9008958091BB29D0
:10D29000882349F01092BB296091BA2980E00E944E
:10D2A0008FCB80E0089583E00895CF93DF93E091E2
:10D2B0003E3BF0913F3B04C0E0933E3BF0933F3B4D
:10D2C000EF018191982F9D7F9032B1F38930A1F3C6
:10D2D0004FE450E0BE0184E49DE30E94D7E56881FD
:10D2E000611105C08091203B81115DC028C0613271
:10D2F00021F4DF91CF910C947459653221F4DF91C0
:10D30000CF910C9478596E3721F4DF91CF910C9422
:10D310007C596B3741F481E08093203BCE01DF9153
:10D32000CF910C94547E70E080E791E20E94ACE5CE
:10D33000892B59F01092203BCE010E94B9C164E4C0
:10D340007DE3DF91CF910C94F9C28091203B811154
:10D3500009C0CE010E94697464E47DE3DF91CF913E
:10D360000C94F9C247EF50E0BE0184E49BE30E94B5
:10D37000D7E584E49BE39F938F9385E791E29F93A6
:10D380008F93DF93CF930E9410E70F900F900F9031
:10D390000F900F900F9080913E3B90913F3BDF911B
:10D3A000CF910C94547EDF91CF910895FF920F930B
:10D3B0001F93CF93DF931F921F92CDB7DEB7F82E46
:10D3C000E2E0FBE324E932E0DF01C9011D920197AD
:10D3D000E9F72FEE32E1208331832093943D30939F
:10D3E000953D09E21CE12CED33E40093083B1093DA
:10D3F000093B20930A3B30930B3B0CEE11E528E7E9
:10D400003FE300930C3B10930D3B20930E3B309376
:10D410000F3B00E010E020EA30E40093103B109353
:10D42000113B2093123B3093133B00E010E020E8C7
:10D430003FE30093143B1093153B2093163B30932E
:10D44000173B83E08093213B8F2D4A8369830E94A1
:10D450009FCB6981862F0E94AACB4A81842F0E948C
:10D46000B5CBF092B929F092B7290F900F90DF91C8
:10D47000CF911F910F91FF900895CF93DF931F924B
:10D480001F92CDB7DEB780E6F82E01E010E00E94D3
:10D49000BC7C8230E1F30E94C37C8230C1F30E94E5
:10D4A000CA4E863009F0D9C00E9483C98090273BBC
:10D4B0009090283BA090293BB0902A3B8616970677
:10D4C000A806B90620F70E9483C96C597F4F8F4F79
:10D4D0009F4F6093273B7093283B8093293B909309
:10D4E0002A3B0E94327CD3CF0E948CC0882329F033
:10D4F0008CEC0E940C53823051F20E94CB59823046
:10D5000031F20E94B6A1823011F20E942F61809305
:10D510001E3E81112EC08091023B9091033B8F3EB5
:10D52000924109F0AAC08091943D9091953D8F3E23
:10D53000924109F0A2C097C00E94B08580931E3E20
:10D54000811117C00E9419B780931E3E811111C02E
:10D550000E94347480931E3E81110BC00E94A1CAA8
:10D5600080931E3E811105C00E94EDB7823031F4D8
:10D570008ECF0E940C538230B9F789CF0E94F6AE4D
:10D58000823009F484CF0E9462B0823009F47FCFE8
:10D590000E941EB1823009F47ACF09831A8360E4B5
:10D5A0007BE3CE0101960E94C4CB80933E3B9093D7
:10D5B0003F3B8F3F2FEF920739F48DE00E94F552E9
:10D5C000823009F464CF04C0892B11F00E945569A0
:10D5D0000E941590823009F45ACF0E946B6F8230FE
:10D5E00009F455CF0E942A72823009F450CF0E946C
:10D5F0000F74823009F449CF0E949950823009F4A7
:10D6000044CF0E9465868430F0F53FCF8091213B66
:10D61000843038F484E08093213B0E9478590E9442
:10D6200065AC83E090E089839A8360E47BE3CE017C
:10D6300001960E94C4CB80933E3B90933F3B8F3F2B
:10D640002FEF920721F48DE00E94F5521ECF892B17
:10D6500009F41BCF0E94556918CF0E94CA4E823030
:10D6600009F44BCF41CF10921E3E0E94C7528093C7
:10D670001E3E882309F460CF7CCFF0921E3E80E6E8
:10D680000E940C5378CF8091CF289091D0280E948F
:10D6900075D4682F70E080E090E00E940DDA23E3FB
:10D6A00033E34BE451E40E946EDB87FFEECE0E9431
:10D6B0004669823009F0AACFE8CE8091B9298093DB
:10D6C000B72908958093B72908958093B8290895BC
:10D6D000CF93C82F80919D23882379F040E050E0BC
:10D6E000BA018C2F0E941D54EC2FFF27E7FDF09507
:10D6F000E353FD4C81E080830AC06C2F8DE197E5F8
:10D700000E941050AB01BC018C2F0E941D5440910F
:10D71000C4235091C5236091C6237091C7238C2FD9
:10D720000E941F5D81E39DE680939E2390939F233B
:10D7300082E0CF910895CF92DF92EF92FF920F9304
:10D740001F93CF93DF93CDB7DEB7E097CDBFDEBF9A
:10D7500098E17E01A9E1EA0EF11CF701A92F1192CF
:10D76000AA95E9F7FE0131966F0111929A95E9F7B2
:10D77000F60194E08902E00DF11D1124408F518FD4
:10D78000628F738F80E090E0A0E8BFE38083918395
:10D79000A283B3830093353310933633209337330A
:10D7A000309338330E94E8860E947C59B601C70145
:10D7B0000E94465780931E3E811101C082E0E09690
:10D7C000CDBFDEBFDF91CF911F910F91FF90EF9002
:10D7D000DF90CF9008950F931F93E0919723FF2739
:10D7E000E7FDF095EE55FF4C9381913099F400914F
:10D7F000A8231091A9232091AA233091AB23409113
:10D80000B0235091B1236091B2237091B3230E9451
:10D810009B6B1DC0E0919823FF27E7FDF095EE5527
:10D82000FF4C9381913099F40091A8231091A92382
:10D830002091AA233091AB234091B0235091B12382
:10D840006091B2237091B32370580E949B6B81E367
:10D850009CE680939E2390939F2382E01F910F91DB
:10D8600008950F931F93CF93C82F85E3C802F0014B
:10D870001124E256FE4C40815181628173818C2FCC
:10D880000E941F5D0091A8231091A9232091AA2333
:10D890003091AB234091A4235091A5236091A623FE
:10D8A0007091A7238C2F0E949B6B80EC9CE6809349
:10D8B0009E2390939F2382E0CF911F910F91089513
:10D8C0000F931F930091A8231091A9232091AA23BD
:10D8D0003091AB234091B4235091B5236091B6238E
:10D8E0007091B7230E949B6B88E69BE680939E23F2
:10D8F00090939F2382E01F910F9108950E94E886E4
:10D900008091BD230E9486538091BC230E942053A6
:10D910008091BE230E9424538091BF230E943257DE
:10D920008091C0239091C123A091C223B091C323C1
:10D930008093353390933633A0933733B093383395
:10D9400064E088EF92E30E94084F0E94275A1092E9
:10D95000C93280E00895CF93C82F4091C4235091DD
:10D96000C5236091C6237091C7230E941F5D8C2F31
:10D970000E947E6C80E00E94C4AE80EFCF9108953B
:10D980000F931F93E0919723FF27E7FDF095EE5546
:10D99000FF4C9381913039F08BEA9CE680939E2373
:10D9A00090939F2318C00091AC231091AD23209138
:10D9B000AE233091AF234091B0235091B1236091B9
:10D9C000B2237091B3230E949B6B80E69CE6809308
:10D9D0009E2390939F2382E01F910F910895FF92C1
:10D9E0000F931F93CF93DF93CDB7DEB7C058D10904
:10D9F000CDBFDEBFF82E0E9431658EEFF81205C054
:10DA000082E891E20E94886619C08F2D0E94BC5A5C
:10DA10001F928F932DE13BE33F932F938E010F5F76
:10DA20001F4F1F930F930E9439E7C8010E94886619
:10DA30000F900F900F900F900F900F9042E062E0C8
:10DA400080EF0E9498668F2D0E947E6C80EFC058F8
:10DA5000DF4FCDBFDEBFDF91CF911F910F91FF90C0
:10DA600008954F925F926F927F929F92AF92BF9272
:10DA7000CF92DF92EF92FF920F931F93CF93DF939A
:10DA80008F3F09F045C02CEA35EC47E257E360913F
:10DA900030347091313480913234909133340E941B
:10DAA0006EDB18160CF469C12CEA35EC47E257E33B
:10DAB000609128347091293480912A3490912B34CC
:10DAC0000E946EDB18160CF45DC12CEA35EC47E2BF
:10DAD00057E360912C3470912D3480912E349091C5
:10DAE0002F340E946EDB18160CF455C12CEA35EC6D
:10DAF00047E257E360913434709135348091363485
:10DB0000909137340E946EDB18160CF43FC171C13E
:10DB10008230A1F52CEA35EC47E257E360912834D6
:10DB20007091293480912A3490912B340E946EDBBD
:10DB300018160CF427C12CEA35EC47E257E3609144
:10DB40002C3470912D3480912E3490912F340E947A
:10DB50006EDB18160CF41FC12CEA35EC47E257E3D4
:10DB600060913434709135348091363490913734EB
:10DB70000E946EDB18160CF409C131C18823D9F25A
:10DB8000813051F32CC17E018DEEE80EF11CF701BE
:10DB900080819181A281B381BC01CD019F772CEA64
:10DBA00035EC47E257E30E946BD987FD46C06E0112
:10DBB000F1EFCF0ED11CF60140805180628073805E
:10DBC00020E030E0A901C301B2010E946BD987FDBA
:10DBD00034C0FE01EF52FF4F2081318142815381D9
:10DBE000349760817181828193810E94C2D79B01A9
:10DBF000AC015F77C301B2010E94C3D72B013C0186
:10DC00009F772CEA35EC47E257E30E946BD987FDFA
:10DC100014C0AB2CAA0C8A2D0E9486C08093952339
:10DC2000992493949A0C892D0E9486C08093962300
:10DC300020919523822780FD02C08B2DDBC0B092FE
:10DC40009423F80180819181A281B381BF77809371
:10DC5000A8239093A923A093AA23B093AB23F70101
:10DC600040815181628173817F774093AC235093CF
:10DC7000AD236093AE237093AF2320FF2DC0A092FD
:10DC800097239092982377FA709477F87094409243
:10DC9000A4235092A5236092A6237092A723F60195
:10DCA00080819181A281B3818093B0239093B1232D
:10DCB000A093B223B093B323CB50DF4F88819981D7
:10DCC000AA81BB818093B4239093B523A093B623FC
:10DCD000B093B7238A2D2AC090929723A0929823BD
:10DCE0004092A4235092A5236092A6237092A7236A
:10DCF000F60180819181A281B381B0588093B023D5
:10DD00009093B123A093B223B093B323CB50DF4FB2
:10DD100088819981AA81BB81B0588093B423909364
:10DD2000B523A093B623B093B723892D0E9486C054
:10DD30008D7F813039F081E39DE680939E2390931F
:10DD40009F2369C0809198230E9486C0811103C0DF
:10DD50008FEF809398238B2D0E94145D6093C423D2
:10DD60007093C5238093C6239093C7238BEE9BE6C5
:10DD700080939E2390939F234EC082E090E032E0F8
:10DD8000B32E0DC080E090E0B12C09C083E090E09C
:10DD900023E0B22E04C081E090E0BB24B394FC01E8
:10DDA000E353FD4C108225E3289FE001299FD00D0D
:10DDB0001124CB53DF4C8E0107511F4FF801808196
:10DDC0009181A281B381BC01CD019F772CEA35EC12
:10DDD00047E257E30E946BD987FFD5CE2ECF81E073
:10DDE0008093CC328EE79CE680939E2390939F2372
:10DDF00012C08EEFDF91CF911F910F91FF90EF90A6
:10DE0000DF90CF90BF90AF909F907F906F905F908A
:10DE10004F900C94EF6C82E0DF91CF911F910F91A6
:10DE2000FF90EF90DF90CF90BF90AF909F907F904A
:10DE30006F905F904F900895CF93DF93C6EFD2E33A
:10DE4000888199810E94EB4E8093BC2388819981BF
:10DE50000E94E64E8093BD23888199810E94F54EF1
:10DE60008093BE23888199810E94FA4E8093BF23BC
:10DE7000888199810E94014F6093C0237093C123D0
:10DE80008093C2239093C32381E00E94205381E0BA
:10DE90000E94245380E00E94865381E00E94325702
:10DEA00081E080939D238FEF8093942381E39DE60F
:10DEB00080939E2390939F2383E08093C932109296
:10DEC000CC3280E0DF91CF9108950E941C6F1092B8
:10DED0009D2380E008958091C932833059F40E94D7
:10DEE000FF4E813049F0E0919E23F0919F23809175
:10DEF0009423199483E0089582E0089586E89FE6CC
:10DF00008093D9239093DA2382E008952F923F9251
:10DF10004F925F926F927F928F929F92AF92BF9239
:10DF2000CF92DF92EF92FF920F931F93CF93DF93E5
:10DF3000CDB7DEB7CA54D109CDBFDEBF98E19E018F
:10DF4000275E3F4F29AB3AABD901E92F1D92EA95E5
:10DF5000E9F7285131091901D9011D929A95E9F77C
:10DF600024E08202F00111242B96EEAFFFAF2B9735
:10DF7000E20DF31D80E090E0A0E8BFE38083918391
:10DF8000A283B383C090D123D090D223E090D32337
:10DF9000F090D4234090CD235090CE236090CF2397
:10DFA0007090D0238090C9239090CA23A090CB2357
:10DFB000B090CC23A5019401C301B2010E946BD99A
:10DFC00018165CF080E090E0A0E8BFE329968CAFE3
:10DFD0009DAFAEAFBFAF29970AC080E090E0A0E848
:10DFE000BFEB29968CAF9DAFAEAFBFAF2997A30112
:10DFF0009201C501B4010E94C2D70E94DAD99B01E7
:10E0000077FF04C022273327261B370BB901882747
:10E0100077FD8095982F0E940DDA25966CAF7DAF25
:10E020008EAF9FAF2597C0923533D0923633E092B2
:10E030003733F09238330E94E8860E947C5920E002
:10E0400030E040E050E425966CAD7DAD8EAD9FADE7
:10E0500025970E946EDB18166CF08091D523909165
:10E06000D623A091D723B091D8238BAF9CAFADAF6F
:10E07000BEAFDBC02AE037ED43E25CE325966CAD32
:10E080007DAD8EAD9FAD25970E946EDB18162CF7E7
:10E0900009E110E08AE0882E87ED982E83E2A82E11
:10E0A0008CE3B82E412C512C32012B96AEADBFAD76
:10E0B0002B97A20DB31D58962196AEAFBFAF2197F7
:10E0C0004BAA5CAA6DAA7EAA8FAA98AEA9AEBAAED8
:10E0D00029962CAD3DAD4EAD5FAD29976FA978ADBA
:10E0E00089AD9AAD0E9410DC9B01AC016091CD23FB
:10E0F0007091CE238091CF239091D0230E94C3D7DB
:10E100002196EEADFFAD2197608371838283938367
:10E11000C0923533D0923633E0923733F0923833B1
:10E12000B101CE0149960E94465780931E3E81114F
:10E13000AAC020E030E040E85FE36BA97CA98DA98C
:10E140009EA90E94C3D76BAB7CAB8DAB9EAB20E08E
:10E1500030E048EC51E40E9472D99B01AC0160E0D0
:10E1600070E080E291E40E9473DC2B013C0180911D
:10E17000D5239091D623A091D723B091D8238BAFEC
:10E180009CAFADAFBEAFC090D123D090D223E09072
:10E19000D323F090D423A7019601BC01CD010E94A6
:10E1A000C2D74B015C0120E030E040E251E4C30102
:10E1B000B2010E9472D99B01AC01C501B4010E9459
:10E1C00010DC9B01AC01C701B6010E94C3D76B01F3
:10E1D0007C012BA93CA94DA95EA9CA01B9010E94E5
:10E1E000C3D720E030E048EC51E40E9472D99B0193
:10E1F000AC016FA978AD89AD9AAD0E94C3D76FAB62
:10E2000078AF89AF9AAF9B01AC0125966CAD7DAD1F
:10E210008EAD9FAD25970E946EDB181634F4015029
:10E2200011090115110509F053CF8BAD9CADADADB2
:10E23000BEAD8093353390933633A0933733B0938C
:10E2400038332B96EEADFFAD2B97E20DF31D809189
:10E25000C9239091CA23A091CB23B091CC23808F66
:10E26000918FA28FB38FB101CE0149960E9446577C
:10E2700080931E3E811107C08AE591E78093D923E0
:10E280009093DA2382E0C65BDF4FCDBFDEBFDF9124
:10E29000CF911F910F91FF90EF90DF90CF90BF90A3
:10E2A000AF909F908F907F906F905F904F903F9036
:10E2B0002F900895CF93DF931F92CDB7DEB7898358
:10E2C0000E94E8864091E3235091E4236091E52386
:10E2D0007091E62389810E941F5D8091E0230E9456
:10E2E00086538091DF230E9420538091E1230E9476
:10E2F00024538091E2230E9432578091DB23909136
:10E30000DC23A091DD23B091DE23809335339093FD
:10E310003633A0933733B093383364E088EF92E319
:10E320000E94084F0E94275A1092C9328EEA91E249
:10E330000E94E3E680E00F90DF91CF9108950F9364
:10E340001F93CF93C82F06EF12E3F80180819181CC
:10E350000E94EB4E8093DF23F801808191810E941F
:10E36000E64E8093E023F801808191810E94F54E72
:10E370008093E123F801808191810E94FA4E80937D
:10E38000E223F801808191810E94014F6093DB2399
:10E390007093DC238093DD239093DE238C2F0E94E7
:10E3A000145D6093E3237093E4238093E5239093BB
:10E3B000E62381E00E94205380E00E94245380E005
:10E3C0000E94865381E00E94325740E050E060E2B4
:10E3D00071E44093D1235093D2236093D32370935D
:10E3E000D42385E3C89FF0011124E257FE4C4081FD
:10E3F0005181628173814093D5235093D6236093DA
:10E40000D7237093D8236C2F8DE197E50E94FD4FA1
:10E410006093CD237093CE238093CF239093D0230A
:10E420000E94EC5D6093C9237093CA238093CB2331
:10E430009093CC23C093C8238EE79FE68093D92383
:10E440009093DA2384E08093C93280E0CF911F91CA
:10E450000F9108958091C932843059F40E94FF4E83
:10E46000813049F0E091D923F091DA238091C823DB
:10E47000199483E0089582E00895E091E923F0E0A3
:10E48000EE55FF4C8381882341F088E592E7809325
:10E49000E7239093E82382E0089566E374E28EE137
:10E4A00094E20E94465780931E3E882371F308959C
:10E4B0001F93CF93DF93E091E923F0E0EE55FF4CFB
:10E4C00081E09381913009F080E08093D332C4EDF4
:10E4D000D2E310E0812F0E94D69AAB01BC01812FBC
:10E4E0000E941D54612F8091F6329091F7320E9464
:10E4F000FD4F69937993899399931F5F163051F774
:10E5000088EB91E20E94547E84EC92E78093E723AB
:10E510009093E82382E0DF91CF911F9108951F939C
:10E52000CF93DF930E94E8868091EA238093A23004
:10E53000E091E923F0E08091EB23EE55FF4C8387D7
:10E540000E94A3C0CEEED3E210E0499159916991A7
:10E550007991812F0E941F5D1F5F1630B1F7809166
:10E56000ED230E9486538091EC230E94245364E0A3
:10E5700088EF92E30E94084F0E94275A1092C932F6
:10E58000DF91CF911F9108950E948F7280E00895CE
:10E590000F931F93CF93DF93CDB7DEB7C058D10948
:10E5A000CDBFDEBF182F0E9431651E3F29F485ECD8
:10E5B00091E20E94886619C0812F0E94BC5A1F9266
:10E5C0008F938BE49BE39F938F938E010F5F1F4F7D
:10E5D0001F930F930E9439E7C8010E9488660F902D
:10E5E0000F900F900F900F900F9042E062E08AEF33
:10E5F0000E9498660E948F728AEFC058DF4FCDBF8D
:10E60000DEBFDF91CF911F910F910895FF920F937D
:10E610001F93CF93DF931092D33282E08093C9325D
:10E620000EEE13E2CEE9D1E3F12C8F2D0E94145DA2
:10E63000F80161937193819391938F01488159817E
:10E640006A817B818F2D0E941F5D6F2D8091F63234
:10E650009091F7320E94FD4FF801648B758B868B89
:10E66000978BF394E596F6E0FF12DFCF6EE174E24C
:10E6700086E094E20E9486C62AE43CE042E85EE33B
:10E680000E946BD987FF03C08EEF0E94C872C2E15F
:10E69000D4E213E069917991899199912C893D890E
:10E6A0004E895F890E94C2D79F772CEA35EC47E2FA
:10E6B00057E30E946EDB18161CF4812F0E94C8726B
:10E6C0001F5F163039F784E08093E9238091B130E1
:10E6D0008093EB2381E08093B1308091A2308093CE
:10E6E000EA231092A2300E94A3C08091F63290914A
:10E6F000F7320E94E64E8093ED238091F63290919E
:10E70000F7320E94F54E8093EC2380E00E94245360
:10E7100080E00E94865380E00E94FFB28DE392E782
:10E720008093E7239093E82382E0DF91CF911F91BC
:10E730000F91FF9008950F931F93CF93DF938C0158
:10E74000EB0180914133882399F08091353390918A
:10E750003633A0913733B0913833BC01CD019F7768
:10E760002CEA35EC47E257E30E946BD987FD4FC096
:10E7700088819981AA81BB81BC01CD019F772CEA58
:10E7800035EC47E257E30E946EDB1816F4F48C81F7
:10E790009D81AE81BF81BC01CD019F772CEA35EC14
:10E7A00047E257E30E946EDB18167CF48885998552
:10E7B000AA85BB85BC01CD019F772CEA35EC47E2E9
:10E7C00057E30E946EDB181624F188E1F801AEE1F0
:10E7D000B4E201900D928A95E1F788E1FE01A6E38B
:10E7E000B4E201900D928A95E1F788E1E4EDF2E35D
:10E7F000DF011D928A95E9F782E08093D33286E0AB
:10E8000093E78093E7239093E82380E003C08EE8AA
:10E8100001C086E8DF91CF911F910F9108958091FB
:10E82000C932823021F08091D332823049F40E9483
:10E83000FF4E813039F0E091E723F091E8231994FD
:10E8400083E0089582E00895E6E9FDE380E2DF01D8
:10E850001D928A95E9F78FEE92E18093B43D9093F3
:10E86000B53D8083918308958091B43D9091B53DED
:10E870008F3E924111F08CE508958091963D9091E4
:10E88000973D8F3E9241B9F780E00895CF93DF9393
:10E89000C82FCB01BA010E94BFDC27E0C29FE00174
:10E8A0001124CA56D24C0E94DAD96D837E838F839D
:10E8B0009887DF91CF91089597E0899FF001112407
:10E8C000EA56F24C65817681878190850E940DDA47
:10E8D00008952F923F924F925F926F927F928F9204
:10E8E0009F92AF92BF92CF92DF92EF92FF920F93DF
:10E8F0001F93CF93DF93CDB7DEB72797CDBFDEBF92
:10E900008C011B828091C832823009F40CC7D80177
:10E91000BC90B11035C780E06E01B3E0CB0ED11CC6
:10E920003DC0F6018081811108C0B72CD7011C922F
:10E930006E01B3E0CB0ED11C20C7883239F4B72C5E
:10E94000F7011082FFEFCF1ADF0A17C78B33B9F335
:10E95000A82EB12CC5010E9433E5892B39F4B501ED
:10E960008FEE91E20E94ACE5892B51F047018FEFC9
:10E97000881A980AC5010E9457E5D7018C93740143
:10E98000BFEFCB1ADB0AF70180818111CACFB72C08
:10E99000D8018C916E01B3E0CB0ED11CF8011CC0E4
:10E9A0008E32E1F090E0C0970A9790F08181803339
:10E9B00091F4828190E0C0970A9760F4DF0111968C
:10E9C00011968C9111978D938111FACF808104C09B
:10E9D000818101C080E331968111E2CFF601A080F0
:10E9E000A11007C036C0D6011196AC90BFEFCB1A6C
:10E9F000DB0A76018A2C912CC4010E9447E5892B01
:10EA000091F7C4010E944FE58D369105A1F4F601FE
:10EA1000818190E00E944FE58337910561F4D60132
:10EA200012968C9190E00E944FE58736910519F47B
:10EA3000F601339602C0FE013396AA2061F08A2DBA
:10EA4000D701893209F41C9211968C918111F9CF6A
:10EA500002C0FE013396BFE2BB1609F466C6808190
:10EA6000882319F0CF010E946F5980E1E6EBFDE3A6
:10EA7000DF011D928A95E9F78BE5E1E2F4E3DF011E
:10EA8000982F1D929A95E9F7E6ECF3E3DF011D92CA
:10EA90008A95E9F788EF92E30E94E34E8093C733AB
:10EAA000812C912C80E8A82E8FE3B82E5524539406
:10EAB00092E0492E24E0322E23C4C701B6010E9401
:10EAC000DFD9862F90E08F35910508F032C6FC0122
:10EAD000EC50FF4F0C94B6E11092C73350922234A1
:10EAE0008091B73D8F5F8093B73D0AC45092C73382
:10EAF000509222348091B73D8F5F8093B73D00C420
:10EB00004092C733509222348091B73D8F5F8093FB
:10EB1000B73DF6C383E08093C7335092223480918F
:10EB2000B73D8F5F8093B73DEBC38DE08093C633D5
:10EB300050922134E5C388E0B2C01092F63350926F
:10EB400051348091B83D8F5F8093B83DD9C35092C6
:10EB5000F633509251348091B83D8F5F8093B83D29
:10EB6000CFC34092F633509251348091B83D8F5FBD
:10EB70008093B83DC5C31092F733509252348091C0
:10EB8000BB3D8F5F8093BB3DBBC35092F733509228
:10EB900052348091BB3D8F5F8093BB3DB1C3C701B1
:10EBA000B6010E942ADD6C837D838E839F8320E0E3
:10EBB00030E040E251E4C701B6010E9410DC6B0175
:10EBC0007C0120E030E040E251E46C817D818E8167
:10EBD0009F810E9410DC9B01AC01C701B6010E941D
:10EBE000C2D70E94DFD9623001F128F4662341F0D8
:10EBF000613089F09EC56330E9F0643001F199C558
:10EC0000B5E0B093C633509221348091B63D8F5F0A
:10EC10008093B63D75C33092C633609321348091A2
:10EC2000B63D8F5F8093B63D6BC35092C633509212
:10EC3000213466C34092C6335092213461C383E0CD
:10EC40008093C633509221345BC3C701B6010E9442
:10EC50002ADD6C837D838E839F8320E030E040E259
:10EC600051E4C701B6010E9410DC6B017C0120E079
:10EC700030E040E251E46C817D818E819F810E9471
:10EC800010DC9B01AC01C701B6010E94C2D70E94F3
:10EC9000DFD9662319F0613061F04BC587E08093BE
:10ECA000C633509221348091B63D8F5F8093B63D3C
:10ECB00027C3E6E0E093C633609321348091B63DEC
:10ECC0008F5F8093B63D1CC3C701B6010E942ADD49
:10ECD0006C837D838E839F8320E030E040E251E4AB
:10ECE000C701B6010E9410DC6B017C0120E030E01E
:10ECF00040E251E46C817D818E819F810E9410DC15
:10ED00009B01AC01C701B6010E94C2D70E94DFD9A6
:10ED1000623009F00EC58EE08093C63350922134E4
:10ED2000EFC25092F93350925434EAC25092F83301
:10ED3000509253348091BF3D8F5F8093BF3DE0C2BE
:10ED40004092F833509253348091BF3D8F5F80934F
:10ED5000BF3DD6C283E016C03092F8335092533490
:10ED60008091BF3D8F5F8093BF3DCAC2F5E0F093B5
:10ED7000F833509253348091BF3D8F5F8093BF3DF5
:10ED8000BFC286E08093F833509253348091BF3DE8
:10ED90008F5F8093BF3DB4C2C701B6010E942ADDD8
:10EDA0006C837D838E839F8320E030E040E251E4DA
:10EDB000C701B6010E9410DC6B017C0120E030E04D
:10EDC00040E251E46C817D818E819F810E9410DC44
:10EDD0009B01AC01C701B6010E94C2D70E94DFD9D6
:10EDE000662319F0613059F0A4C41092FB3350929D
:10EDF00056348091C03D8F5F8093C03D81C2609347
:10EE0000FB33609356348091C03D8F5F8093C03D4B
:10EE100077C24092FB33509256348091C03D8F5F51
:10EE20008093C03D6DC23092C7335092223480919E
:10EE3000B73D8F5F8093B73D63C2C701B6010E94A3
:10EE40002ADD6C837D838E839F8320E030E040E267
:10EE500051E4C701B6010E9410DC6B017C0120E087
:10EE600030E040E251E46C817D818E819F810E947F
:10EE700010DC9B01AC01C701B6010E94C2D70E9401
:10EE8000DFD9662319F0613059F053C41092FC3376
:10EE9000509257348091B93D8F5F8093B93D30C215
:10EEA0001092FD33609358348091B93D8F5F809309
:10EEB000B93D26C2C701B6010E942ADD6C837D835D
:10EEC0008E839F8320E030E040E251E4C701B60129
:10EED0000E9410DC6B017C0120E030E040E251E454
:10EEE0006C817D818E819F810E9410DC9B01AC0131
:10EEF000C701B6010E94C2D70E94DFD9662319F06C
:10EF0000613059F016C45092FC33509257348091BE
:10EF1000B93D8F5F8093B93DF3C16093FD3360933A
:10EF200058348091B93D8F5F8093B93DE9C1C701E5
:10EF3000B6010E942ADD6C837D838E839F8320E04F
:10EF400030E040E251E4C701B6010E9410DC6B01E1
:10EF50007C0120E030E040E251E46C817D818E81D3
:10EF60009F810E9410DC9B01AC01C701B6010E9489
:10EF7000C2D70E94DFD9613089F028F06230A1F059
:10EF80006330C1F0D6C399E09093C63350922134D8
:10EF90008091B63D8F5F8093B63DB2C1AAE0A09349
:10EFA000C63360932134ACC1BBE0B093C6335092FA
:10EFB0002134A6C1ECE0E093C63350922134A0C1C5
:10EFC0001092F13350924C348091BA3D8F5F809310
:10EFD000BA3D96C15092F13350924C348091BA3D73
:10EFE0008F5F8093BA3D8CC1C701B6010E94DFD903
:10EFF000862F90E08D33910508F099C3FC01ED5AFE
:10F00000FE4F0C94B6E11092C83350922334809195
:10F01000C13D8F5F8093C13D73C15092C833509200
:10F0200023348091C13D8F5F8093C13D69C150926F
:10F03000033450925E348091C33D8F5F8093C33D13
:10F040005FC14092033450925E348091C33D8F5F24
:10F050008093C33D55C11092033450925E34809129
:10F06000C33D8F5F8093C33D4BC15092003450929B
:10F070005B3446C15092013450925C348091C43D5F
:10F080008F5F8093C43D3CC15092023450925D34F6
:10F090008091C43D8F5F8093C43D32C11092023491
:10F0A00050925D348091C43D8F5F8093C43D28C1F0
:10F0B0005092F43350924F348091C53D8F5F8093CE
:10F0C000C53D1EC11092F43350924F348091C53D1E
:10F0D0008F5F8093C53D14C15092F23350924D34EE
:10F0E0008091C53D8F5F8093C53D0AC150920C341D
:10F0F000509267348091C53D8F5F8093C53D00C1BC
:10F10000C701B6010E942ADD0E94DFD96093FF3358
:10F1100050925A34F5C0C092E533D092E633E09273
:10F12000E733F092E8338092403490924134A092D9
:10F130004234B0924334E4C0C0920D34D0920E34C5
:10F14000E0920F34F09210348092683490926934D7
:10F15000A0926A34B0926B34D3C0C0920434D0927F
:10F160000534E0920634F092073480925F34909236
:10F170006034A0926134B0926234C2C0C092CD3388
:10F18000D092CE33E092CF33F092D03380922834B5
:10F1900090922934A0922A34B0922B34B1C0C092FC
:10F1A000D133D092D233E092D333F092D4338092E1
:10F1B0002C3490922D34A0922E34B0922F34A0C0D3
:10F1C000C092D533D092D633E092D733F092D83371
:10F1D0008092303490923134A0923234B0923334F1
:10F1E0008FC0C092D933D092DA33E092DB33F09201
:10F1F000DC338092343490923534A0923634B0921D
:10F2000037347EC0C092DD33D092DE33E092DF33FC
:10F21000F092E0338092383490923934A0923A34AC
:10F22000B0923B346DC0C092E133D092E233E092B1
:10F23000E333F092E43380923C3490923D34A092D8
:10F240003E34B0923F345CC0C0921534D092163434
:10F25000E0921734F09218348092703490927134A6
:10F26000A0927234B09273344BC0C0921934D092D1
:10F270001A34E0921B34F0921C34809274349092D1
:10F280007534A0927634B09277343AC0C0921D346F
:10F29000D0921E34E0921F34F09220348092783461
:10F2A00090927934A0927A34B0927B3429C0C09283
:10F2B0001134D0921234E0921334F09214348092CC
:10F2C0006C3490926D34A0926E34B0926F3418C04A
:10F2D000C701B6010E94DFD96093C9337093CA3366
:10F2E0008093CB339093CC3381E090E0A0E0B0E00A
:10F2F0008093243490932534A0932634B0932734FC
:10F30000D8012C90222009F422C2822D90E00E9484
:10F310003EE5892B09F42DC23801BFEF6B1A7B0A39
:10F32000F8018181803349F48281883531F40E5FA0
:10F330001F4FC12CD12C7601FEC1BE016F5F7F4FE4
:10F34000C3010E94D6E16B017C0109811A8160161C
:10F35000710609F0F0C10FC28091F1330E9432575B
:10F36000182F01C010E060914034709141348091B9
:10F370004234909143340E94DFD9662359F0609162
:10F38000E5337091E6338091E7339091E8330E9442
:10F390000157182F60914434709145348091463460
:10F3A000909147340E94DFD9662371F06091E93370
:10F3B0007091EA338091EB339091EC330E94DFD966
:10F3C000862F0E94DD58182F60914834709149347F
:10F3D00080914A3490914B340E94DFD9662371F0BA
:10F3E0006091ED337091EE338091EF339091F03373
:10F3F0000E94DFD9862F0E941C59182F60915F341C
:10F400007091603480916134909162340E94DFD9B0
:10F41000662359F06091043470910534809106346C
:10F42000909107340E9433B3182F60916334709128
:10F43000643480916534909166340E94DFD96623EC
:10F4400071F0609108347091093480910A34909180
:10F450000B340E94DFD9862F0E945B59182F8091B0
:10F460005A34882329F08091FF330E949A57182F2D
:10F4700080915B34882329F0809100340E94CE571C
:10F48000182F80915E34882329F0809103340E94E4
:10F49000FFB2182F80915C34882329F080910134C9
:10F4A0000E940358182F80915D34882329F08091A1
:10F4B00002340E943758182F80914D34882329F048
:10F4C0008091F2330E94B258182F80914E348823D5
:10F4D00029F08091F3330E94F158182F80916734FE
:10F4E000882329F080910C340E943059182F809184
:10F4F0004F34882329F08091F4330E94AA58182FA2
:10F500008091C6338D3029F0809151348823A9F041
:10F510000FC060910D3470910E3480910F34909132
:10F5200010340E943A5780931E3E882369F32DC100
:10F530008091F6330E941C53182F809152348823F7
:10F5400029F08091F7330E942053182F8091533473
:10F55000882329F08091F8330E948653182F8091D8
:10F560005634882329F08091FB330E943657182F98
:10F5700080915734882329F08091FC330E942453D2
:10F58000182F4091C63350E04F30510508F0B4C0F9
:10F59000FA01E057FE4F0C94B6E10E948356182FF3
:10F5A000ABC068E274E38DEC93E30E948E56182F93
:10F5B000A3C00E94C256182F9FC068E274E38DEC6E
:10F5C00093E30E94CD56182F97C00E941C6F182FEE
:10F5D00093C068E274E38DEC93E30E944D54182FBE
:10F5E0008BC00E94656F182F87C068E274E38DECB2
:10F5F00093E30E949B73182F7FC060910D3470912C
:10F600000E3480910F34909110340E94DFD9862FF0
:10F6100048E254E36DEC73E30E942853182F6CC04A
:10F6200068E274E38DEC93E30E94CA54182F64C01F
:10F630000E947D55182F60C00E94E455182F5CC0B1
:10F640000E941B56182F58C06091F93388EF92E33F
:10F650000E947E4F8091C733843038F48230D8F4D2
:10F66000882349F0813079F047C0843009F044C0E4
:10F670008093FC3241C068E274E38DEC93E30E9416
:10F680005356182F39C068E274E38DEC93E30E945F
:10F690004657182F31C0A0901D34B0901E34C09032
:10F6A0001F34D0902034E0901934F0901A34009137
:10F6B0001B3410911C342091153430911634409134
:10F6C0001734509118348F93809114348F93809114
:10F6D00013348F93809112348F93809111348F93D0
:10F6E00068E274E38DEC93E30E947888182F0F9002
:10F6F0000F900F900F900F9060E088EF92E30E94C0
:10F700007E4F80912334813061F48091C833811120
:10F7100004C00E945A5A812F38C00E948B5A812FF0
:10F7200034C0812F32C08BEC30C083E02EC084E81F
:10F730002CC083E82AC0822D90E0FC01E154F1093D
:10F74000EA31F105B0F7E156FE4F0C94B6E11092A4
:10F750001E3E6091C9337091CA338091CB33909132
:10F76000CC330E94184F80914C34882309F4FACD91
:10F77000F3CD85E60AC086E608C0D8018C910EC993
:10F7800068018B2D78017B2CD8C82796CDBFDEBFB2
:10F79000DF91CF911F910F91FF90EF90DF90CF906D
:10F7A000BF90AF909F908F907F906F905F904F90A1
:10F7B0003F902F900895CF93DF93EC0164E47DE3B5
:10F7C0000E94F16580931E3E811102C095E09F83E7
:10F7D000DF91CF910895FC018789908D0C94697415
:10F7E00083FF06C0E0919A30F0919B3090E29583C0
:10F7F00082FF06C0E0919C30F0919D3090E29583AD
:10F8000081FF06C0E0919E30F0919F3090E2958399
:10F8100080FF06C0E091A030F091A13080E28583A6
:10F82000089583FF06C0E0919A30F0919B3090E2FA
:10F83000968382FF06C0E0919C30F0919D3090E26B
:10F84000968381FF06C0E0919E30F0919F3090E258
:10F85000968380FF06C0E091A030F091A13080E255
:10F86000868308958091223B811107C084E00E9425
:10F87000F07B81E08093223B089584E00E94117C1C
:10F880001092223B0895CF92DF92EF92FF920F9356
:10F890001F93CF93DF93C12C26E0D22EC0928A30E3
:10F8A000D0928B3030EAE32E36E0F32EE0928C30AB
:10F8B000F0928D3000E816E000938E3010938F3078
:10F8C000C0E6D6E0C0939030D0939130C092923091
:10F8D000D0929330C0939430D0939530009396306B
:10F8E00010939730E0929830F09299302DEC3CECE8
:10F8F0004CED50E40E946EDBC0929A30D0929B3067
:10F90000E0929C30F0929D3018164CF4C0939E30DB
:10F91000D0939F300093A0301093A13008C0009383
:10F920009E3010939F30C093A030D093A130DF91D0
:10F93000CF911F910F91FF90EF90DF90CF9008959E
:10F940000E9415D760E070E080E091E40E94437C63
:10F950000C9434D781E080932B3B089520E093E012
:10F9600088ED08B618BE84BF909380002091820075
:10F9700021FDFCCF08BEFFCF80912B3B81110E945F
:10F98000AE7C83E0089580912C3B882341F0F8946D
:10F9900061E089E790E00E9417D782E0089583E054
:10F9A0000895CF93DF93CDB7DEB7AD97CDBFDEBF60
:10F9B00021E2E2EFF1E2DE01119601900D922A952B
:10F9C000E1F722E02093CA01DE019296E8E0F0E040
:10F9D00024912D933196EE30F105D1F72DE228A731
:10F9E000E0E1F0E0E491EF7121E030E02C0F3D1F09
:10F9F0002E0F311DF901208129A7E2E1F0E0E49109
:10FA0000EF719E012E0F311DF90121812AA7E4E13A
:10FA1000F0E0E491EF719E012E0F311DF90121817B
:10FA20002BA71CA61092CA0125E0FC012783BE016A
:10FA30006E5D7F4F0E94F16580931E3EAD96CDBFF7
:10FA4000DEBFDF91CF91089581E080932C3B80E071
:10FA50000895CF93DF93EC0120E030E040E051E4E3
:10FA600069857A858B859C850E946EDB18166CF003
:10FA7000CE010E941A6369857A858B859C850E94D8
:10FA8000437C0E94A3C080E001C08DE6DF91CF914E
:10FA900008956DEE7BE30C9436C66FEC7BE30C941B
:10FAA00036C660EB7BE30C9436C662E97BE30C94CC
:10FAB00036C66EE77BE30C94E1C5CF93DF9383E317
:10FAC00097E49F938F93C6EDDAE589818F938881C0
:10FAD0008F930E9445E68DEF94E49F938F938981E5
:10FAE0008F9388818F930E9445E685E794E49F93E6
:10FAF0008F9389818F9388818F930E9445E68BEA4B
:10FB000093E49F938F9389818F9388818F930E9431
:10FB100045E60E9465AC8DB79EB740968DBF9EBFEF
:10FB200080E0DF91CF910895CF93DF9386E893E44F
:10FB30009F938F93C6EDDAE589818F9388818F93A8
:10FB40000E9445E688E192E49F938F9389818F9389
:10FB500088818F930E9445E68DE890E49F938F9370
:10FB600089818F9388818F930E9445E685E794E48D
:10FB70009F938F9389818F9388818F930E9445E60D
:10FB80008BEA93E49F938F9389818F9388818F93DE
:10FB90000E9445E68DB79EB744968DBF9EBF80E01C
:10FBA000DF91CF910895CF93DF938CE690E49F93FC
:10FBB0008F93C6EDDAE589818F9388818F930E94B8
:10FBC00045E68EEE9CE39F938F9389818F93888186
:10FBD0008F930E9445E68BEA93E49F938F938981EC
:10FBE0008F9388818F930E9445E68DB79EB70C96C0
:10FBF0008DBF9EBF80E0DF91CF910895CF93DF93BB
:10FC000086EC9CE39F938F93C6EDDAE589818F9311
:10FC100088818F930E9445E685E59CE39F938F93AF
:10FC200089818F9388818F930E9445E68BEA93E4C4
:10FC30009F938F9389818F9388818F930E9445E64C
:10FC40008DB79EB70C968DBF9EBF80E0DF91CF91A0
:10FC50000895CF93DF9382E39CE39F938F93C6ED48
:10FC6000DAE589818F9388818F930E9445E689E048
:10FC70009CE39F938F9389818F9388818F930E94B8
:10FC800045E68BEA93E49F938F9389818F938881D4
:10FC90008F930E9445E68DB79EB70C968DBF9EBF91
:10FCA00080E0DF91CF9108952F923F924F925F9223
:10FCB0006F927F928F929F92AF92BF92CF92DF927C
:10FCC000EF92FF920F931F93CF93DF93CDB7DEB7E1
:10FCD0006A97CDBFDEBF5C010E9431652C011F8693
:10FCE000188A198A1A8AF50101900020E9F73197DC
:10FCF000EA19FB09E130F24008F002C2D5018C910B
:10FD0000882359F17501BFEFEB1AFB0A850120E04A
:10FD1000211115C0883229F08132C8F08F37B9F02F
:10FD200001C021E06801EFEFCE1ADE0A90E02A8FD1
:10FD30000E944FE5D8018C9386012A8D08C021E0EE
:10FD4000893209F420E0F80180830F5F1F4FD7014B
:10FD50008D917D018111DCCF01C08501F8011082F8
:10FD600010921E3EFDE19F2EAAE36A2EA2E27A2E99
:10FD7000812CB6E02B2E03C09A9409F49CC18BE72A
:10FD80009CE2A2E2B0E08B879C87AD87BE876B8A3E
:10FD90007C8A8D8A8DE79CE2A2E2B0E08F8398870F
:10FDA000A987BA87E3E1F2E2DE011196822D019084
:10FDB0000D928A95E1F7C2010E9438648501075FC0
:10FDC0001F4F75019FEFA91AB90AD7016C9170E016
:10FDD000CE010B960E94ACE5892B21F487010E5DC4
:10FDE0001F4F04C0A016B10661F793C16501BFEFB4
:10FDF000AB1ABB0AF601608170E0CE0143960E9407
:10FE0000ACE5892B91F0D6011D928D0192012F5EF8
:10FE10003F4F288F398F46E050E0B701C9010E945B
:10FE2000D7E53AE0C30ED11C04C0A016B106F1F626
:10FE300070C15801D8013D908D01E32CF12CC70110
:10FE40000E9433E5892B59F4B701CE0101960E9437
:10FE5000ACE5892B21F40C151D0559F75AC1850114
:10FE6000BEE63B1641F0E2E23E120CC0D50111960F
:10FE70008C918232A9F5F2011782118612861386BF
:10FE80001486A3C0B0E3EB1AF108EAE0EE16F10421
:10FE900018F0FDE23F1217C0BE016A5E7F4FC50138
:10FEA0000E94D6E1D20119966D937D938D939C9318
:10FEB0001C978E899F898A159B0509F42DC1E4E062
:10FEC0001796EC9382C0FBE73F124FC0E7E0D201E8
:10FED0001796EC93FFEFAF1ABF0AE2E0FE2E95C033
:10FEE0002FEFA21AB20AE5E0D2011796EC9362E274
:10FEF00070E0C5010E94ACE58E8B9F8B009709F4E2
:10FF000008C1DC011C92F50101900020E9F731974E
:10FF1000EA19FB093397C8F0F80181818033A9F40D
:10FF20008281883791F440E050E060E070E0C501E4
:10FF30000E9447E3D20119966D937D938D939C9314
:10FF40001C9783E017968C9308C0B501C2010E94EC
:10FF5000F16580931E3E811153C0AE88BF88BFEF0C
:10FF6000AB1ABB0AAE8ABF8A30C0E4E73E120EC0AD
:10FF7000E1E0D2011796EC9380E090E0A0E8BFE3C7
:10FF8000F20181879287A387B4871FC0F6E63F12EC
:10FF90000CC0E1E0D2011796EC93179719961D92C9
:10FFA0001D921D921C921C9710C0BBE53B12B1C064
:10FFB000F2012782B501C2010E94F16580931E3EC5
:10FFC00081111EC077E6F72E7DC0BE01695F7F4FAD
:10FFD000C5010E94F1E55C01009709F49AC0DC01BB
:10FFE0008C918D3729F411968C91F50131965F0132
:10FFF0008C3209F48BC0FFEFAF1ABF0AF12C05C099
:020000021000EC
:10000000F82E22E0281708F45DC08F858201035F77
:100010001F4F882341F043E050E0BE01615F7F4FF6
:10002000C8010E94D7E5688D798DC8010E9491634F
:10003000D20114968D939C9315978F3FBFEF9B072A
:10004000B9F10E94E068882371F0888D998D0E9433
:100050007A63882341F043E050E0688D798DCE01CA
:100060000F960E94D7E5F20142805380411451045B
:1000700011F1F11081CE8091B635811108C08FEA5F
:1000800095E30E942D6080931E3EF82E1BC0809148
:10009000C832823099F08FEA95E30E940360809322
:1000A0001E3E81110EC08FEA95E30E9480600AC057
:1000B00064E6F62E07C050E7F52E04C04BECF42E94
:1000C00001C0F82E42E060E08F2D0E94986681E02A
:1000D0000E94C4AE6A96CDBFDEBFDF91CF911F9163
:1000E0000F91FF90EF90DF90CF90BF90AF909F90D7
:1000F0008F907F906F905F904F903F902F900895DA
:100100008BE680931E3E3BE6F32EDCCF22E0F22E00
:100110007CCF9FE6F92ED6CF86E6F82ED3CF2F924E
:100120003F924F925F926F927F928F929F92AF9287
:10013000BF92CF92DF92EF92FF920F931F93CF93D4
:10014000DF9300D000D0CDB7DEB78C0169837A830E
:100150004B835C835A0128E0A21AB108A60EB71E91
:10016000DC0116967C907B01BFEFEB1AFB0A8BE754
:10017000FB01808380E0912C95E0692E2DE1422ED9
:1001800022E2522E39E1232E32E2332E4DE7842E25
:10019000ED82FE82D80117969C919F3F09F429C1F8
:1001A000882339F02CE2ED81FE8120833196ED83A6
:1001B000FE838091C83D811119C0C80141969F936B
:1001C0008F933F922F923E813F938D818F930E9418
:1001D00010E7AD81BE81A80FB91FAD83BE830F901C
:1001E0000F900F900F900F900F9018C0C80141967C
:1001F0009F938F935F924F92BE81BF93ED81EF9358
:100200000E9410E72D813E81280F391F2D833E83E8
:100210000F900F900F900F900F900F90D80117969E
:100220008C911797843059F51996CD90DD90ED900B
:10023000FC901C97A7019601C701B6010E9431DD11
:10024000811117C0E894F7F82FEF3FEF4FE75FE712
:10025000C701B6010E9431DD811121C12FEF3FEFAF
:100260004FE75FE7C701B6010E946BD918160CF083
:1002700016C1F801118612861386148610C18111E9
:1002800013C0E3E2F2E2AD81BE81862D01900D92B2
:100290008A95E1F72D813E812C5F3F4F2D833E8370
:1002A000D80117968C9199C0823061F4F801848549
:1002B0008F9383858F9382858F9381858F93A8E217
:1002C000B2E214C0833029F5D8011C968C911C979A
:1002D0008F931B968C911B978F931A968C911A97DC
:1002E0008F9319968C918F93AEE2B2E2BF93AF9346
:1002F000FE81FF932D812F930E9410E7AD81BE8177
:10030000A80FB11DAD83BE83F8018781CDBFDEBFCD
:1003100064C0853059F4D80158968C9158978F93C2
:1003200057968C918F93A6E3B2E20CC0863009F504
:10033000D80158968C9158978F9357968C918F939C
:10034000ABE3B2E2BF93AF93FE81FF932D812F9376
:100350000E9410E7AD81BE81A80FB11DAD83BE83A1
:10036000F80187810F900F900F900F900F900F90D2
:1003700034C0813091F52CEA35EC47E257E3D801DF
:1003800019966D917D918D919C911C970E946BD9CE
:1003900087FF12C0E0E4F2E2AD81BE8186E0019009
:1003A0000D928A95E1F7ED81FE813596ED83FE830E
:1003B000D80117968C9111C0E6E4F2E2AD81BE81BE
:1003C000862D01900D928A95E1F7ED81FE8134969C
:1003D000ED83FE83D80117968C91873049F42BE783
:1003E000ED81FE8120833196ED83FE8380E001C0A4
:1003F00081E0AD81BE81AA15BB0518F08FEF9FEF9C
:1004000065C0F801028113810115110549F0D80179
:1004100016969C912FEF290D99153CF0992EBACE86
:10042000ED80FE807914B4F020C0ED81FE81D8010A
:10043000CF010196808216969C9016973FEF320F5F
:1004400092161CF4232FFC01F3CF8D839E838D0124
:1004500081E0A0CEF7012DE7CF01019620839A9489
:10046000791414F4FC01F8CF7C018DE79AE0A0E048
:10047000F70180839183A283F2E0EF0EF11C898162
:100480009A812B813C81820F931F8E159F0508F462
:10049000B5CFC701A981BA818A1B9B0B17C0C801C0
:1004A0000E94F068F8014185528563857485208536
:1004B0008D819E810E947AC82D813E81280F311D39
:1004C0002D833E83D80117968C9187CF2696CDBF7A
:1004D000DEBFDF91CF911F910F91FF90EF90DF90E2
:1004E000CF90BF90AF909F908F907F906F905F90D4
:1004F0004F903F902F90089540E052E064E47BE3FA
:100500000E948F806091D65A7091D75A84E49BE301
:100510000C9494E6EF92FF920F931F93CF93DF9387
:10052000CDB7DEB76297CDBFDEBFF82E9091C63D46
:10053000992309F4B2C08FE6F81212C00E94316507
:1005400064E47DE380913E3B90913F3B0E945AC81A
:10055000BC018CE091E20E944F660FEA15E34AC0AD
:100560008091C8320FEA15E3882309F443C0EE24D2
:10057000EA94C8010E94F8638823E1F1823029F4EB
:100580008091CD3D811120C01DC0843029F480911F
:10059000CA3D811119C016C08530B1F48091CC3D9F
:1005A000882381F0F80181859285A385B485BC01FB
:1005B000CD019F772CEA35EC47E257E30E946BD9D7
:1005C00087FF02C0F801E782F8010281138101155B
:1005D000110579F60FC0F80102811381011511058B
:1005E00049F440E052E064E47BE386E995E30E944D
:1005F0008F8053C0F80197819F3F69F78091BF2991
:1006000081111AC08091413B8F938091403B8F9321
:100610001F92FF928BE492E29F938F93CE010196FB
:100620007C01FF928F930E9410E71092403B109242
:10063000413BCDBFDEBF13C00E94FACC1F928F9307
:100640001F92FF9283E592E29F938F93CE010196D2
:100650007C01FF928F930E9410E7CDBFDEBFB701F0
:10066000C8010E94F165F801168286E0878386E65C
:1006700090E0818B928B1282138240E052E064E41E
:100680007BE386E995E30E948F806091D65A709152
:10069000D75A84E49BE30E9494E66296CDBFDEBF06
:1006A000DF91CF911F910F91FF90EF9008956130EE
:1006B00019F0623029F008958FEA95E30C947C825A
:1006C0000C948A82CF92DF92EF92FF92FC01C18458
:1006D000D284E384F48420E030E040EA50E4C701AF
:1006E000B6010E946EDB18160CF453C0C701B601A8
:1006F0000E94DFD96093C63D1092C93D1092CA3D59
:100700001092CB3D1092CC3D1092CD3D20E030E0D8
:1007100040E85FE3C701B6010E946EDB87FD03C0BE
:1007200081E08093C93D20E030E040E050E4C70123
:10073000B6010E946EDB87FD03C081E08093CA3D55
:1007400020E030E040E450E4C701B6010E946EDBD7
:1007500087FD03C081E08093CB3D20E030E040E89E
:1007600050E4C701B6010E946EDB87FD03C081E043
:100770008093CC3D20E030E040EA50E4C701B60170
:100780000E946EDB87FD07C081E08093CD3D80E055
:1007900003C08EE601C080E0FF90EF90DF90CF9025
:1007A000089565ED77E40C94F7C56EE777E40C9453
:1007B000F7C56AE477E40C94F7C5BF92CF92DF9255
:1007C000EF92FF920F931F93CF93DF93CDB7DEB7D6
:1007D0006897CDBFDEBF6B0128E1FC01DE011196F9
:1007E00001900D922A95E1F789E8E82E81E3F82E31
:1007F0008E010F5F1F4FB12CF7018081823029F4E9
:10080000F8011082118212821382809158598B1143
:1008100014C020916B5930916C5940916D59509191
:100820006E59F80160817181828193810E9410DC90
:10083000F6016083718382839383809177598B1152
:1008400014C020918A5930918B5940918C59509104
:100850008D59F80160817181828193810E9410DC41
:10086000F6016483758386839783809196598B11F3
:1008700014C02091A9593091AA594091AB59509177
:10088000AC59F80160817181828193810E9410DCF2
:10089000F60160877187828793878091B5598B11A4
:1008A00014C02091C8593091C9594091CA595091EA
:1008B000CB59F80160817181828193810E9410DCA3
:1008C000F6016487758786879787B394F5E3EF0E03
:1008D000F11C0C5F1F4F86E0B8128ECF6896CDBF1B
:1008E000DEBFDF91CF911F910F91FF90EF90DF90CE
:1008F000CF90BF900895F8940E94A07C0E94D2846B
:100900000E9434D70E9456CA0E945EB70E94247487
:100910000E94A3C00E94BAA940E060E080E00E946B
:10092000D6690E946E650E94C0840E94C4860E949F
:10093000BC530E942CD78091A20084608093A200B7
:100940008091A20082608093A2008091A2008160C9
:100950008093A20078940E9465AC0E94B8C10E9466
:100960003D6AFDCFE82FF0E0EE0FFF1FEF5FF74B82
:10097000659174914FE450E08EEC9DE30C947EE51C
:1009800080911F3B823041F440E060E081E00E94B2
:10099000D66980E00E94656B0C94F8CD682F81E0E9
:1009A0000C9449CB10921F3E1092203E1092213E93
:1009B0001092223E0895CF93DF93EC018C819D81AC
:1009C000880F991F880F991F2091213E3091223E58
:1009D000820F931F8093233E9093243E44E050E087
:1009E00069E27EE30E942CD64091293E50912A3E36
:1009F00060912B3E70912C3E49875A876B877C878C
:100A000080E0DF91CF9108958F929F92AF92BF9235
:100A1000CF92DF92EF92FF92CF93DF93EC01809120
:100A2000C932882369F089E0DF91CF91FF90EF9080
:100A3000DF90CF90BF90AF909F908F900C94EDABD4
:100A400089859A85AB85BC858093253E9093263E0B
:100A5000A093273EB093283ECE010E94DB84809372
:100A60001E3E81116EC0C984DA84EB84FC84A70128
:100A70009601C701B6010E9431DD81112FC04601E8
:100A80005701E894B7F82FEF3FEF4FE75FE7C50155
:100A9000B4010E9431DD81110AC02FEF3FEF4FE713
:100AA0005FE7C501B4010E946BD91816BCF08090B5
:100AB000253E9090263EA090273EB090283EA5016E
:100AC0009401C701B6010E94C2D79F772CEA35EC8A
:100AD00047E257E30E946EDB181674F58091253EBD
:100AE0009091263EA091273EB091283E8093293ECA
:100AF00090932A3EA0932B3EB0932C3E8C819D81F7
:100B0000880F991F880F991F2091213E3091223E16
:100B1000820F931F8093233E9093243E44E050E045
:100B200069E27EE30E94BDD68090253E9090263EED
:100B3000A090273EB090283E89869A86AB86BC86D8
:100B400080E0DF91CF91FF90EF90DF90CF90BF904A
:100B5000AF909F908F9008950E94B9BC80E0089557
:100B600080912D3E90912E3E8F3E924111F08EE568
:100B700008958091533E9091543E8F3E9241B9F733
:100B80008091553E9091563E8F3E924181F78091E3
:100B9000DE559091DF558F3E924149F78091E055A7
:100BA0009091E1558F3E924111F78091735790914A
:100BB00074578F3E9241D9F680E0089594E0899F62
:100BC000F0011124E35DF14C428353836483758308
:100BD000089594E0899FF0011124E052FA4A45AB50
:100BE00056AB67AB70AF08955F926F927F928F9212
:100BF0009F92AF92BF92CF92DF92EF92FF920F93AC
:100C00001F93CF93DF93CDB7DEB76097CDBFDEBF25
:100C1000BE016F5F7F4F85E196E50E94DD83CE01C7
:100C200001964C018DE8A82E86E5B82E9DE9C92EC7
:100C300096E5D92E2DEAE22E26E5F22E0DEC16E5EC
:100C40003FEE632E39E5732E512CF4014191519101
:100C5000619171914F01F5014193519361937193AA
:100C60005F01F60141935193619371936F01F70115
:100C700041935193619371937F01852D0E94467436
:100C8000F80111921192119211928F01F3011082C9
:100C90001182128213825394F8E16F0E711C84E06A
:100CA0005812D3CF6096CDBFDEBFDF91CF911F9199
:100CB0000F91FF90EF90DF90CF90BF90AF909F90FB
:100CC0008F907F906F905F9008958091573E089528
:100CD0001F93CF93DF938BE897E1E5E5FEE3DF0118
:100CE0009C011D9221503040E1F78FEE92E18093FC
:100CF000553E9093563E8093DE559093DF55CEE55A
:100D0000DEE3C093583ED093593EC0935A3ED093F1
:100D10005B3EC0935C3ED0935D3E81E090E062E23A
:100D200075E520E030E01CEB129FA001139F500DF1
:100D30001124FA01EB5AF14CD90111961A9F900136
:100D40001B9F300D1124225A314C23873487618731
:100D50007287BA01625A714C9C01019680329105EA
:100D600019F78CEB829FF001839FF00D1124EB5A51
:100D7000F14CC387D4876187728780E28093573EA6
:100D8000DF91CF911F910895CF93DF93E0EEF5E5CA
:100D900085E991E0DF01EC011D922197E9F7ADE2D1
:100DA000BEE388E2ED0119928A95E9F78FEE92E1B0
:100DB0008D939C938093533E9093543E8083918374
:100DC0008093735790937457DF91CF910C946886FA
:100DD0000E94E1900E94688680E00C94CD4EE091E4
:100DE000583EF091593E848581111BC02281338188
:100DF000808191814CEBDF011D924A95E9F72283B6
:100E000033838083918381E084878091573E815032
:100E10008093573E828193818093583E9093593EB0
:100E200005C08CE10E94EDABE0E0F0E0CF01089559
:100E3000AAE5BEE3ED91FC911197858781E0878754
:100E400082E08487828193818D939C9381E00E94CC
:100E500015B00C94FFB9EF92FF920F931F93CF93AD
:100E6000DF9300D01F92CDB7DEB78C014B835C833C
:100E700069837A830E94EF86FC014B815C816981E2
:100E80007A81009761F48EE02496CDBFDEBFDF91BA
:100E9000CF911F910F91FF90EF900C940C5383E032
:100EA00085878CEA95E884839583068317838B0175
:100EB0007A0126E0D8014D915D916D917D918D0172
:100EC000CF0185599F4FDC014D935D936D937C93CA
:100ED0001397D7014D915D916D917D917D01418B6E
:100EE000528B638B748B215034962111E3CF83E0B6
:100EF0002496CDBFDEBFDF91CF911F910F91FF9060
:100F0000EF900C941887CF92DF92EF92FF926B01D3
:100F10007C010E94EF86009739F48EE0FF90EF90FD
:100F2000DF90CF900C940C5326E038E8FC0124832A
:100F30003583E556FF4FC082D182E282F38221E001
:100F4000FC01278782E00E94188780E0FF90EF90E5
:100F5000DF90CF90089580915C3E90915D3EFC01C2
:100F600024853EEF320F323018F424E024870895B0
:100F7000243011F080E090E00895E0915C3EF09123
:100F80005D3E22813381808191814CEBDF011D9296
:100F90004A95E9F72283338380839183E0915C3E15
:100FA000F0915D3E0280F381E02DE0935C3EF09392
:100FB0005D3E8485823011F483E084878091573EC2
:100FC0008F5F8093573E8FEF0E9415B081E0409174
:100FD000583E5091593E20915C3E30915D3E421703
:100FE000530709F080E00895BC016F5E7F4FDC017C
:100FF0001696ED91FC91179785599F4F19950E9470
:10100000BD8781110E94275A80E0089585569F4F21
:1010100020E034E244E759E4FC016081718182817F
:1010200093810E9410DC0E94DFD90E940BDA0E949B
:10103000C3BC0E94BD8781110E94275A80E0089599
:1010400080915C3E90915D3EFC0124853EEF320F25
:10105000323018F424E024870895243011F080E021
:1010600090E00895CF93DF93C0915C3ED0915D3EB8
:101070008C859EEF980F923018F484E08C8705C021
:10108000843019F080E090E010C02097D9F3DE01A1
:101090001296ED91FC9113978785882329F0EC1720
:1010A000FD0711F0DF01F4CFCD01DF91CF9108955D
:1010B000CF93DF93EC012A813B81888199814CEBAE
:1010C000FB01DE0101900D924A95E1F72A833B83F3
:1010D00088839983DF91CF9108958FEE92E1809379
:1010E000755790937657809332589093335808955C
:1010F0002F923F924F925F926F927F928F929F9228
:10110000AF92BF92CF92DF92EF92FF920F931F9315
:10111000CF93DF93CDB7DEB76A97CDBFDEBF4C016B
:101120001B0129013A01E986FA860B871C871A2DD3
:101130000B2DE8A8B9A8AAA82BA92983809141332F
:10114000882399F08091353390913633A0913733CD
:10115000B0913833BC01CD019F772CEA35EC47E2E2
:1011600057E30E946BD987FD11C780916C34909131
:101170006D34A0916E34B0916F34BC01CD019F7776
:1011800031E03D832CEA35EC47E257E30E946EDB09
:10119000181614F01D8210C02DEC3CEC4CEC5DE3F5
:1011A0006091113470911234809113349091143401
:1011B0000E946BD987FDECC6F10180819181A281EB
:1011C000B381BC01CD019F77F1E0FD872CEA35ECBE
:1011D00047E257E30E946EDB18160CF01D86F10102
:1011E00084819581A681B781BC01CD019F77F1E013
:1011F000F98B2CEA35EC47E257E30E946EDB1816B8
:101200000CF0198AF10180859185A285B385209122
:1012100070343091713440917234509173342E8B0C
:101220003F8B488F598F20917434309175344091A1
:101230007634509177342A8B3B8B4C8B5D8B40916D
:1012400078345091793460917A3470917B34F09095
:101250004233F11021C01092BD5781E08093BE57F8
:1012600082E08093BF573D81332341F04D8541118A
:1012700095C65989511192C68CE9C1C6CB01BA01F4
:101280009F772CEA35EC47E257E30E946EDB181695
:101290000CF089C68BE9B3C6BC01CD019F77A1E0F4
:1012A000AA8F2CEA35EC47E257E30E946EDB181652
:1012B0000CF01A8EB1E0FB1216C01092BD5782E0FE
:1012C0008093BE57F092BF57ED81EE2339F0FD8534
:1012D000F11164C62A8D222379F260C66A897B895E
:1012E0008C899D89CDCF32E0F31217C081E08093C5
:1012F000BD57F092BE571092BF574D81442341F025
:10130000598951114BC68A8D882309F4B5CF46C639
:101310006E897F89888D998DB3CFB101C4010E94F8
:101320001C519D81992309F451C02091FD323091C7
:10133000FE324091FF3250910033609152337091F0
:10134000533380915433909155330E94C2D79F7785
:101350002CEA35EC47E257E30E946BD987FF36C091
:101360002091013330910233409103335091043383
:10137000609156337091573380915833909159331F
:101380000E94C2D79F772CEA35EC47E257E30E94D0
:101390006BD987FF1BC020910533309106334091F4
:1013A00007335091083360915A3370915B338091C9
:1013B0005C3390915D330E94C2D79F772CEA35EC65
:1013C00047E257E30E946BD987FDE4C58CA980935F
:1013D000FC3288EF92E30E94244F86E5E8EFF2E3C7
:1013E000ACEDB7E501900D928A95E1F788E1E2E571
:1013F000F3E3A8E7B7E501900D928A95E1F78091B4
:1014000043338111D5C523E333E34BEC51E46E2D17
:101410007B2D8A2D99810E9410DC4B015C01609329
:10142000A8577093A9578093AA579093AB5723E37B
:1014300033E34BEC51E4C301B2010E9410DC609332
:10144000905770939157809392579093935723E3BB
:1014500033E34BEC51E469857A858B859C850E944A
:1014600010DC6093945770939557809396579093A0
:10147000975723E333E34BEC51E4612F702FC60100
:101480000E9410DC162F072F412F502FBC014093D4
:1014900098575093995760939A5770939B578091A0
:1014A0000D3490910E34A0910F34B0911034BC01E2
:1014B000CD019F770E9448DA0E94DFD96093B95727
:1014C0007093BA578093BB579093BC57A091BD5768
:1014D000A98BB091BE57BA8BEB2FF0E0ED83FE8362
:1014E0007F01EE0CFF1CEE0CFF1CF101EE0DFF1D49
:1014F00080819181A281B381BC01CD019F772CEACB
:1015000035EC47E257E30E946BD9D82EDD1CDD2471
:10151000DD1C3989232F30E029833A838901000FAC
:10152000111F000F111FF101E00FF11F8081918148
:10153000A281B381BC01CD019F772CEA35EC47E253
:1015400057E30E946BD9881F8827881F8D218093BD
:10155000B8572CEA35EC47E257E3C501B4019F7751
:101560000E946EDB18160CF0F9C0F801E350FD4C38
:10157000D801AE5ABC4C2D913D914D915C9160814A
:101580007181828193810E94C2D76B017C01ED81C0
:10159000FE81EE0FFF1FEE0FFF1FE350FD4CAD81EC
:1015A000BE81AA0FBB1FAA0FBB1FAE5ABC4C2D9108
:1015B0003D914D915C9160817181828193810E9406
:1015C000C2D769877A878B879C87A5019401C5015B
:1015D000B4010E9410DC20E030E040E850E40E94BA
:1015E00010DC6D877E878F87988BA7019601C701D6
:1015F000B6010E9410DC2B013C0129853A854B8500
:101600005C85CA01B9010E9410DC9B01AC01C301D9
:10161000B2010E94C3D79B01AC016D857E858F8589
:1016200098890E94C2D72B013C0120E030E0A9013B
:101630000E946EDB1816C4F4C301B2010E94E9DCFB
:101640002B013C0129853A854B855C85C701B60194
:101650000E947BDB9B01AC01C301B20190580E9448
:1016600072D92B013C0103C0412C512C32018091D5
:10167000FC32833021F477FA709477F8709420E08C
:1016800030E0A901C501B4010E946BD987FF04C0F5
:1016900077FA709477F8709409811A81000F111FFE
:1016A000000F111FA8014B58584A5A01A30192017B
:1016B00069857A858B859C850E9410DC9B01AC0135
:1016C000C701B6010E94C2D720E030E040E05FE3EE
:1016D0000E9410DCD5015B966D937D938D939C9356
:1016E0005E97AD80BE80AA0CBB1CAA0CBB1CF5018A
:1016F000EB58F84A4F01A3019201C701B6010E94BD
:1017000010DC9B01AC0169857A858B859C850E94E4
:10171000C3D720E030E040E05FE30E9410DCD4015A
:101720005B966D937D938D939C935E97E091BF57ED
:10173000F0E0EE0FFF1FEE0FFF1FEB58F84A138E7D
:10174000148E158E168EB091A857B987E091A957BF
:10175000ED872090AA573090AB5725C05701F7016D
:10176000EB58F84A838D948DA58DB68D9C01AD0103
:101770005058F801EB58F84A838D948DA58DB68D9D
:10178000BC01CD0190580E947BDB9B01AB01BC01E9
:101790004093A8575093A9576093AA577093AB579B
:1017A00029873D871C01D801AB58B84A5B96CD907C
:1017B000DD90ED90FC905E97E981FA81EE0FFF1FBE
:1017C000EE0FFF1FEF51F84A13962D913D914D9169
:1017D0005C91169760817181828193810E94C2D74A
:1017E000A70196010E94C2D769837A838B839C8369
:1017F000D501AB58B84A5B964D905D906D907C904A
:101800005E97ED81FE81EE0FFF1FEE0FFF1FEF5180
:10181000F84A13962D913D914D915C9116976081F8
:101820007181828193810E94C2D7A30192010E949B
:10183000C2D76D837E838F8398879B01AC016981BA
:101840007A818B819C810E947BDB29853D85A1016A
:101850000E94C2D74B015C01E894B7F820E030E069
:1018600040E85FE3C501B4010E946EDB18160CF47A
:10187000C3C32AE037ED43EA5BE3C501B4010E942C
:101880006EDB181694F42FE632E143E85AE36985DB
:101890007D85C1010E9410DC9B01AC01C501B40132
:1018A0000E946EDB18160CF4A7C3A30192015058D6
:1018B000C701B60190580E9436D84B015C01609375
:1018C000A0577093A1578093A2579093A3578091EC
:1018D0004233813039F4412C512C30E8632E3FEBF8
:1018E000732E06C0412C512C20E8622E2FE3722E5D
:1018F0008091B8578823D1F16091B9577091BA5748
:101900008091BB579091BC570E940BDA6B017C0110
:101910002CEA35EC47E257E30E946BD987FD10C0F3
:101920001091FC322BED3FE049EC50E4C701B601C9
:101930000E9410DC9B01AC01C12CD12C7601B9C0F6
:1019400081E090E0A0E0B0E08093B9579093BA575F
:10195000A093BB57B093BC571091FC322BED3FE0E6
:1019600049EC50E4C12CD12C7601A3C02D813E81DD
:101970004F81588569817A818B819C810E9436D8FC
:1019800069837A838B839C836093A4577093A55754
:101990008093A6579093A757A50194010E94C2D7A0
:1019A0006B017C019F772CEA35EC47E257E30E94FC
:1019B0006BD987FF18C01091FC326091B9577091B4
:1019C000BA578091BB579091BC570E940BDA2BED10
:1019D0003FE049EC50E40E9410DC9B01AC01C12CBB
:1019E000D12C760166C029813A814B815C81C50189
:1019F000B4010E946EDB1816F4F42BED3FE049ECC5
:101A000050E4C301B2010E9410DC9B01AC0169816A
:101A10007A818B819C810E94C3D76093A457709375
:101A2000A5578093A6579093A757A50194010E94AC
:101A3000C2D76B017C011091FC32133099F0609198
:101A4000B9577091BA578091BB579091BC570E947B
:101A50000BDA2BED3FE049EC50E40E9410DC9B01D7
:101A6000AC0127C02BED3FE049EC50E4C301B201CB
:101A70000E9410DC9B01AC01C701B6010E94C2D7D5
:101A80007B018C016091B9577091BA578091BB5717
:101A90009091BC570E940BDA2BED3FE049EC50E4EB
:101AA0000E9410DC9B01AC01C701D8016C017D01D3
:101AB0000BC0123049F4C301B2010E9410DCA7012F
:101AC00096010E94C3D70AC0C301B2010E9410DC74
:101AD0009B01AC01C701B6010E94C2D77B01AB01DB
:101AE000BC014093AC575093AD576093AE57709381
:101AF000AF578C015090BF57A52DB0E0FD01EE0F00
:101B0000FF1FEE0FFF1FEF51F84AAA0FBB1FAA0FCE
:101B1000BB1FAB58B84A13962D913D914D915C91E6
:101B2000169760817181828193810E94C2D74B0197
:101B30005C016093B0577093B1578093B257909304
:101B4000B3579701A80169857D85C1010E9410DC0A
:101B50006B017C016093B4577093B5578093B6576F
:101B60009093B757A50194010E947BDB69837A8328
:101B70008B839C8360939C5770939D5780939E5753
:101B800090939F5780914133811117C0F091353365
:101B9000FD8340903633209137332E8B309138338C
:101BA0003A8F1092353310923633109237331092A9
:101BB000383381E08093413312C020913533309126
:101BC0003633409137335091383369817A818B8134
:101BD0009C810E9472D96D83472E8E8B9A8F598972
:101BE00045E3549FF0011124E657FE4C20813181DA
:101BF00042815381C701B6010E9472D9662E072F18
:101C0000182F792E2D81342D4E895A8D0E946BD933
